:020000040800F2
:10000000000001203D760008EF330008F1330008BE
:10001000F3330008F5330008F73300080000000050
:10002000000000000000000000000000F93300089C
:10003000FB33000800000000FD330008FF33000818
:100040008D7600088D760008013400088D76000852
:100050008D7600088D7600080D3400081D340008E8
:100060008D7600082D3400088D76000835340008A0
:10007000413400084D3400088D7600088D76000864
:10008000593400085D3400088D7600088D7600082C
:10009000000000008D760008693400088D760008A5
:1000A0008D7600088D7600088D7600088D76000824
:1000B0008D7600088D7600088D7600088D76000814
:1000C0008D7600088D7600086D3400088D76000866
:1000D0008D760008793400088D7600088D7600084A
:1000E0008D7600088D760008853400088D7600082E
:1000F0008D76000800000000000000008D760008EA
:100100008D7600088D760008913400088D76000801
:100110008D7600088D7600088D7600088D760008B3
:100120008D7600088D7600088D7600088D760008A3
:080130008D7600088D760008B1
:1001400010B5054C237833B9044B13B10448AFF311
:1001500000800123237010BDC807002000000000AC
:100160003C1B030808B5034B1BB103490348AFF31D
:10017000008008BD00000000CC0700203C1B0308E5
:1001800014214160704714207047406A7047000096
:1001900081010008870100088B010008A101000807
:1001A00010B5044604F1100000F05CFCC4F8F8003F
:1001B0000148C4F87C0110BD90010008F8B5E6B014
:1001C00004460D4616461F460A4906A800F0CAFE18
:1001D00070996F9A05910492009733466E996D9AC3
:1001E000039102922A466C990191214600F060F831
:1001F00067B0F0BD9C010008F8B5E6B004460D46B6
:1002000016461F46094906A800F0ACFE6F996E9A83
:100210000491039200976D996C9A02910192334672
:100220002A46214600F087F867B0F0BD9C0100081F
:1002300038B500281CBF01680029184A23D1184B83
:100240001C684FF6F0710C404CF24025AC421FBFC9
:100250001B6819404CF27024A14212D1114D29683B
:1002600079B911490B68C3F30B03B3F58A6F1FBF4C
:100270000968C1F30B0140F28343994204BF012195
:10028000117028B905E0094B994204BF0121117092
:100290004068BDE8324002F073BC00BFE4070020B4
:1002A00000ED00E0002004E00010005C0000374892
:1002B0002DE9F04104460D46216816464A681F465E
:1002C00090478046B8F5403F2ED122680A9993683E
:1002D000204698478046B8F5403F25D12368089AC4
:1002E0000799D3F80CC02046E0478046B8F5403F58
:1002F0001AD12368069A39461F692046B8478046B6
:10030000B8F5403F10D1236829465D693246204642
:10031000A8478046B8F5403F06D123680B9A099953
:100320009D692046A847804621680A682046904774
:100330004046BDE8F0812DE9F04104460D462168B4
:1003400016464A681F4690478046B8F5403F2ED172
:1003500022680A999368204698478046B8F5403F3E
:1003600025D12368089A0799D3F80CC02046E047A6
:100370008046B8F5403F1AD12368069A39461F696E
:100380002046B8478046B8F5403F10D1236829463B
:100390005D6932462046A8478046B8F5403F06D101
:1003A00023680999DD6900222046A8478046216814
:1003B0000A68204690474046BDE8F0814FF440303F
:1003C00070470000F0B50C4685B0114600281A466B
:1003D0001CBF0568002D0B4B11D082B104B971B957
:1003E0000D9860B10F9E0E9F0A9B02900496039792
:1003F0000B980C9E009001962046A847034618468D
:1004000005B0F0BD020003002DE9F04F0646D0B064
:100410000868F56DD6F860E0726EB76EF36E00BADC
:1004200000906C46486800BA60600DF1400888682A
:1004300000BAA060C86800BAE060086900BA20612C
:10044000486900BA6061886900BAA061C86900BAE9
:10045000E061086A00BA2062486A00BA6062886A8D
:1004600000BAA062C86A00BAE062086B00BA2063F2
:10047000486B00BA6063886B00BAA063C86B00BAAF
:10048000E063402058F80C1C58F820CC58F838ACE1
:100490008CEA010158F840CC8AEA01018CEA010992
:1004A0004FEAF979401E48F8049BEBD187EA020035
:1004B00000EA0E00784010EBF5610098DFF824C4E4
:1004C00041186144C81882EABE032B404FEAF0612C
:1004D00053405918636859186144CF194FEAB5035E
:1004E00083EABE01014081EABE0111EBF765A16814
:1004F0004D196544A91883EAB0023A404FEAF16504
:100500005A405519E26855194FEAB70282EAB00716
:1005100065440F4005EBBE0E97EAB00717EBFE658A
:1005200027697D194FEAB10782EA0701654401EAAC
:100530000E01EB18514011EBF36561694D194FEA5B
:10054000BE0187EA010E65440EEA030E15EBB0000A
:100550008EEA070E0EEBF065D4F818E0754465449A
:10056000AA1881EAB30505404FEAF26E4D40AE4449
:10057000E569AE44E64477444FEAB00080EAB30E42
:100580000EEA020E8EEAB30E0EEBF765D4F820E009
:1005900075446544691880EAB2053D404FEAF16E42
:1005A0004540AE44656AAE44E6440EEBB3034FEA01
:1005B000B70787EAB20E0EEA010E8EEAB20E0EEB14
:1005C000F365D4F828E075446544281887EAB10536
:1005D0001D404FEAF06E7D40AE44E56AAE44E6440D
:1005E0000EEBB2024FEAB30383EAB10E0EEA000E3D
:1005F0008EEAB10E0EEBF265D4F830E07544654436
:10060000EF1983EAB00515404FEAF76E5D40AE443E
:10061000656BAE44E6440EEBB1014FEAB20282EAEA
:10062000B00E0EEA070E8EEAB00E0EEBF165D4F8AE
:1006300038E075446544EB1882EAB7050D404FEA8F
:10064000F36E5540AE44E56BAE44E6440EEBB000AD
:100650004FEAB10181EAB70E0EEA030E8EEAB70E39
:100660000EEBF065D4F840E07544654481EAB30EC2
:10067000AA180EEA000E4FEAF2658EEA010E7544E2
:10068000DDF844E04FEAB000754480EAB30E6544FB
:100690000EEA020E15EBB7078EEAB30E0EEBF76506
:1006A000DDF848E04FEAB202754480EA020E654484
:1006B0000EEA070E69188EEA000E0EEBF165DDF802
:1006C0004CE07544654405EBB3034FEAB70E1427BD
:1006D0000DF1500CDFF810528EEA010B82EA0B0B81
:1006E0000BEBF36A5CF804BBDA44AA44504483EA97
:1006F000B10B4FEAF06A8EEA0B0BDA445CF804BBEC
:10070000DA44AA44524480EAB30B4FEAF26A8BEA15
:10071000B10BDA445CF804BBDA444FEAB000AA44F7
:1007200080EA020BD6448BEAB30B0BEBFE6A5CF853
:1007300004BBDA444FEAB202AA4482EA0E0B0AEB87
:10074000B10180EA0B0B0BEBF16A5CF804BBDA44F5
:100750007F1DAA44282F0AEBB3034FEABE0EBBD37A
:100760003C2F61D3502F4DD204EB870CC7F15407B7
:100770005E4CA7FB04A504465D4FA8088EEA010A5B
:1007800082EA0A0A5CF804BB0AEBF3655D447D1952
:100790002C1983EAB10A4FEAF4658EEA0A0A554435
:1007A0005CF804AB5CF804BB55447D19AA1884EAD4
:1007B000B30A4FEAF2658AEAB10A55445D444FEA4A
:1007C000B4047D1984EA020AAE448AEAB30A0AEB49
:1007D000FE655CF804AB55444FEAB2027D1982EA2B
:1007E0000E0A15EBB10184EA0A0A5CF804BB0AEBB5
:1007F000F1655D447D1915EBB303401E4FEABE0E53
:10080000BCD12046F46D1B19F365336EC9183166EF
:10081000716E71447166B36ED218B266F16E401893
:10082000F06650B0BDE8F08F4EEA010B0EEA010A07
:100830000BEA020B4BEA0A0A0AEBF36554F827A00D
:10084000DFF8B0C0554443EAB10B654403EAB10A8E
:100850000BEA0E0B28184BEA0A0A7F1C0AEBF0651C
:1008600054F827A0554440EAB30B654400EAB30AA4
:100870000BEAB10BAA184BEA0A0A7F1C0AEBF265D5
:1008800054F827A055444FEAB00040EA020B6544F3
:1008900000EA020A0BEAB30BAE444BEA0A0A7F1CD9
:1008A0000AEBFE6554F827A055444FEAB20242EA2B
:1008B0000E0B654402EA0E0A0BEA000B15EBB101C0
:1008C0004BEA0A0A7F1C0AEBF16554F827A055444D
:1008D0007F1C65443C2F05EBB3034FEABE0EA3D348
:1008E00040E700BF9979825AA1EBD96ECDCCCCCC30
:1008F000D6C162CADCBC1B8F00B581B00168074A53
:10090000914200D110B9064801B000BD7C212DF004
:10091000C4FE4FF4003001B000BD00BF040A00085F
:10092000030002002DE9F0410B4A92E8F85188B02B
:10093000694681E8F8510268084B9A4200D118B91B
:10094000074808B0BDE8F0811422083000F04FFBE2
:1009500008B0BDE8F08100BFE4090008040A0008FF
:1009600003000200152904D20268044B9A4200D108
:1009700008B903487047083000F048BB040A000873
:100980000300020010B481B013460268074CA24273
:1009900000D118B901B010BC0548704701B000F192
:1009A000240210BC083000F035BB00BF040A000868
:1009B0000300020010B481B013460268074CA24243
:1009C00000D118B901B010BC054870470A4601B003
:1009D00000F1240110BC083000F070BB040A0008CC
:1009E000030002000123456789ABCDEFFEDCBA9816
:1009F00076543210F0E1D2C3000000000000000085
:100A000000000000F9080008250900086509000831
:100A100085090008B509000809040008810F0008CD
:100A2000CD0F0008890F0008F0B5A3B004460B48AD
:100A300002900D4616461F46094B0822402104A885
:100A400000F0D1FA28980190009733462A462146B3
:100A500002A800F01BF823B0F0BD00BF040A000894
:100A6000180A000810B5040008BF002408D0054883
:100A7000054B20600822402104F1080000F0B3FA81
:100A8000204610BD040A0008180A00082DE9F041AC
:100A900004460E46216817464A681D469047804620
:100AA000B8F5003F19D12268069993682046984707
:100AB0008046B8F5003F10D123683146DE683A46DB
:100AC0002046B0478046B8F5003F06D12368079A14
:100AD00029461D692046A847804621680A682046A5
:100AE00090474046BDE8F08110B500F033FA4FF46E
:100AF000403400280EBF034C4FF4C0712DF0CDFDE3
:100B0000204610BD0200030010B5044600F022FA92
:100B100008B9054810BD0021A160D0F87C211168FA
:100B200088474FF4403010BD0200030070B5044602
:100B30000D4600F00FFA064E40B1D0F87C01416836
:100B40008847A84224BF65604FF44036304670BDE8
:100B5000020003002DE9FF4715000C4600D02CB120
:100B6000064600F0F7F95FEA000801D16448C3E0E7
:100B7000D8F8F80001684A689047B0F5003F17D1EF
:100B8000D8F87C118A68404690478146B9F1810FB8
:100B900080F09E80A94508F1FC0A17D2D8F8F80029
:100BA0000368D3F80CC02A462146E047B0F5003F61
:100BB00040F08E80D8F8F8000368D3F810C06A4679
:100BC0005146E047B0F5003F76D10AE0002004E04E
:100BD000215C0AF800100098401C00900098A84280
:100BE000F6D34FF0000C4749474A484B01AC0098F8
:100BF000844558D2D3E9007001ADC5E90070107882
:100C000000281ABF042086464FF0000E085854F8FA
:100C10000E5028443E4D05600127D0F800E0876063
:100C2000019D4F681AF80C007D408EEA050585F09D
:100C3000040E65680F687D4085F0FC05754485F0FD
:100C4000A30568400AF80C000CF1010CCFE7D3E9CA
:100C5000004501A8C0E9004510782E4D002814BFBA
:100C60004FF0040E4FF0000E01A8744651F80EE04C
:100C70000459A6440127CEF80050DEF80040CEF813
:100C800008704D68019F40687D406C400D68684069
:100C900084F0040480F0FC00041984F057040AF87E
:100CA0000C400CF1010CCC45D1D3D8F8F800016808
:100CB0004A689047B0F5003F0AD1D8F8F8000368B9
:100CC000D3F80C804A465146C047B0F5003F01D0EA
:100CD000114811E0002006E05AF8201081F06A3136
:100CE0004AF82010401CB0EB990FF5D3B06840F0E3
:100CF0000100B0604FF4403004B0BDE8F08700BFA1
:100D000002000300745C0308E40700202C0F0008B5
:100D1000ADBE4ED70DBE75A10100030038B50C461F
:100D2000017A1546CA0702D500F014F908B9084837
:100D300032BDD0F8F80003682146DC682A46A04797
:100D4000B0F5003F01D0034832BD4FF4403032BD12
:100D500002000300010003002DE9F84191B00546AF
:100D60000E461746402101A82DF097FC297AC807A6
:100D700004D5284600F0EEF8040002D1DFF8A48084
:100D80004BE0D4F8F800DFF8A0800368D3F810C077
:100D90006A4601A9E047B0F5003F3ED1D4F8F8001B
:100DA00001684A689047B0F5003F36D1D4F87C110D
:100DB0008A6820469047D4F8F830024618461B68E7
:100DC000D3F80CC004F1FC01E047B0F5003F24D19A
:100DD000D4F87C0141688847D4F8F83002461846B8
:100DE0001B68D3F80CC001A9E047B0F5003F14D14F
:100DF000D4F8F8000268696893689847B0F5003F36
:100E00000BD1D4F8F80003681C693A463146A04774
:100E1000B0F5003F08BF4FF44038404612B0BDE87F
:100E2000F08100BF02000300010003002DE9F8413A
:100E3000A5B0074688461646402115A82DF02DFC82
:100E400000220492402105A82DF027FC387AC10722
:100E50005ED5384600F07EF8050059D0D5F8F80088
:100E60002D4C0368D3F810C06A4605A9E047B0F5D9
:100E7000003F3CD1D5F8F80001684A689047B0F5CA
:100E8000003F34D1D5F87C118A6828469047D5F8C0
:100E9000F830024618461B68D3F80CC005F1FC0177
:100EA000E047B0F5003F22D1D5F87C014168884782
:100EB000D5F8F830024618461B68D3F80CC005A9CF
:100EC000E047B0F5003F12D1D5F8F8000268796824
:100ED00093689847B0F5003F09D1D5F8F80003684A
:100EE0001D6904AA15A9A847B0F5003F01D0204606
:100EF0000FE00A4B0A490B4A0396029101924046C1
:100F00001C68049B009415AA796800F0E5F900E0DC
:100F1000054826B0BDE8F081010003007C5C0308B1
:100F2000936E030026C703000200030004B0010112
:100F300000170145E90A0008090B00082D0B0008FD
:100F4000BD030008550B00081D0D0008590D0008D1
:100F50002D0E00080168024A914218BF0020704718
:100F6000340F000810B5040008BF002404D0034863
:100F70002060204609688847204610BD340F0008CD
:100F800020225C302DF085BBF0B58468A3080022D8
:100F900004F0030407E000F15C0555F8226035BA5F
:100FA00041F82250521C9A42F5D300220BE000F186
:100FB0005C0502EB830755F82360D500C5F11805E1
:100FC000EE40CE55521CA242F1D3F0BD30B5C468FC
:100FD00003690022E31AD5188C5C0544521C082AC8
:100FE0002C77F8D330BD0360C1600261704738B51B
:100FF000044615460022626023685A689047002024
:101000006061A061A5604FF4003032BD81604FF493
:10101000003070472DE9F84304462079D4F80C805D
:10102000450748BF244845D466691D46A8F101001C
:1010300000EAD60306EBC506B6EBC50F666102D221
:10104000A669761CA6611746A66906EB5576A661C9
:101050000E46E918884225D2A8EB03094A463146D4
:10106000F8182DF016FB2268136839460FE0424647
:1010700038462DF00EFB23681A6839462046904703
:1010800007E0311811F00300F1D1226813682046FF
:101090009847484600EB0809A9F10101A942F0D39D
:1010A000002300E000202A1A3118F8182DF0F1FA78
:1010B0004FF40030BDE8F283040002002DE9FC4F3C
:1010C000024685B0D0681369DFF86CC1DFF86C8127
:1010D000A0EB030A506840F004005060002703A80A
:1010E00002900DF10C0ED8E9003403A8544DC0E96C
:1010F00000342878534D00280CBF00230423994660
:101100005CF803305EF80940234401261D601C682A
:101110009E60DCF80430039DDCF80090DEF804608B
:101120005D406540484C654089EA0606474C66408C
:101130007519474C6540D8E9006B03AC0028C4E939
:10114000006B0EBF002404200424029E5CF8000003
:10115000345920183F4C04600126046886600398C7
:10116000029E43406340384C7068634089EA000047
:10117000364C6040034438484340280018BF0120E3
:101180005B1E9B41042F2CBFC0B2D80F02F1140389
:1011900053F8200007F00303C3F10303DB00D8403A
:1011A0000DF807007F1C082F9DD315460C466A6971
:1011B000AB69E868D20842EA4372401E00EA0207BF
:1011C000002302409B420AD8524508D28020E055B5
:1011D0007F1C574516D2AAEB0701E01910E08020CA
:1011E000E05500E0E355E8687F1C8742FAD32A689F
:1011F000136828469847BAF1000F03D0514620469D
:101200002DF04BFA2A68069E059F9368694628468A
:1012100098472A68D2F8009021462846C8472B688C
:10122000DA683946284690470EB1A86830604FF416
:10123000003007B0BDE8F08F745C03085C12000852
:10124000E40700205FC5109304850012FC68017A52
:10125000C0F524FF24AF33D426AF698B04B001015D
:1012600000170145F8B501240094002300240DE087
:10127000009D065D0F5D7E40F643761CF60F86F0FE
:10128000010635400095641C009DEB189442EFD395
:101290001846F2BDF8B5002301240094002A11E09D
:1012A000009C85188F1815F8016C17F8015C6E40CA
:1012B000F643761CF60F86F0010634400094009C3D
:1012C000E318521EECD11846F2BD0000651200086A
:1012D00095120008010000002DE9F84F1D46DDF8C9
:1012E00028900B9F0D9C4FF0FF3300930E469246C3
:1012F000D9F800B0804632465146D847834664B399
:10130000D9F8043032465146404698476FEA0B02FE
:10131000521C42EA0B0200996FEAD2735B1C19401F
:10132000C2430091521C024300996FEAD2735B1CC6
:101330001940009186F05531484087EA000181F05C
:101340005531216080F05531C943491C0843009A4A
:101350006FEAD070401C82430092D9F8080001283F
:1013600009D17540E943491C0D4300986FEAD572D5
:10137000521C90430AE0F11C85EA9102D243521CB0
:10138000154300986FEAD5735B1C984386F0AA3624
:10139000009086EA0B0686F0AA33F243DB430C98F2
:1013A000C2F3C0725B1C42EAD3720099D243521C52
:1013B00091430091774000998843009987F0AA37BC
:1013C0000F403843BDE8F28F00000000000000002D
:1013D00001F0FF01102A2BDB10F0070F08D010F8E6
:1013E000013B013A8B422DD010F0070F42B3F6D1EA
:1013F000F0B441EA012141EA014122F007047FF003
:1014000000070023F0E80256083C85EA010586EA59
:10141000010685FA47F5A3FA87F586FA47F6A5FA95
:1014200087F68EB9EED1F0BC01F0FF0102F00702A1
:1014300032B110F8013B013A83EA010313B1F8D14C
:101440000020704701387047002D06BF354603382D
:10145000073815F0010F07D1013015F4807F02BF66
:10146000013015F4C03F0130F0BC0138704700BFB7
:10147000034613F8012B002AFBD1181A01387047D4
:1014800081F0004102E000BF83F0004330B54FEA35
:1014900041044FEA430594EA050F08BF90EA020FA2
:1014A0001FBF54EA000C55EA020C7FEA645C7FEA35
:1014B000655C00F0E2804FEA5454D4EB5555B8BF58
:1014C0006D420CDD2C4480EA020281EA030382EAC9
:1014D000000083EA010180EA020281EA0303362D5B
:1014E00088BF30BD11F0004F4FEA01314FF4801C2E
:1014F0004CEA113102D0404261EB410113F0004F40
:101500004FEA03334CEA133302D0524263EB4303F6
:1015100094EA050F00F0A780A4F10104D5F1200E94
:101520000DDB02FA0EFC22FA05F2801841F10001EF
:1015300003FA0EF2801843FA05F359410EE0A5F1C3
:1015400020050EF1200E012A03FA0EFC28BF4CF0F4
:10155000020C43FA05F3C01851EBE37101F00045AA
:1015600007D54FF0000EDCF1000C7EEB00006EEBB7
:101570000101B1F5801F1BD3B1F5001F0CD3490841
:101580005FEA30004FEA3C0C04F101044FEA445298
:1015900012F5800F80F09A80BCF1004F08BF5FEA1F
:1015A000500C50F1000041EB045141EA050130BDFF
:1015B0005FEA4C0C404141EB0101013C28BFB1F511
:1015C000801FE9D291F0000F04BF01460020B1FA5C
:1015D00081F308BF2033A3F10B03B3F120020CDA2F
:1015E0000C3208DD02F1140CC2F10C0201FA0CF00D
:1015F00021FA02F10CE002F11402D8BFC2F1200C72
:1016000001FA02F120FA0CFCDCBF41EA0C01904027
:10161000E41AA2BF01EB0451294330BD6FEA040470
:101620001F3C1CDA0C340EDC04F11404C4F120025B
:1016300020FA04F001FA02F340EA030021FA04F36D
:1016400045EA030130BDC4F10C04C4F1200220FAC4
:1016500002F001FA04F340EA0300294630BD21FA02
:1016600004F0294630BD94F0000F83F4801306BFC8
:1016700081F480110134013D4EE77FEA645C18BFBC
:101680007FEA655C29D094EA050F08BF90EA020F53
:1016900005D054EA000C04BF1946104630BD91EA4B
:1016A000030F1EBF0021002030BD5FEA545C05D14E
:1016B0004000494128BF41F0004130BD14F580048D
:1016C0003CBF01F5801130BD01F0004545F0FE4101
:1016D00041F470014FF0000030BD7FEA645C1ABF36
:1016E000194610467FEA655C1CBF0B46024650EA6D
:1016F000013406BF52EA033591EA030F41F4002199
:1017000030BD00BF90F0000F04BF0021704730B51E
:101710004FF4806404F132044FF000054FF00001F3
:1017200050E700BF90F0000F04BF0021704730B5B4
:101730004FF4806404F1320410F0004548BF404289
:101740004FF000013EE700BF42004FEAE2014FEADE
:1017500031014FEA02701FBF12F07F4393F07F4FB9
:1017600081F06051704732F07F4208BF704793F0BC
:101770007F4F04BF41F40021704730B54FF46074CF
:1017800001F0004521F000411CE700BF50EA0102D2
:1017900008BF704730B54FF000050AE050EA01027B
:1017A00008BF704730B511F0004502D5404261EBEB
:1017B00041014FF4806404F132045FEA915C3FF42C
:1017C000D8AE4FF003025FEADC0C18BF03325FEAC9
:1017D000DC0C18BF033202EBDC02C2F1200300FA7A
:1017E00003FC20FA02F001FA03FE40EA0E0021FA9F
:1017F00002F11444BDE600BF70B54FF0FF0C4CF48D
:10180000E06C1CEA11541DBF1CEA135594EA0C0F3E
:1018100095EA0C0F00F0DEF82C4481EA030621EA79
:101820004C5123EA4C5350EA013518BF52EA0335B4
:1018300041F4801143F4801338D0A0FB02CE4FF066
:101840000005E1FB02E506F00042E0FB03E54FF096
:101850000006E1FB03569CF0000F18BF4EF0010E8E
:10186000A4F1FF04B6F5007F64F5407404D25FEA8A
:101870004E0E6D4146EB060642EAC62141EA55513D
:101880004FEAC52040EA5E504FEACE2EB4F1FD0C7F
:1018900088BFBCF5E06F1ED8BEF1004F08BF5FEAFD
:1018A000500E50F1000041EB045170BD06F00046AF
:1018B00046EA010140EA020081EA0301B4EB5C045C
:1018C000C2BFD4EB0C0541EA045170BD41F4801154
:1018D0004FF0000E013C00F3AB8014F1360FDEBF79
:1018E000002001F0004170BDC4F10004203C35DA55
:1018F0000C341BDC04F11404C4F1200500FA05F3D8
:1019000020FA04F001FA05F240EA020001F0004278
:1019100021F0004110EBD37021FA04F642EB0601EE
:101920005EEA430E08BF20EAD37070BDC4F10C0418
:10193000C4F1200500FA04F320FA05F001FA04F2DC
:1019400040EA020001F0004110EBD37041F10001C8
:101950005EEA430E08BF20EAD37070BDC4F12005D3
:1019600000FA05F24EEA020E20FA04F301FA05F23B
:1019700043EA020321FA04F001F0004121FA04F2E3
:1019800020EA020000EBD3705EEA430E08BF20EAB3
:10199000D37070BD94F0000F0FD101F000464000ED
:1019A00041EB010111F4801F08BF013CF7D041EA6F
:1019B000060195F0000F18BF704703F00046520073
:1019C00043EB030313F4801F08BF013DF7D043EA44
:1019D0000603704794EA0C0F0CEA135518BF95EAFA
:1019E0000C0F0CD050EA410618BF52EA4306D1D181
:1019F00081EA030101F000414FF0000070BD50EAA0
:101A0000410606BF1046194652EA430619D094EA29
:101A10000C0F02D150EA013613D195EA0C0F05D113
:101A200052EA03361CBF104619460AD181EA030167
:101A300001F0004141F0FE4141F470014FF000001F
:101A400070BD41F0FE4141F4780170BD70B54FF0BA
:101A5000FF0C4CF4E06C1CEA11541DBF1CEA13553A
:101A600094EA0C0F95EA0C0F00F0A7F8A4EB05041C
:101A700081EA030E52EA03354FEA013100F0888013
:101A80004FEA03334FF0805545EA131343EA1263DC
:101A90004FEA022245EA111545EA10654FEA002691
:101AA0000EF000419D4208BF964244F1FD0404F54A
:101AB000407402D25B084FEA3202B61A65EB0305A6
:101AC0005B084FEA32024FF480104FF4002CB6EB63
:101AD000020E75EB030E22BFB61A754640EA0C00E3
:101AE0005B084FEA3202B6EB020E75EB030E22BF23
:101AF000B61A754640EA5C005B084FEA3202B6EB64
:101B0000020E75EB030E22BFB61A754640EA9C0022
:101B10005B084FEA3202B6EB020E75EB030E22BFF2
:101B2000B61A754640EADC0055EA060E18D04FEAB0
:101B3000051545EA16754FEA06164FEAC30343EA50
:101B400052734FEAC2025FEA1C1CC0D111F4801F1D
:101B50000BD141EA00014FF000004FF0004CB6E716
:101B600011F4801F04BF01430020B4F1FD0C88BFB5
:101B7000BCF5E06F3FF6AFAEB5EB030C04BFB6EBC0
:101B8000020C5FEA500C50F1000041EB045170BDB3
:101B90000EF0004E4EEA113114EB5C04C2BFD4EBE0
:101BA0000C0541EA045170BD41F480114FF0000E64
:101BB000013C90E645EA060E8DE60CEA135594EAE0
:101BC0000C0F08BF95EA0C0F3FF43BAF94EA0C0FE3
:101BD0000AD150EA01347FF434AF95EA0C0F7FF458
:101BE00025AF104619462CE795EA0C0F06D152EAAC
:101BF00003353FF4FDAE1046194622E750EA410690
:101C000018BF52EA43067FF4C5AE50EA41047FF4A0
:101C10000DAF52EA43057FF4EBAE12E74FF0FF3C05
:101C200006E000BF4FF0010C02E000BF4FF0010CD6
:101C30004DF804CD4FEA410C7FEA6C5C4FEA430C4F
:101C400018BF7FEA6C5C1BD001B050EA410C0CBF9E
:101C500052EA430C91EA030F02BF90EA020F002000
:101C6000704710F1000F91EA030F58BF994208BF67
:101C700090422CBFD8176FEAE37040F00100704724
:101C80004FEA410C7FEA6C5C02D150EA013C07D17B
:101C90004FEA430C7FEA6C5CD6D152EA033CD3D0C6
:101CA0005DF8040B704700BF8446104662468C46C0
:101CB0001946634600E000BF01B5FFF7B7FF0028F3
:101CC00048BF10F1000F01BD4DF808EDFFF7F4FF1C
:101CD0000CBF012000205DF808FB00BF4DF808EDA7
:101CE000FFF7EAFF34BF012000205DF808FB00BFCA
:101CF0004DF808EDFFF7E0FF94BF012000205DF8EC
:101D000008FB00BF4DF808EDFFF7CEFF94BF0120A0
:101D100000205DF808FB00BF4DF808EDFFF7C4FF99
:101D200034BF012000205DF808FB00BF4FEA410CE2
:101D30007FEA6C5C02D150EA013C0AD14FEA430CC5
:101D40007FEA6C5C02D152EA033C02D14FF0000002
:101D500070474FF0010070474FEA410212F5001240
:101D600015D211D56FF47873B3EB625212D94FEAE2
:101D7000C12343F0004343EA505311F0004F23FACC
:101D800002F018BF404270474FF00000704750EA21
:101D9000013005D111F0004008BF6FF000407047DE
:101DA0004FF00000704700BF4FEA4102B2F1E0433C
:101DB00024BFB3F5001CDCF1FE5C0DD901F0004C32
:101DC0004FEAC0024CEA5070B2F1004F40EB830082
:101DD00008BF20F00100704711F0804F21D113F1AE
:101DE0003872BCBF01F00040704741F480114FEAE7
:101DF0005252C2F11802C2F1200C10FA0CF320FA70
:101E000002F018BF40F001004FEAC1234FEAD3238C
:101E100003FA0CFC40EA0C0023FA02F34FEA4303F6
:101E2000CCE77FEA625307D150EA01331EBF4FF07F
:101E3000FE4040F44000704701F0004040F0FE409A
:101E400040F40000704700BF80F0004002E000BF97
:101E500081F0004142001FBF5FEA410392EA030F95
:101E60007FEA226C7FEA236C6AD04FEA1262D2EBDF
:101E70001363C1BFD218414048404140B8BF5B42E4
:101E8000192B88BF704710F0004F40F4000020F07D
:101E90007F4018BF404211F0004F41F4000121F093
:101EA0007F4118BF494292EA030F3FD0A2F10102DD
:101EB00041FA03FC10EB0C00C3F1200301FA03F11B
:101EC00000F0004302D5494260EB4000B0F5000F3E
:101ED00013D3B0F1807F06D340084FEA310102F1FD
:101EE0000102FE2A51D2B1F1004F40EBC25008BFAF
:101EF00020F0010040EA03007047490040EB000079
:101F0000013A28BFB0F5000FEDD2B0FA80FCACF179
:101F1000080CB2EB0C0200FA0CF0AABF00EBC250A6
:101F200052421843BCBFD0401843704792F0000F94
:101F300081F4000106BF80F400000132013BB5E7E7
:101F40004FEA41037FEA226C18BF7FEA236C21D05D
:101F500092EA030F04D092F0000F08BF08467047C2
:101F600090EA010F1CBF0020704712F07F4F04D190
:101F7000400028BF40F00040704712F100723CBFA3
:101F800000F50000704700F0004343F0FE4040F4CD
:101F9000000070477FEA226216BF08467FEA23638B
:101FA0000146420206BF5FEA412390EA010F40F476
:101FB000800070474FF0000304E000BF10F00043C2
:101FC00048BF40425FEA000C08BF704743F09643A9
:101FD00001464FF000001CE050EA010208BF7047C4
:101FE0004FF000030AE000BF50EA010208BF70474B
:101FF00011F0004302D5404261EB41015FEA010C60
:1020000002BF84460146002043F0B64308BFA3F157
:102010008053A3F50003BCFA8CF2083AA3EBC25339
:1020200010DB01FA02FC634400FA02FCC2F1200258
:10203000BCF1004F20FA02F243EB020008BF20F08F
:102040000100704702F1200201FA02FCC2F12002F5
:1020500050EA4C0021FA02F243EB020008BF20EAEA
:10206000DC7070474FF0FF0C1CEAD0521EBF1CEA18
:10207000D15392EA0C0F93EA0C0F6FD01A4480EA06
:10208000010C400218BF5FEA41211ED04FF00063EF
:1020900043EA501043EA5111A0FB01310CF000401B
:1020A000B1F5000F3EBF490041EAD3715B0040EA41
:1020B000010062F17F02FD2A1DD8B3F1004F40EB11
:1020C000C25008BF20F00100704790F0000F0CF0E4
:1020D000004C08BF49024CEA502040EA51207F3AA8
:1020E000C2BFD2F1FF0340EAC250704740F4000083
:1020F0004FF00003013A5DDC12F1190FDCBF00F074
:1021000000407047C2F10002410021FA02F1C2F121
:10211000200200FA02FC5FEA310040F1000053EABD
:102120004C0308BF20EADC70704792F0000F00F00B
:10213000004C02BF400010F4000F013AF9D040EA11
:102140000C0093F0000F01F0004C02BF490011F4A5
:10215000000F013BF9D041EA0C018FE70CEAD153A3
:1021600092EA0C0F18BF93EA0C0F0AD030F0004C23
:1021700018BF31F0004CD8D180EA010000F00040D7
:10218000704790F0000F17BF90F0004F084691F095
:10219000000F91F0004F14D092EA0C0F01D14202CF
:1021A0000FD193EA0C0F03D14B0218BF084608D198
:1021B00080EA010000F0004040F0FE4040F40000E2
:1021C000704740F0FE4040F4400070474FF0FF0C75
:1021D0001CEAD0521EBF1CEAD15392EA0C0F93EABC
:1021E0000C0F69D0A2EB030280EA010C49024FEA0E
:1021F000402037D04FF0805343EA111143EA1013C7
:102200000CF000408B4238BF5B0042F17D024FF47E
:10221000000C8B4224BF5B1A40EA0C00B3EB510F59
:1022200024BFA3EB510340EA5C00B3EB910F24BF42
:10223000A3EB910340EA9C00B3EBD10F24BFA3EBC7
:10224000D10340EADC001B0118BF5FEA1C1CE0D18F
:10225000FD2A3FF650AF8B4240EBC25008BF20F042
:10226000010070470CF0004C4CEA50207F32C2BF96
:10227000D2F1FF0340EAC250704740F400004FF033
:102280000003013A37E792F0000F00F0004C02BF64
:10229000400010F4000F013AF9D040EA0C0093F02E
:1022A000000F01F0004C02BF490011F4000F013B88
:1022B000F9D041EA0C0195E70CEAD15392EA0C0FF0
:1022C00008D142027FF47DAF93EA0C0F7FF470AF28
:1022D000084676E793EA0C0F04D14B023FF44CAF6B
:1022E00008466EE730F0004C18BF31F0004CCAD100
:1022F00030F000427FF45CAF31F000437FF43CAF3C
:102300005FE700BF4FF0FF3C06E000BF4FF0010C5D
:1023100002E000BF4FF0010C4DF804CD4FEA40023F
:102320004FEA41037FEA226C18BF7FEA236C11D089
:1023300001B052EA530C18BF90EA010F58BFB2EB3C
:10234000030088BFC81738BF6FEAE17018BF40F0BC
:10235000010070477FEA226C02D15FEA402C05D170
:102360007FEA236CE4D15FEA412CE1D05DF8040BF5
:10237000704700BF844608466146FFE70FB5FFF788
:10238000C9FF002848BF10F1000F0FBD4DF808ED40
:10239000FFF7F4FF0CBF012000205DF808FB00BF31
:1023A0004DF808EDFFF7EAFF34BF012000205DF88B
:1023B00008FB00BF4DF808EDFFF7E0FF94BF0120D8
:1023C00000205DF808FB00BF4DF808EDFFF7D2FFD5
:1023D00094BF012000205DF808FB00BF4DF808ED18
:1023E000FFF7C8FF34BF012000205DF808FB00BFE5
:1023F0004FEA40024FEA41037FEA226C02D15FEAD2
:10240000402C08D17FEA236C02D15FEA412C02D133
:102410004FF0000070474FF0010070474FEA400254
:10242000B2F1FE4F0FD34FF09E03B3EB12620DD902
:102430004FEA002343F0004310F0004F23FA02F06C
:1024400018BF404270474FF00000704712F1610F13
:1024500001D1420205D110F0004008BF6FF00040EA
:1024600070474FF00000704742000ED2B2F1FE4FAD
:102470000BD34FF09E03B3EB126209D44FEA002353
:1024800043F0004323FA02F070474FF0000070471A
:1024900012F1610F01D1420202D14FF0FF307047BB
:1024A0004FF00000704700BF53B94AB9002908BF78
:1024B00000281CBF4FF0FF314FF0FF3000F06AB929
:1024C000ADF1080C6DE904CE00F006F8DDF804E08B
:1024D000DDE9022304B070472DE9F047089D0C4662
:1024E000002B4ED194468C458646B2FA82F262D9D0
:1024F0004AB1C2F12003914020FA03F30CFA02FC26
:10250000194300FA02FE4FEA1C471FFA8CF6B1FB92
:10251000F7F44FEA1E4307FB141143EA014304FB9F
:1025200006F199420AD91CEB030304F1FF3080F055
:102530001281994240F20F81023C6344591A1FFAFA
:102540008EF3B1FBF7F007FB101143EA014300FBE8
:1025500006F69E420AD91CEB030300F1FF3180F01E
:10256000FC809E4240F2F980634402389B1B40EAA3
:10257000044000211DB1D3400022C5E90032BDE86E
:10258000F0878B4205D90DB1C5E90001002108464D
:10259000F5E7B3FA83F1002946D1A34202D3904272
:1025A000C0F0F080861A64EB03030120002DE6D012
:1025B000C5E90063E3E7002A40F09080A1EB0C043A
:1025C0004FEA1C481FFA8CF70121B4FBF8F64FEADA
:1025D0001E4308FB164443EA044307FB06F09842F7
:1025E00008D91CEB030306F1FF3402D2984200F233
:1025F000CD8026461C1A1FFA8EF3B4FBF8F008FBB8
:10260000104443EA044300FB07F79F4208D91CEB40
:10261000030300F1FF3402D29F4200F2B080204653
:10262000DB1B40EA0640A5E7C1F120068B4022FAF9
:1026300006F71F4320FA06FC04FA01F343EA0C03F1
:10264000F44000FA01F8380C4FEA1349B4FBF0FEED
:102650001FFA87FC00FB1E4449EA04440EFB0CF9F8
:10266000A14502FA01F20AD93C190EF1FF3A80F0B5
:102670008480A14540F28180AEF1020E3C44A4EB7F
:1026800009041FFA83F9B4FBF0F300FB134449EA91
:10269000044403FB0CFCA44507D93C1903F1FF30AB
:1026A00067D2A44565D9023B3C4443EA0E40A0FBF7
:1026B0000293A4EB0C049C42CE469C4651D34ED0D0
:1026C00055B1B8EB0E0364EB0C0404FA06F6CB40EC
:1026D0001E43CC40C5E90064002150E7C2F120034D
:1026E00020FA03F10CFA02FC24FA03F394400C43A1
:1026F0004FEA1C4800FA02FE1FFA8CF7B3FBF8F011
:1027000008FB1031230C43EA014300FB07F1994217
:1027100008D91CEB030300F1FF362CD299422AD9C9
:10272000023863445B1AA4B2B3FBF8F108FB11331F
:1027300044EA034401FB07F3A34208D91CEB040459
:1027400001F1FF3613D2A34211D902396444E41ACD
:1027500041EA004139E70446F0E6084606E7C84585
:10276000AED2B9EB020E63EB070C0138A8E7314695
:10277000EDE7034699E73046D4E7D6467FE7634462
:1027800002384DE70646234608460FE7023E6344FB
:1027900030E700BF704700BF00487047001BB74BD1
:1027A00070B50C4601F02CFA104E05460821304653
:1027B00006F068F8012804D001F022FA431BA34276
:1027C00007D30821094806F05DF8431E58425841D6
:1027D00070BD72B60821304606F054F8012800D0CA
:1027E00030BF62B6BFF36F8FE0E700BF0004004860
:1027F00008B5002210214FF0904006F049F8054836
:102800000022202106F044F8BDE80840022001F033
:10281000FFB900BF0004004810B50C4C0122102184
:10282000204606F035F8052001F0F2F92046012295
:10283000202106F02DF84FF090400122102106F0E3
:1028400027F8BDE81040022001F0E2B9000400487A
:1028500070B54FF090400C46164610210022144DE2
:1028600006F016F800232B701248B3B22246214618
:1028700007F002FAD8B901F0C3F941F287360446ED
:102880002B783BB1BDE87040012210214FF0904001
:1028900005F0FEBF01F0B4F9031BB342F2D872B6E3
:1028A0002B7803B930BF62B6BFF36F8FE8E770BD16
:1028B000E507002048090020014B01221A707047EB
:1028C000E507002000487047805C030813B5114BF2
:1028D0000446186800909B88ADF804300120FFF78B
:1028E0009BFF062269460120FFF7B2FF0120FFF798
:1028F0007FFF9DF80430112B08D19DF80520122A86
:1029000004D101202370627002B010BD00231A466A
:102910001846F7E7581B03080CB4F0B5ADB032AB5E
:1029200006AF53F8042B059305460E46384696210C
:102930002BF002FE9528C1BF42F62E63ADF8AA30F7
:102940002E23ADF8AC3000F037F83C24042D4FF4C2
:102950007A7E1449B0FBFEFCB0FBF1F14EF6602329
:10296000B0FBF3F3B3FBF4F204FB1232BCFBF4F361
:1029700004FB13C30EFB1C049ABF0B48405D3F20B1
:10298000CDE90040CDE9026708482BF055FD084B22
:102990001B6898682BF07AFC2DB0BDE8F04002B0BF
:1029A000704700BF80EE3600DE5C0308BC5C0308A5
:1029B000F405002001F02CB901F022B91348144AA3
:1029C00008B54FF00043C0E9002304224261012210
:1029D0000023C2614FF480510722C0E90233C0E9ED
:1029E0000933C0E90C1203610383837680F8203039
:1029F00080F82C30826380F83C30C36404F09AFE87
:102A000018B1BDE8084000F099BB08BDE8070020F8
:102A1000002401400268084B9A4282B00AD14FF06C
:102A2000B0431A6E42F400721A661B6E03F4007310
:102A30000193019B02B07047002401400268054BDE
:102A40009A4201BF4FF0B042136E23F40073136635
:102A5000704700BF0024014030B585B00024054612
:102A6000CDE901440394FFF7A9FF144805F0F6F9F6
:102A700008B100F063FB1148039401A9CDE90154AA
:102A800004F0B6FF08B100F059FB0C4805F010F94E
:102A900008B100F053FB4FF0FF31084804F04AFF43
:102AA000064805F0BDF9054804F09EFF04460348BA
:102AB00005F060F9204605B030BD00BFE8070020F2
:102AC000014B024A1A607047E807002000240140C9
:102AD00008B50948FFF7C0FF68B1084BB3F8AA3042
:102AE0004FF6FF72934216BF40F6E442044B534345
:102AF000B3FBF0F398B208BD002000B40075FF1FCF
:102B0000D8084C0013B50023ADF80630FFF7E0FFFE
:102B100004461948FFF7A0FF184BB3F8C820B3F8D4
:102B2000A8108A4204FB00F018D040F6E443B0FB42
:102B3000F3F364205B1A4343521A93FBF2F31E3300
:102B40001BB2ADF80630BDF806305BB21B02ADF823
:102B50000630BDF8060000B202B010BD4FF47A7224
:102B600040F6FF73B0FBF3F35343A3F53923A3F50A
:102B70000C6340F6C412E0E7001000B00075FF1FC0
:102B80004FF0B04382B09A6A22F480529A629A6CF3
:102B900042F480529A649B6C03F480530193019B2E
:102BA000002002B070474FF0B04307B59A6C42F076
:102BB00004029A649A6C02F004020192019A9A6CDF
:102BC00042F001029A649B6C002203F0010311465B
:102BD00000930B20009B05F0DFF90B2005F00EFAA7
:102BE000002211460C2005F0D7F90C2005F006FA5A
:102BF000002211460D2005F0CFF90D2005F0FEF959
:102C0000002202210F2005F0C7F90F2005F0F6F988
:102C100000221146102005F0BFF9102005F0EEF952
:102C200000221146112005F0B7F9112003B05DF81C
:102C300004EB05F0E3B9000008B505F023FC10B182
:102C40006FF0040008BD064B9A6942F040429A6159
:102C50004CF2FA321A6105F027FC0028F2D0EFE7B7
:102C600000400058F0B585B000230D46009306469D
:102C7000A8B3FFF7E1FF044670BB05F003FC88BB77
:102C80001A481B4A02230193D0F8E01506F1784355
:102C900002EA8121B3FBF1F701FB1733DB0A029350
:102CA000D0F8E00505F178410139314402EA80228B
:102CB000B1FBF2F002FB1011C3EBD12301336946E3
:102CC00001A8039305F070FC20B1022814BF6FF037
:102CD0000104012405F0E8FB204605B0F0BD6FF0CB
:102CE0000504F9E76FF00404F6E700BF0070FF1F6A
:102CF00000FCFF03014B1860002070474C080020C7
:102D00002DE9F04FB0F1006F89B006460F469046AE
:102D1000C0F0C080DFF89091644DD9F8E03505EA45
:102D2000832303F10063013B984200F2B380002942
:102D300000F0B38040EA02035B0740F0AE80FFF78B
:102D40007BFF044690BB05F09DFB002840F0A88067
:102D5000D9F8E015009705EA812106F17842B2FB27
:102D6000F1F301FB132208F17843013B3344B3FB39
:102D7000F1F001FB1033DB0A01334FEAD22AA3EB57
:102D8000D222012A039388BFC6F30A050AF58037C9
:102D9000C6F108038CBFC5F500654546FF02B34682
:102DA0000693039B9A4505D305F07EFB204609B0A8
:102DB000BDE8F08FA6F10803069A1A4495421CD884
:102DC000009B04950193CDF814B04FF00009059BCA
:102DD00009EB0301049B99453DD3009BAB442B4475
:102DE000A8EB0505B5F5006F009328BF4FF400650B
:102DF0000AF1010A07F50067D3E753F8081F5A687C
:102E0000B2F1FF3F08BFB1F1FF3FD5D0284B1868A2
:102E100010B96FF00504C7E727B14FF400623946D7
:102E200011F04EFEDFF888900099D9F80030CBF30E
:102E30000A001844AAB211F043FE4FF4006138466C
:102E4000FFF710FF00BBD9F8003001934FF4006387
:102E500005970493B9E7019B07914B440293012026
:102E6000D3E9002305F05AFB88B90799019BD1E902
:102E7000000259F80310029B5B689A4208BF88421F
:102E800005D109F10809A2E76FF001048CE76FF0A2
:102E9000030489E74FF0FF3488E76FF0050485E706
:102EA0006FF0040482E700BF0070FF1F00FCFF0307
:102EB0004C080020B1F1006F70B510D30B4BD3F864
:102EC000E0650B4B03EA862303F10063013B994263
:102ED00005D838B192B211F0F3FD002070BD4FF06B
:102EE000FF30FBE76FF00500F8E700BF0070FF1F41
:102EF00000FCFF03B0F1006F10B40DD3084BD3F802
:102F0000E045084B03EA842303F10063013B984248
:102F100002D810BCFFF7A6BE4FF0FF3010BC7047C0
:102F20000070FF1F00FCFF034FF0B04382B0DA6C6B
:102F30000243DA64DB6C03400193019B02B07047EB
:102F40002DE9F04186B01422002101A82BF012FBDC
:102F50000220464EFFF7E8FF0420FFF7E5FF0120BF
:102F6000FFF7E2FF04213046002205F091FC002229
:102F700010214FF0904005F08BFC04230024012524
:102F800002270DEB03013046CDE901354FF0100863
:102F9000CDE9034705F056FB01A93046CDE901858F
:102FA000CDE9037405F04EFB202301A93046CDE99D
:102FB0000135CDE9037405F045FB01A94FF09040C0
:102FC000CDE90185CDE9034405F03CFB08224FF42F
:102FD000881301A93046CDE901234FF00308CDE95C
:102FE000034705F02FFB4FF4441301A94FF0904025
:102FF000CDE90183CDE9035705F024FB4FF440539D
:1030000001A93046CDE90135CDE9034805F01AFBA9
:103010004FF404134021CDE901131548039501A98C
:1030200005F010FB22460F21062004F0B5FF062014
:1030300004F0E4FF22460F21072004F0ADFF072033
:1030400004F0DCFF22462146092004F0A5FF0920F8
:1030500004F0D4FF22462146092004F09DFF0920F8
:1030600004F0CCFF06B0BDE8F08100BF00040048CA
:103070000008004800B59BB04822002108A82BF0AA
:1030800079FA1822002102A82BF074FA05F01AFC34
:103090004FF0B0420120D2F8903023F01803C2F86C
:1030A0009030D2F8003423F4C06343F40073C2F8C4
:1030B0000034D2F8003403F4C0630193019B24234D
:1030C000089381230B930023CDE91003B02208A8B5
:1030D000CDE9122305F06EFD08B172B6FEE74F236D
:1030E000CDE90230CDE90400CDE90600022102A8B5
:1030F00005F0FAFF08B172B6FEE71BB05DF804FBFD
:1031000008B504F0C5FAFFF7B5FFFFF719FFFFF7A1
:103110004AFD00F0FDFF00F0ADFE00F089F8064822
:103120000122042105F0B4FB02F066FC00F048FC2B
:1031300002F069FCFCE700BF0004004872B6FEE73D
:1031400000B58DB02C22002101A82BF013FA1748EE
:10315000174B03601F2383604FF080420023C0E9B8
:103160000433C0E9072383614FF48073436206F0A0
:1031700061FA08B1FFF7E2FF0C4806F087FB08B1DF
:10318000FFF7DCFF4FF00053002207930748089237
:103190004FF4807301A9029206920B9306F0AAFAEB
:1031A00008B1FFF7CBFF0DB05DF804FB500800201D
:1031B0000028004010B5044690B03822002102A833
:1031C0002BF0D8F92268194B9A422CD14FF4803356
:1031D000029302A84FF480730F9306F0A9F808B188
:1031E000FFF7ACFF4FF0B0430220D3F8902042F439
:1031F0000042C3F890209A6D42F480629A659B6DFC
:10320000002203F4806311460193019B04F0C4FE85
:10321000022004F0F3FE00222A20114604F0BCFE36
:103220002A2004F0EBFE10B010BD00BF00280040C3
:103230001148124A08B54FF48273C0E900230023F5
:103240004FF4E062C0E902324FF400712822C0E975
:1032500006120722C0E90433C0E90833C0E90B2392
:1032600083620823436306F081FC18B1BDE808407F
:10327000FFF764BF08BD00BF4809002000300140CF
:10328000F0B5054689B01422002103A82BF072F98D
:103290002A68374B9A4269D14FF0B04302261A6E22
:1032A00042F480521A661A6E02F480520292029A16
:1032B000DA6C42F00102DA64DA6C02F00102019287
:1032C000019ADA6C42F00202DA64DB6C03F002036A
:1032D00000930524009B0327D02303A94FF09040BF
:1032E000CDE90336CDE9067405F0ACF92023CDE92C
:1032F00003364FF09040002603A90794CDE90567F7
:103300001C4C05F09FF91C4826620723C4E9000302
:1033100080232046C4E90266C4E90436C4E906668F
:1033200004F0CCFE08B1FFF709FF144AAC65A562B2
:10333000134C0823C4E900231021002380222046D7
:10334000C4E90213C4E90423C4E90633236204F088
:10335000B5FE08B1FFF7F2FE002222206C6511468F
:10336000A56204F019FE222004F048FE09B0F0BD69
:1033700000300140E80800201C00024030000240FC
:10338000880800207047000008B504F097F9044B46
:103390000120C3F88800BDE8084005F0EBBA00BF83
:1033A0000004005808B504F090F900F0C1FFFFF7E1
:1033B000C7FDFFF7F8FB00F05DFDBDE80840FFF733
:1033C00037BF08B504F081F9FFF7BAFDFFF7EBFB53
:1033D000BDE80840FFF72CBF08B504F06FF9BDE861
:1033E00008400121002005F075BA70477047FEE7DC
:1033F000FEE7FEE7FEE7FEE770477047704770475D
:10340000014806F069BA00BF50080020024B0120B5
:10341000187005F04BBA00BFAA1E0020024B012213
:1034200002201A7005F042BAA91E0020082005F0FB
:103430003DBA0000014804F0B7BF00BF541300209C
:10344000014804F0B1BF00BFE8080020014804F0C3
:10345000ABBF00BF8808002070470000014804F09F
:10346000A3BF00BF0814002070470000014806F009
:10347000F1BD00BF48090020014807F029BF00BF87
:1034800068140020014806F05BB800BF5008002017
:10349000014807F070B800BF401300202DE9F04349
:1034A00089B080460020109E0790894615461F4629
:1034B000FCF7BEFEF0B9104CCDE90090CDE9020456
:1034C00007AB0E480593142304933A464346294616
:1034D0000068FCF777FF2346324604F1140153F8E5
:1034E000044B42F8044B8B42F9D1079B337509B06A
:1034F000BDE8F0830120FAE7C2090020705C0308F0
:103500007FB5124C00253C2302A86375CDE9025516
:10351000257500F01FFB042303AA009412210C4818
:10352000FFF7BCFF0B49142220462BF013F8064688
:10353000B0FA80F040096075074B00902A46294692
:10354000022011F0B7F9304604B070BDAC0900207C
:103550001A5D03085E210020FC5C0308034A04484E
:1035600040F21B53002107F029BD00BFD6090020FF
:10357000B4130020312BF0B52DD81825102415FBDD
:103580000343194D00244FF0800C4CFA04F6A3F1CC
:103590001007314205EB470714BF4FF0240E4FF0E0
:1035A000140EA7F806E0A3F10807304205EB470721
:1035B00014BF4FF0240E4FF0140E0134324205EBCD
:1035C0004306A7F806E00CBF14272427082CF78031
:1035D00003F10103D9D1054B1B781BB9BDE8F040BD
:1035E000FFF7BCBFF0BD00BFD6090020081F0020B8
:1035F00010B500240022E3B2114610460134FFF753
:10360000B9FF322CF6D1BDE81040FFF7A7BF00008C
:1036100070B504460D46FFF7EBFF0F4B04EB440477
:1036200000261C44142000F0F3FAA2786178207878
:1036300012FB05F211FB05F110FB05F0F3B2D2B25B
:10364000C9B2C0B20136FFF795FF322EEAD1BDE80C
:1036500070400A2000F0DCBA080000202DE9F0419B
:1036600006460F462048904600214FF416622AF085
:1036700081FF1E4A10254FF0800C2B4600244CFA87
:1036800004F1A3F110000F4202EB400014BF4FF011
:10369000240E4FF0140EA0F806E0A3F108000E422D
:1036A00002EB400014BF4FF0240E4FF0140E013413
:1036B00018EA010F02EB4301A0F806E00CBF14204A
:1036C0002420082CC88003F10103D8D11835B5F5A2
:1036D000986FD2D1064B1B781BB9BDE8F041FFF7BC
:1036E0003DBFBDE8F08100BFDC090020D609002005
:1036F000081F002003460846072B1CD8DFE803F00C
:1037000004070A0E121417190022114600E00022C5
:10371000104601E000221146FFF7A0BF0A46002133
:103720000020F9E70022F7E70A460021F0E70A4601
:10373000F6E70A46E9E770477FB502AC204611F08C
:103740001BFB94E80300824C824D2378012B85E813
:10375000030009D080490B7833B1804A13781BB13C
:103760007F4B1878052823D17E4B1A686AB92968DF
:1037700019607D49186808607C490A601B680093DD
:1037800011467B4B032011F095F87A487A4D037867
:10379000DBB20A2B32D8DFE813F02C004D005100C9
:1037A000570060009700AA00B600C300C300C30022
:1037B0002078012806D1097821B9127812B91B782E
:1037C000052BE2D0694B1A68002ADED129681960FE
:1037D0006A491868086063490A6018681B680968C4
:1037E0005B1ACDE900031146654B032011F062F826
:1037F000CBE7644B1B78DBB2634A13700378634EEC
:10380000012B06D0624C227802F0FF03002A00F060
:103810008C805D4A002313702B703370FFF7E8FE35
:103820005C4A002313705C4A13705C4B01221A70CF
:1038300004B070BD544B00221A70DFE7584A12786A
:10384000012A08BF0123D7E7237813B94E4B012281
:10385000F2E72378012BD1D146E0444B414A1B6863
:1038600012689B1A042BC9D923783C4A53B93A4BA6
:103870001B78012B06D11378012BD9B202D1424B10
:103880001970BBE72378012B05D0334B1B7813B19C
:103890001378002BB2D13C4B0221197041490C78AE
:1038A000032C03D104212970197008E00C78012C35
:1038B00001D10821F7E70C78022CE1B2F3D012789D
:1038C000002A9BD10822B7E7237833B9344B1B7801
:1038D000012BDAB201D12C4BAEE72378012B03D0B8
:1038E0002F4B1B78002B89D1274B0222A4E723788A
:1038F0001BB92D4B1B78002BA8D02378012BF3D0BC
:10390000294B1B78A6E723781BB9154B1B78042B92
:103910009CD02378012BE7D0114B1B78052B9AE71D
:103920000F4B1A78042AF8D190E7227812B9164B77
:103930001B78DBB22B701D4B28781978FFF7DAFE65
:10394000237803B12B782B78DBB2337068E700BFA4
:103950008B1E0020901E00200A010020090100207B
:10396000891E0020A41E00209C1E0020A01E0020F6
:103970002C5D03080601002006000020981E002090
:103980004F5D030804000020070000200100002014
:10399000081F00208E1E00208D1E0020001F00200A
:1039A0005D210020121500208A1E0020000000204A
:1039B000024803680021596307F07ABBB413002062
:1039C000002270B50F4B1146022010F073FF012446
:1039D0000A25294620461435FFF78CFEEDB2322029
:1039E00000F016F96E2DF4D10134E4B2FFF700FEB9
:1039F0000A2CEDD10022BDE87040034B1146022095
:103A000010F058BF865D0308B95D0308054808B586
:103A10000823036006F0CCFB18B1BDE80840FFF7AF
:103A20008DBB08BD401300204FF0B04307B55A6E60
:103A300042F001025A665B6E002203F0010301931B
:103A400011463220019B04F0A7FA322003B05DF842
:103A500004EB04F0D3BA00000CB407B5054A05AB7B
:103A60001021019311F036FB03B05DF804EB02B0B6
:103A7000704700BFEF5D030830B585B0044602A86B
:103A80000D4611F053F9BDF90C30064A0093102190
:103A9000029B2046FFF7E0FF2046FDF7E9FC288067
:103AA00005B030BDEF5D03084FF0B04210B593682C
:103AB00023F40043936011F0C1F9104B01241C70F2
:103AC00000F0ACF810F08CFE0D4810F0A3FE0D4B8A
:103AD0004FF400421A61022010F0A2FEFEF7F0FF40
:103AE00000F002F910F096FF2146204610F0B2FFD8
:103AF00021462046BDE8104010F096BF4C13002030
:103B0000793A00080040005810F0BABF08B5FEF737
:103B1000DFFF40F6B83398420CD8B0F5E16F0BD315
:103B2000FE23A0F5E16058434FF49663B0FBF3F039
:103B3000C0B208BDFE20FCE70020FAE77FB568466A
:103B400000F0B6F80198FEF769FC00B207B05DF826
:103B500004FB0000194A38B5D2F88035591C0446D8
:103B600019D103F0B9FD054603F0C2FD054403F089
:103B7000B9FD2B0EE3712B0CA3712B0A6371030E9D
:103B8000E370C0F30742C0F307232571C0B2A270EF
:103B90006370207038BD190AC3718171190C1B0E36
:103BA00041710371D2F88435C370D2F88405C0F333
:103BB0000722C0F30743000EE9E700BF0070FF1FB4
:103BC00038B5094BD3F8803503600133054609D178
:103BD00003F082FD044603F085FD444003F088FDB8
:103BE00044402C6038BD00BF0070FF1F012102203F
:103BF00010F01ABF0021022010F016BF00207047FD
:103C0000024B187808B100F0BFB970474C13002080
:103C100082B00190019802B000F052BAF0B5224A89
:103C2000224CD2F8903043F4804389B0C2F89030EF
:103C300003F064FD03F06AFD03F070FD01230493BB
:103C40000323069300254FF0B04305950795DA6CE2
:103C500042F00202DA64DA6C02F002020292029A84
:103C6000DA6C42F00202DA64DB6C03F002030193C7
:103C70004FF4805703A92046019B03974FF4005649
:103C800004F0E0FC03A92046039604F0DBFC2A467E
:103C90003946204604F0FCFD2A463146204604F011
:103CA000F7FD09B0F0BD00BF00080058000400484F
:103CB00010B50446FEF726FF074BA36040F30F2024
:103CC000FEF77CF9054B064A2360064B6060C4E9A9
:103CD0000323002010BD00BF0000484200007A44CA
:103CE0000D093E00AB03050000207047012070471E
:103CF00008B52AF0A1FC162303604FF0FF3008BD81
:103D000008B52AF099FC16230360FEE770B50D464E
:103D100014460E46731B9C4201DC204670BDAFF377
:103D2000008006F8010BF5E730B5104600234FF090
:103D30006042834200DB30BDD2F8804EE50707D5F4
:103D4000D2F8004EE40703D5CC5C156815B11470A9
:103D50000133EEE700BFF8E74FF0FF3070474FF454
:103D600000534B60002070470120704700207047CF
:103D70000B4A116810B5034609B90A491160106869
:103D800009490A4C0344091B8B4206D92AF054FC0A
:103D90000C2303604FF0FF3010BD1360FCE700BF41
:103DA00050130020104100200000012000080000F6
:103DB00037B5184B02689A42054628D14FF0B043F8
:103DC000154C1A6E42F400621A661B6E134A03F415
:103DD00000630193019B1723C4E9002310210023F2
:103DE0008020C4E902134FF48073C4E904034FF444
:103DF000806C2023C4E906C320464FF4005323629D
:103E000004F05CF908B1FFF799F96C62A56203B0A0
:103E100030BD00BF002C01405413002008000240B8
:103E200010B5044686B01422002101A82AF0A2FB96
:103E300022680F4B9A4218D14FF0B04301A9DA6CB7
:103E400042F00102DA64DB6C03F00103009302220A
:103E5000009B4FF48073CDE901324FF09040012375
:103E6000CDE90332059304F0EDFB06B010BD00BFB1
:103E7000002C014010B58EB01022002103A82AF0BA
:103E800079FB00241C2221460DEB0200CDE9004401
:103E900002942AF06FFB1F481F4B8460C0E9003476
:103EA0003B23C0E90334C0E9054406F0CDFD08B169
:103EB000FFF744F94FF480531648039303A906F023
:103EC000E1FE08B1FFF73AF9124806F0EDFD08B13E
:103ED000FFF734F900240F4802946946CDE9004405
:103EE00007F0E8F808B1FFF729F9602309480D94B5
:103EF000002207A9CDE90734CDE90944CDE90B44F7
:103F000006F03AFE08B1FFF719F90248FFF788FFFB
:103F10000EB010BDB4130020002C0140014B1868F6
:103F2000704700BF001400200320704708B5014609
:103F30004FF47A7200238002890DFEF7B5FA08BDAE
:103F40004FF47A73A0FB0303800A40EA8350704762
:103F5000034B98689A689042FBD1C043704700BFFA
:103F60000028004008B5FFF7F3FF014B186008BDBB
:103F70000014002008B5FFF7EBFF024B1B68C01AC6
:103F800008BD00BF00140020024B187808B1FFF7ED
:103F9000DFBF70470414002010B5074B074C012207
:103FA000DA654FF48071204605F090FA4FF0FF3348
:103FB0002363002010BD00BF0028004050080020EF
:103FC00002460021014805F098BC00BF50080020BF
:103FD00002460121014805F090BC00BF50080020B6
:103FE00010B58CB02C220021044601A82AF0C2FA98
:103FF000FFF7D2FF0C4B0D481B681C4400230893AD
:1040000006934FF00053E443079301224FF480736B
:1040100001A902940B9305F06DFB08B1FFF78EF830
:1040200000200CB010BD00BF00140020500800207C
:1040300038B50546FFF78CFF02210446074805F016
:1040400063FCC4F309024FF47A71A2FB0121920AC6
:10405000A30A2A8043EA805038BD00BF50080020E0
:104060000148002105F050BC500800200148012102
:1040700005F04ABC50080020F8B50F4D2E78CEB997
:104080000E4C4FF0FF372763FFF75AF8FFF784FF16
:104090004FF48071204605F019FA2046276305F099
:1040A000D7FB32462046022105F027FCFFF75AFFD6
:1040B00001232B700020F8BD0414002050080020BC
:1040C000014610B54FF47A7200238002890DFEF785
:1040D000EBF90146FFF73CFF0446FFF739FF031BEE
:1040E0008B4200D310BD00BFF7E710F0AFBF000058
:1040F00010B5064C0221204605F006FC0221421CA8
:104100002046BDE8104005F0F8BB00BF5008002075
:104110001648174A08B54FF4E133C0E900230023DD
:104120000C22C0E90233C0E90523C0E90733C0E926
:104130000933036107F0B1FE08B1FEF7FFFF0B483A
:10414000002108F022F808B1FEF7F8FF0748002127
:1041500008F03BF808B1FEF7F1FF044807F0F5FF5F
:1041600018B1BDE80840FEF7E9BF08BD681400209B
:104170000044004070B596B006461422002103A802
:104180002AF0F8F93822002108A82AF0F3F9326859
:10419000274B9A424AD10223089308A84FF44023A0
:1041A0000A9305F0C5F808B1FEF7C8FF4FF0B04319
:1041B00000259A6D1F4C42F400329A659A6D02F404
:1041C00000320292029ADA6C42F00102DA64DB6C8D
:1041D00003F001030193019B0C220223CDE9032389
:1041E00003A907234FF090400793CDE9055504F04C
:1041F00029FA114925621423C4E900131023C4E9E4
:10420000023520468023C4E90435C4E9065503F08D
:1042100055FF08B1FEF792FF2520F4670022022126
:10422000A66203F0B9FE252003F0E8FE16B070BDCB
:1042300000440040081400208000024002680C4B3B
:104240009A4210B5044612D14FF0B0420C21936D42
:1042500023F4003393654FF0904004F09FFAE06F31
:1042600003F09EFFBDE81040252003F0D5BE10BD31
:104270000044004008B50A460146024806F08CFF9B
:10428000002008BD6814002013B5114B114C1860B4
:104290004FF40013009302AB13E90600204607F029
:1042A000F8FE2368DA69D103FCD4DA695202FCD53E
:1042B0009A68084842F480029A6007F030FF064985
:1042C0000448012207F09EFE002002B010BD00BF8E
:1042D000FC140020681400200415002008B5074BCA
:1042E0001860FEF760FCFFF713FF054AD2F8803034
:1042F00043F00063C2F88030002008BD00150020A4
:104300000008005808B54FF0B04308489A6B42F4D3
:1043100000329A639A6B22F400329A63FFF78EFFA1
:10432000112003F079FE002008BD00BF68140020B2
:1043300008B5074807F0B1FD08B1FEF7FFFE0548D4
:1043400003F0BCFE18B1BDE80840FEF7F7BE08BD9B
:1043500068140020081400200268044B9A4203D11C
:10436000034B00201B681847704700BF0044004003
:104370000015002002680B4B9A4210B504460FD17D
:10438000094B1B682BB1D0F8902012B907480121C6
:10439000984720460549BDE81040012207F032BE8B
:1043A00010BD00BF00440040FC1400200415002094
:1043B0002DE9F04F9DB0FEF785FA13F0EFFA0246B3
:1043C00040B90146644B022010F074FA01201DB080
:1043D000BDE8F08F012013F089FB12F085F8044648
:1043E000039040B9024601465C4B022010F062FA8D
:1043F00013F048FBEAE75A4D296812F0C5FC6968DA
:10440000204612F0DBFC297A204612F00BFD697A77
:10441000204612F03BFD6969204612F0C7FDE868AE
:10442000FEF722F881B2204612F04AFD29692046A3
:1044300012F012FDA97A204612F0DAFC0221204681
:1044400012F08CFD1021204612F0CAFD039812F0E4
:10445000D3F80246049040B90146424B022010F0C6
:1044600029FA03A812F0A0F8C2E703A812F09CF8FA
:10447000049812F029FC024640B901463A4B02204A
:1044800010F018FA04A812F0D5F9B1E7374EDFF8AA
:10449000E0A0DFF8E0B0002333604FF0020804989A
:1044A00005AB0A2208A912F001FA054628BB02460C
:1044B0000146314B022010F0FDF930682C49FDF720
:1044C000D1FD4FF07C51FDF7CDFD3060049812F026
:1044D0002BFC044604A812F0ADF913F0D3FA002C1B
:1044E0003FF474AF002D3FF471AF0022234B11460F
:1044F000032010F0DFF9002069E731680998FDF723
:10450000A9FCBDF81890306000221D4BCDF800903A
:104510001146022010F0CEF908AC0027BBB2994535
:1045200004F1080405D8B8F1010FC6D04FF0010816
:10453000B5E754F8040C5146FDF794FDFDF794FFE0
:10454000019034F8083C009300225B46114602209B
:1045500010F0B0F90137E1E7485E0308605E030838
:1045600020000020955E0308BC5E0308AC1E0020FE
:1045700000007A441F5F0308E55E0308365F030806
:104580000E5F030830B5044685B008461449154649
:10459000FDF768FDFDF742FFCCB1114902902846B6
:1045A000FDF760FDFDF73AFF0E4901902846FDF743
:1045B0004FFC0D49FDF70AFEFDF756FF0022009063
:1045C0000A4B1146032010F075F905B030BD00907C
:1045D000074B22462146032010F06CF9F5E700BF97
:1045E00000007A44CDCC4C3FCDCCCC3E4F5F03088D
:1045F0007C5F03082DE9F04FADF2344D4FF40072AB
:1046000000210CA829F0B6FF4FF4007200218CA8FD
:10461000B34E29F0AFFF002537464FF000082C4677
:10462000B9682046FDF716FC796804462846FDF770
:1046300011FC08F10408B8F5007F054607F11007E2
:10464000EED14FF070512046FDF70CFD4FF0705148
:1046500004462846FDF706FD0025DFF8848207465C
:104660004FF00009AA46D8F808002146FDF7F0FBF4
:104670000146FDF7F7FC01465046FDF7EBFB3946D6
:104680008246D8F80400FDF7E3FB0146FDF7EAFC9B
:1046900001462846FDF7DEFB09F10409B9F5007F64
:1046A000054608F11008DED14FF070515046FDF775
:1046B000D9FC4FF070510A902846FDF7D3FC824692
:1046C0000A98FDF741F8874B00222BF0C9FECDE98F
:1046D00004015046FDF738F8824B00222BF0C0FE53
:1046E000FDF762FB0DF130090546C84600234FF087
:1046F000000BB168B0690693FDF7AAFBFDF78EFECB
:104700000028B8BF4042FDF759FC48F8040B0146A9
:104710005846FDF79FFB069B0433B3F5FE7F8346A7
:1047200006F11006E5D17049FDF750FD0DF1300896
:10473000064600234FF0000B314658F8040B069351
:10474000FDF786FB0146FDF78DFC069B01461846EA
:10475000FDF780FB0BF1010B1FFA8BFBBBF17F0F09
:104760000346E9D16049FDF731FDFCF7EDFF5D4BF4
:1047700000222BF075FECDE906010DF50C78C3463D
:10478000002200234846D9F8001040680B93089295
:10479000FDF75EFBFDF742FE0028B8BF4042FDF783
:1047A0000DFC089A4BF8040B01461046FDF752FB2E
:1047B0000B9B01339BB27E2B09F104090246E1D128
:1047C0004A49FDF703FD4FF0000B8146002349469F
:1047D00058F8040B0893FDF73BFB0146FDF742FC3C
:1047E000089B01461846FDF735FB0BF1010B1FFA3C
:1047F0008BFBBBF17E0F0346E9D13C49FDF7E6FC9C
:10480000FCF7A2FF374B00222BF02AFECDE908016E
:1048100037492846FDF726FCFDF700FE3449029093
:104820005046FDF71FFCFDF7F9FD31490190384670
:10483000FDF718FCFDF7F2FD00222E4B009011460B
:10484000022010F037F82C4A13889BB2FA2B00F2A2
:10485000D580108880B2FDF7B1FB2946FDF7B4FD85
:10486000264F08B105233B70254B1A78254B1B8832
:104870009BB29A4280F08D80234B1A78234B1B8881
:104880009BB29A4206D222492046FDF7A7FD08B105
:1048900001233B701F4FDFF880A03B880A9A013349
:1048A0009BB23B803B889BB20A2B04BF00233B801A
:1048B0003B884FF01C0B9BB20BFB03F3DDE90401BB
:1048C0004AF803403B889BB20BFB03A35A603B882A
:1048D0009BB20BFB03A8FDF767FA3B881EE000BF05
:1048E0002C1600200000E03F0000FE420000FC42C9
:1048F00000007A44925F03083C000020121500205B
:10490000A70300200A150020A60300200815002098
:10491000CDCC4C3F2C1E002014150020C8F80800F8
:104920009BB20BFB03A34FF08641DD603D88304610
:10493000FDF798FBADB20BFB05A528613D88DDE9CD
:104940000601FDF731FA4FF08641FDF78BFBADB262
:104950003B880BFB05A59BB26861334D0BFB03AA9B
:104960002A788AF81820DDE90801FDF71DFA4FF0D2
:104970008641FDF777FBFDF777FD2C4BC0B2188021
:104980002B78012B05D10022294B114602200FF074
:1049900091FF284F244D3B78DFF89C80012B24D1D8
:1049A000DFF89890264EB9F80030B9F800204FF0A3
:1049B0001C0A9BB292B20AFB03F30AFB0262F05894
:1049C0009168FDF747FA2146FDF708FDC0B10223C3
:1049D0002B702B78022BD8B204D10022194B114630
:1049E0000FF068FF2B78DBB23B702B78DBB23B70AB
:1049F000C8F800400DF2344DBDE8F08F12482CE7A6
:104A0000B9F80030D8F800909BB20AFB0366204644
:104A1000B168FDF71FFA4946FDF7E0FC10B103232A
:104A20002B70E2E72870E0E7121500200615002041
:104A3000D85F0308101500200C1500202C1E002044
:104A4000141500201D60030800007A432DE9F04F83
:104A50009FB0FDF737FF12F0A1FF024640B90146B3
:104A6000A84B03200FF026FF01201FB0BDE8F08FF8
:104A7000012013F03BF810F04FFC04460D9040B9B4
:104A800002460146A04B03200FF014FF12F0FAFF7C
:104A9000EAE79E4F3B78012BDDB252D0022D6FD05A
:104AA000002D39D1042110F0FDFF0121204610F026
:104AB00027FF9749204610F057FF9649204610F0EF
:104AC00039FF9549204610F0E7FE9449204610F042
:104AD000FDFE0221204611F019F89149204610F000
:104AE000FBFF214606A810F059FF8E4A19928E4A04
:104AF0001A924FF07C53002218A9204618931B925B
:104B00001C921D9310F076FF2946204610F096FF68
:104B10000321204610F0ACFF0D9800243C7010F0EB
:104B200091FC02460E9000286DD1804B0146032077
:104B30000FF0C0FE0DA810F05DFC0EA810F010FDE7
:104B4000A4E77B4E294610F0DBFE7149204610F0A9
:104B50000BFFB168204610F09FFEF168204610F070
:104B6000B5FE716A204610F0E5FEF16C204610F0AB
:104B7000B3FF704B0022114601200FF09BFECBE7E4
:104B80006B4D012110F0BCFEE969204610F0ECFEEF
:104B9000696A204610F0CEFEA968204610F07CFE1F
:104BA000E968204610F092FEA86CFDF75DFC81B22A
:104BB000204610F0ABFFE96C204610F08DFF214637
:104BC00006A810F0EBFE2B6B18936B6B1993AB6B75
:104BD0001A93EB6B1B932B6C1C9318A96B6C1D9396
:104BE000204610F007FFA86AFDF73EFCC1B2204640
:104BF00010F024FF286AFDF737FCC1B2204610F000
:104C00009FFF4D4BB6E710F041FD38B900224B4BEA
:104C1000114603200FF04EFE002026E71422214605
:104C200013A829F0A7FC0026DFF8EC80DFF810912C
:104C3000DFF810A1212537460E980FA910F07EFD50
:104C40000246002840F08A8001463F4B03200FF0C7
:104C500031FEDFF8F8800E9810F038FDB8F800301B
:104C600000229BB2114600930320394B0FF022FE25
:104C70000D9D0121284610F043FE0421284610F026
:104C800011FF2349284610F06FFE2249284610F0F4
:104C900051FE2149284610F0FFFD2049284610F01A
:104CA00015FE0221284610F031FF1D49284610F05C
:104CB00013FF294606A810F071FE1A4A1992254AD8
:104CC0001B924FF07C534FF07E5218A928461C923D
:104CD00018931A931D9310F08DFE0021284610F0B2
:104CE000ADFE0321284610F0C3FE0D990EA810F06A
:104CF00061FC0246002840F084800146164B0220E9
:104D000016E700BF485E030862600308A81E002083
:104D1000000082429A99993FCDCC4C3F0000204040
:104D20006666263F000020410AD7233CE460030862
:104D3000301E002082600308B2600308FF60030891
:104D4000CDCCCC3EA40300201D6103082E1E002004
:104D500046610308CDCC4C3E7B610308119A109943
:104D60009DF83C00FFF70EFC9DF83C30FBB1DDF8F0
:104D700044B038465946FDF76DF81099074630465D
:104D8000FDF768F8414606465846FDF761F8494682
:104D9000FDF71CFAFDF768FB1EAB80B203EB400089
:104DA000013430F82C3C0133E4B220F82C3C9AF862
:104DB0000030012B1ED1DFF81CB2874ABBF800304F
:104DC00011999BB202EB03139960BBF800309BB2C0
:104DD00002EB0312109B5360BBF800309BB25A1CCD
:104DE00092B2802BABF8002004D1FFF703FC002324
:104DF000ABF800300F20FDF7DDFD013D7FF41CAF67
:104E000027E70E9810F042FC00283FF4FFAE0DA8F3
:104E100010F0F0FADFF8C4B14FF021090E980FA995
:104E200010F08CFC054600287ED1024601466C4BF2
:104E300003200FF03FFDB8F80030DFF8A891DFF84D
:104E4000A8B100229BB2114600930320674B0FF0DC
:104E500031FD012C94BF0023012389F8003000F0BC
:104E6000B1FD99F800300022CDE900431146604BB6
:104E700003200FF01FFD0DF14C084FF0000A38F829
:104E8000022B3AB1CDE900A200225B461146012077
:104E90000FF010FD0AF1010ABAF10A0FEFD15549DE
:104EA0003846FDF7DFF807462046FDF787F88046CD
:104EB00001463846FDF78AF94E4907463046FDF768
:104EC000D1F84146FDF782F94B4B1F604B4B002157
:104ED00018608046FDF75AFA0646A8B942234046B4
:104EE00099F80090CDE90343FDF798FA029038460F
:104EF000FDF794FA5FFA89F9CDE90090404B32460C
:104F0000314603200FF0D6FC0E9810F0DFFB04466C
:104F10000EA810F025FB12F0B5FD002C3FF4A4AD57
:104F200085F00100C0B2A0E5119A10999DF83C00EF
:104F3000FFF728FB9DF84930002B43D19DF83C300A
:104F4000FBB1DDF844A038465146FCF783FF1099C9
:104F500007463046FCF77EFF2A4906465046FCF7D6
:104F600077FF5946FDF732F9FDF77EFA1EAB80B2A6
:104F700003EB4000013430F82C3C0133E4B220F85C
:104F80002C3C214B1B78012B1CD1B8F80030124A65
:104F900011999BB202EB03139960B8F800309BB2F1
:104FA00002EB0312109B5360B8F800309BB25A1CFE
:104FB00092B2802BA8F8002004D1FFF71BFB00233E
:104FC000A8F800300F20FDF7F5FCB9F101097FF4D6
:104FD00025AF30E72E1E00202C160020CDCCCC3E75
:104FE0001D6103088B1E0020FA6103089B61030802
:104FF000C661030800007A44841E0020801E002041
:105000001A620308CDCC4C3FA40300202DE9F043E5
:10501000ADB014230DF10E0204A9ADF80E3012F05C
:1050200045FF044648B902460146194B03200FF0DC
:1050300041FC20462DB0BDE8F0830022154B164FF1
:10504000DFF85880DFF85890114603200FF032FC4B
:105050000025BDF80E30AAB29342EAD9AAB22CAB11
:1050600003EBC202032012F89C6C52F8A03C002E05
:1050700014BF3A464246CDE9003200224B46114663
:105080000FF018FC002E05F1010508BF3446E0E7DB
:1050900074620308976203086A6203086F62030878
:1050A000BB62030830B5102289B0002529460446AA
:1050B0000DEB0200039529F05DFA14F0A1FA2A46DF
:1050C000A34B0090294603200FF0F4FBFDF7FAFBF9
:1050D00012F064FC8DF80C0012F00AFD431B18BF9F
:1050E000012301218DF80D30029012F01FFD02986E
:1050F00012F0BEFE029812F033FD0298FFF786FF11
:10510000002840F0008102A812F002FD12F0BAFC63
:10511000029812F041FD029812F05AFD0298FFF732
:1051200075FF002840F0F38002A812F0F1FC12F0A5
:10513000A9FC029812F068FD0022864B114603205C
:105140000FF0B8FB029812F07BFD0298FFF75EFFAC
:10515000002840F0E08002A812F0DAFC12F092FC85
:10516000029812F089FD002211467B4B03200FF0BC
:10517000A1FB0022794B114603200FF09BFB029804
:1051800012F006FE0298FFF741FF002840F0C780AA
:1051900002A812F0BDFC12F075FC029812F014FE89
:1051A000002211466E4B03200FF084FB00226D4B52
:1051B000114603200FF07EFB029812F021FE0298A8
:1051C000FFF724FF002840F0AE8002A812F0A0FCF8
:1051D00012F058FC029812F02FFE00221146624B8A
:1051E00003200FF067FB0022604B114603200FF0F5
:1051F00061FB029812F05CFD0298FFF707FF0028A0
:1052000040F0958002A812F083FC12F03BFC02985B
:1052100012F06AFD00221146554B03200FF04AFBA5
:105220000022544B114603200FF044FB029812F069
:1052300077FD0298FFF7EAFE00287CD102A812F061
:1052400067FC12F01FFC029812F086FD0022114646
:10525000494B03200FF02EFB0022404B1146032048
:105260000FF028FB029812F093FD0298FFF7CEFE94
:10527000002864D102A812F04BFC12F003FC029843
:1052800012F0A2FD00221146354B03200FF012FB55
:105290000022344B114603200FF00CFB029812F051
:1052A000AFFD0298FFF7B2FE00284CD102A812F021
:1052B0002FFC12F0E7FB029812F0BEFD002211460F
:1052C000294B03200FF0F6FA002211462B4B032046
:1052D0000FF0F0FA01238DF8173003AB03CB002257
:1052E0002060186861600C23A060114600930320C1
:1052F000234B0FF0DFFA02A812F00AFC12F0C2FBF7
:10530000002009B030BD01238DF80E3000E70123E5
:105310008DF80F300DE701238DF8103020E70123C1
:105320008DF8113039E701238DF8123052E701234F
:105330008DF813306BE701238DF8143083E70123D8
:105340008DF815309BE701238DF81630B3E700BFC9
:10535000D1620308FA6203082D6303085E63030841
:105360008D630308BA630308EF630308226403082C
:105370005564030886640308B6640308E4640308FC
:105380001165030802480122102103F081BA00BF11
:105390000004004802480022102103F079BA00BF3F
:1053A0000004004813B5134C23785BB9E37C03F089
:1053B000FF023BB9104B1146022002B0BDE810407D
:1053C0000FF078BAFEF79CF800380C4B18BF01209C
:1053D000400018701A78022A02BF00222270E2747C
:1053E0001B7800930022064B114603200FF062FA4F
:1053F00002B010BD5E21002030650308081F0020A8
:105400004C65030838B5184C23785BBBE37C03F08C
:10541000FF023BBB154D2B68012B0CD92B68042BCD
:1054200009D81146124B02200FF044FA114A042108
:10543000012000F095FF2B68042B13D900220E4B9E
:10544000114602200FF036FAFEF75AF800380B4BDF
:1054500018BF0120400018701B78022B02BF0023E8
:105460002370E37438BD00BF5E210020041F0020BC
:1054700063650308886503088D650308081F00201D
:1054800010B5124C237863B101214FF0904003F026
:10549000F9F90F4B0022187022701B780D4ADBB20D
:1054A00013700D4C237863B102214FF0904003F04C
:1054B000E9F90A4B0022187022701B78084ADBB207
:1054C0001370BDE81040FEF737B900BFAA1E0020D8
:1054D0000A01002008010020A91E00200901002067
:1054E0000701002010B5164B1A78022A26D91B781E
:1054F000072B23D8FFF7AAFA1248134A037811782A
:105500005B1A124918BF01230B7003781048DBB2F5
:105510001370104B104A1C780378E31A18BF01234C
:1055200013700E4B04701B7823B100230B700C49D1
:105530000B701370BDE81040FEF7FEB810BD00BF41
:10554000060100208B1E0020881E00208C1E0020DB
:10555000101500201215002011150020081F002032
:105560008E1E002008B501214FF0904003F08AF90B
:10557000064B012816BF022218701A701878044BC7
:105580001978BDE80840FEF743B800BF06000020C8
:105590000000002038B5324D324C287BFCF70AFD64
:1055A0003149FCF75FFDA060687BFCF703FD2E49E5
:1055B000FCF758FDE060A87BFCF7FCFC2A49FCF7EF
:1055C00051FD6062E87BFCF7F5FC2849FCF74AFDD9
:1055D000274BE0642361287CFCF7ECFC6060687C6E
:1055E000FCF7E8FCA061A87CFCF7E4FCE061E87C47
:1055F000FCF7E0FC2062287DFCF7DCFCA062687D03
:10560000FCF7DCFC1849FCF72DFD2063A87DFCF7B6
:10561000D1FC6063E87DFCF7D1FC1449FCF722FD66
:10562000A063287EFCF7C6FCE063687EFCF7C6FC3E
:105630000D49FCF717FD2064A87EFCF7BFFC0A4962
:10564000FCF710FD6064E87EFCF7B4FCA064287FE2
:10565000FCF7B0FC074BE06202221A7038BD00BFB5
:1056600058030020301E0020CDCCCC3D0AD7233C6F
:10567000CDCCCC3EA81E002038B5114D114C287B56
:10568000FCF79CFC1049FCF7EDFCA060687BFCF784
:1056900095FC0D49FCF7E6FCE060A87BFCF78EFC6E
:1056A0000949FCF7DFFC6062E87BFCF787FC0749EF
:1056B000FCF7D8FC064BE06401221A7038BD00BF2D
:1056C00058030020301E0020CDCCCC3D0AD7233C0F
:1056D000A81E002073B52B4D2B4E2B7803702B4B3F
:1056E0001B784370044601214FF0904003F0CAF844
:1056F0003378A070E37002214FF0904003F0C2F8BD
:10570000234B20711B7863713378012B37D1214BE8
:105710001868FCF7A9FE204BE0801868FCF7A4FE8F
:1057200080B21E4BA0831B7884F82430191F4A4294
:105730004A41012BA2770FD1194B00930022194B3C
:10574000114602200FF0B6F8174B1B8884F825305D
:10575000164B1B8884F82630154B1B7853B1154B1C
:105760001B683BB1144B1B78012B01BF134A082364
:1057700013702B70124B01221A7002B070BD002002
:10578000E080CEE7060000208B1E002006010020EE
:105790008A1E0020841E0020801E0020121500207A
:1057A00052000020C06503080A15002006150020DD
:1057B000A5030020A41E00205B210020070000207C
:1057C000001F0020024B0122002103200FF072B8BD
:1057D000EE65030808B50122074B002103200FF0F6
:1057E00069F8FFF7CFFDFFF7D5FE044A00231370D9
:1057F000034A137008BD00BF34660308A81E0020CA
:105800005921002010B5134B0122002102200FF076
:1058100051F8114B04225A700024012263211A709E
:1058200083F82D1083F82E201C635C639C63DC637B
:105830001C645C649C64DC6483F827401C855C8485
:105840009C77FFF79FFDFFF7BDFFFFF7C3FF034BFB
:105850001C7010BD6A660308B01E0020592100208C
:105860001FB5114B11491C6858681A7A5B7ACDE94B
:105870000223FCF7F7FBFCF7F7FD0C4901902046EB
:10588000FCF7F0FBFCF7F0FD0022094B00901146FD
:1058900003200FF00FF8FEF78BFD642004B0BDE885
:1058A0001040FEF7B5B900BF2000002000007A4488
:1058B000A166030870B586B00D460446FFF762FD89
:1058C00001F0E6FEFDF73CFB9620FEF7A1F900266D
:1058D000AE420AD101AB03CB1B882381094B206068
:1058E000002261601A7006B070BDFEF769F801A869
:1058F000FFF7D8FB41F28830FEF78AF90136FFF74F
:10590000AFFFE5E75921002030B585B004460025FA
:1059100003A8ADF80C50FCF7D9FF70B19DF80C301E
:105920009DF80D20237062702946CDE900320320D6
:10593000034B2A460EF0BEFF012005B030BD00BF6C
:10594000D6660308022801D8FFF71CBD704702285D
:1059500001D8FFF71FBD7047022803D80248102165
:1059600002F09BBF704700BF0004004807B56846BF
:105970000FF002FA064A009B1178064A19B9136320
:1059800003B05DF804FB116B5B1A5363F8E700BFCB
:1059900003000020B01E002007B568460FF0ECF9A8
:1059A000064A009B1178064A19B9936303B05DF863
:1059B00004FB916B5B1AD363F8E700BF0200002081
:1059C000B01E002007B568460FF0D6F9084A009BC4
:1059D0001178012904D1074A136403B05DF804FB70
:1059E0001278002AF9D1034A116C5B1A5364F4E768
:1059F0008B1E0020B01E002008B5FEF755F8BDE84C
:105A0000084000F0DBBE4FF0FF300FF09DB870474C
:105A100070470000014BD870704700BF180100208C
:105A2000014B1874704700BF1801002007B5064BE2
:105A300000221B5C00931146044B02200EF03AFF3B
:105A400003B05DF804FB00BF15670308FB6603089D
:105A500008B5002102200FF03FF80A4B1B7803F035
:105A6000FF014BB9084B1A68042A05D81A681020A0
:105A700001321A600FF030F8BDE8084003480FF01B
:105A800093BA00BF5E210020041F0020C020002028
:105A9000002101200FF020B813B5104A104C42F23B
:105AA0001073002818BF03460E48236013600FF0E0
:105AB0002DFA21680B480FF0B1FA0A480FF074FA7A
:105AC00023684FF47A72B3FBF2F30022009311467D
:105AD000054B01200EF0EEFE02B010BD9C0300202D
:105AE00014010020C02000201967030813B50D4CD5
:105AF000206023680BB90C4B23600C480FF006FAAA
:105B000021680A480FF08AFA08480FF04DFA236816
:105B100000930022064B114603200EF0CBFE02B08C
:105B200010BD00BF9C030020A08601000C1F0020B8
:105B30004567030813B50F4C2060236813B942F280
:105B4000107323600C480FF0E1F921680A480FF048
:105B500065FA09480FF028FA23684FF47A72B3FB0C
:105B6000F2F3002200931146044B01200EF0A2FE36
:105B700002B010BDA0030020241F0020816703088D
:105B800037B50446002841D090F90650002D4AD17F
:105B900028480FF0BBF9FDF72BFD274B01221A70A7
:105BA000FDF7DCFC2A462946244B02200EF082FE3B
:105BB000E379012B0CBF224B224B2A4629460220B7
:105BC000214D0EF077FEE3792B70204B1868FFF71C
:105BD0008DFF1F4B1868FFF75FFF29781D4A1E4B8A
:105BE000012908BF13460022009311461B4B0120D8
:105BF0000EF060FE94F90530019394F9043000939F
:105C00000022174B114603200EF054FE154B0122C3
:105C1000002102201A700EF05FFF134803B0BDE8A8
:105C200030400FF0C1B90022104B114602200EF097
:105C300041FEDFE76C1F002006000020C367030859
:105C4000D8670308F56703085A2100209C03002049
:105C500014010020BA670308BE670308126803082E
:105C60004A68030858210020541F002031680308A7
:105C70000A460149FDF71EB900F0030870B5164841
:105C80000FF044F906F002FF044650B10022134B16
:105C9000114602200EF00EFEBDE8704010480FF0D5
:105CA00083B9104D104B0246014602200EF002FE51
:105CB00001260E4B2E702246214602200EF0FAFDE0
:105CC0000B4806F077FD2878314606F0CBFA0248FB
:105CD0000FF06AF9E0E700BFC020002073680308F6
:105CE000A82000207C01002091680308A568030813
:105CF00018010020F0B59FB0FDF708FF054606F03B
:105D0000ABFB074600283ED16F4C0AA8FFF7E2FC28
:105D1000132323706D4B1A7802F0FF06002A43D03C
:105D20001F70142323706A4B62681B7863F07F0333
:105D30001370636828B200EB400000EB4010FE22B5
:105D4000B0FBF2F058700223624A1278012A88BF31
:105D500000236370604C637A33B106F069FB01285D
:105D600002D120460FF0D2F85C4B5748D978002278
:105D700006F088FB0146002840F091800122584B34
:105D800010460EF097FD002456480FF0BFF8564B12
:105D900054481968A14238BF21460FF03FF95148D5
:105DA0000FF002F91FB0F0BD504A117801F0FF0367
:105DB0000029C9D0464B16701B78626863F07F03D8
:105DC000137063689DF828505D7062689DF82930F3
:105DD000937062689DF82A10D17062689DF82B104C
:105DE000117162689DF82C10517162689DF82D1038
:105DF0009171BDF82E206168120ACA716068BDF801
:105E00002E200272BDF84420120A4272BDF84420CE
:105E100082729DF84620C2729DF84C2002739DF854
:105E20004F204273BDF85020120A8273BDF85020F3
:105E3000C27303EB83032E4A03EB830313440193E2
:105E40002C4B05EB850503EB4503009332462A4BAB
:105E5000314601200EF02EFD9DF84C300893BDF820
:105E60004A3007939DF846300693BDF844300593B9
:105E7000BDF82E3004939DF82D3003939DF82C30FF
:105E800002939DF82B3001939DF82A3000933246FF
:105E90001A4B314601200EF00DFD102354E7063158
:105EA0007FF471AF06F0BEFA044600283FF46BAFF2
:105EB00001224FF47A730021B0FBF3F310460093F4
:105EC0000F4B0EF0F7FC5FE70C010020582100207B
:105ED000B41F0020081F00206C1F002018010020A4
:105EE000F9690308C020002014010020001F0020D1
:105EF0007D010020F4020020C4680308EC68030858
:105F0000086A030813B568460EF036FF164B009A70
:105F10001978164B11B9196B511A596314485C6BF7
:105F200001788C4205D9012183F82710596B89B279
:105F300019851049097811B9996B511AD9630E491D
:105F40000978012902BF196C521A5A64596C0278F7
:105F5000914205D9012283F82C205A6C92B25A85BD
:105F6000064B1B7802B010BD03000020B01E0020BD
:105F7000A5030020020000208B1E00201215002027
:105F800000B503468DB000282CD0407802280AD0F6
:105F900003282AD0164B0022114602200DB05DF8CE
:105FA00004EB0EF087BC1A7F0B92DA7E0A929A7E7F
:105FB00009925A7E08921A7E0792DA7D06929A7D9D
:105FC00005925A680492DA68039293F914200292B7
:105FD000B3F9122001921B7C00930022054B11465D
:105FE0000EF068FC0DB05DF804FB034BD3E700BF77
:105FF000266A03083D6A0308AF6A030801284FF0C8
:1060000000020CBF024B034B114602200EF052BCA3
:10601000CE6A0308E06A03081FB50446002831D0A1
:106020000378002B2ED01D480EF0BEFF0022114633
:106030001B4B02200EF03EFC94F91830039394F9A8
:106040000A300293237C0193E368009300221146F7
:10605000144B03200EF02EFC0022134B114603209C
:106060000EF028FC237A012B0ED1617A0F4A104BD7
:10607000002918BF13460022009311460D4B032040
:106080000EF018FC04B010BD00220B4B114603208B
:1060900004B0BDE810400EF00DBC00BF9C1F0020F6
:1060A000F96A03082A6B03085B6B0308F56A0308A7
:1060B000F46A0308686B0308796B030808B5104B92
:1060C0000122002102201A700EF006FD0D480EF08C
:1060D0006BFF0D4B1B788BB10C4B1A7872B9DB7CC4
:1060E00063B90B4B1A68042A9EBF1A6801321A6002
:1060F0000021BDE8084010200EF0EEBC08BD00BF36
:10610000582100200C1F00205A2100205E21002071
:10611000041F002008B5002140200EF0DDFC074BD5
:106120001B7853B1064B1A78012A06D10021197049
:10613000BDE8084002200EF0CFBC08BD5A21002067
:106140008C1E0020044B1B78022B03D10021082059
:106150000EF0C2BC704700BF7C010020044B1B78CE
:10616000012B03D0002180200EF0B6BC704700BF89
:106170000601002008B506F092FC80B906F058F937
:1061800001280CD1BFF34F8F0549064BCA6802F4B2
:10619000E0621343CB60BFF34F8F00BFFDE708BD44
:1061A00000ED00E00400FA0538B504460D46074846
:1061B0004FF40061FCF79EFE30B92A4621460348A1
:1061C000BDE83840FCF79CBD38BD00BF00F00308B7
:1061D00010B506F0F9FC10F1080F07D1064B0022AC
:1061E000BDE81040114602200EF064BB013001D121
:1061F000024BF4E710BD00BF876B03089D6B0308DB
:1062000038B5154C2378082B0DD1144C23781E215A
:106210000BB1022000E00320FDF76CFA237883F035
:106220000103237038BD2378092B07D10B4C237849
:106230001E2103F0FF00002BEED0EAE7084D2A787C
:1062400023789A42EED020781E21FDF753FA237866
:10625000DBB22B70E6E700BF0600002098030020A9
:106260005C21002070470000022837B5044636D074
:1062700040285CD001285DD12F4B1B78002B59D0D2
:10628000FA20FDF7C5FC21464FF0904002F0FAFAE3
:106290002A4B214618704FF0904002F0F3FA214645
:1062A00005464FF0904002F0EDFA254A254B0028B4
:1062B00008BF13460022CDE900531146224B0220AD
:1062C0000EF0F8FAFFF752FB002120200EF004FC3C
:1062D0000021022003B0BDE830400EF0FDBB1B4B97
:1062E0001B783BB3FA20FDF793FC21464FF090401A
:1062F00002F0C8FA164B214618704FF0904002F099
:10630000C1FA214605464FF0904002F0BBFA114A0F
:10631000114B002808BF13460022CDE90053114657
:106320000E4B20460EF0C6FAFFF736FBCCE70021F5
:106330000420CFE703B030BDAA1E002003000020D8
:10634000B56B0308C16B0308E76B0308A91E0020A7
:1063500002000020CD6B0308DA6B03080D6C030804
:1063600073B505460C46164606F076F80346002837
:1063700040D000242A480EF0C9FD2A4B284819684D
:10638000A14238BF21460EF049FE254802B0BDE8C3
:1063900070400EF009BE4A68F05CD0540133DAB2A6
:1063A0009442F8D8204B0D701A781B78012A88BFC8
:1063B00000244C700022CDE900341C4C1C4B1146CB
:1063C00001200EF077FA637A33B106F031F8012834
:1063D00002D120460EF09AFD164B1748D9780022BC
:1063E00006F050F8014638B9144B012203200EF094
:1063F00061FABEE71049D2E70631BAD106F012F8C9
:1064000004460028B6D04FF47A730122B0FBF3F3B0
:106410000021009303200A4B0EF04CFAAAE700BFBC
:10642000C020002014010020081F00206C1F002045
:10643000326C0308180100200C010020F9690308E0
:10644000086A0308044B1B7823B9044A052101207C
:10645000FFF786BF704700BF081F0020636C03086A
:1064600010B5002490B03C22214601A8009428F0E9
:1064700081F8374B2022DA7219788DF8001059789C
:106480008DF8011099788DF80210D9788DF80310E5
:1064900019798DF8041059798DF8051099798DF8CE
:1064A0000610D9798DF80710197A8DF80810597AE5
:1064B0008DF80910997A8DF80A108DF80B20214675
:1064C0000DF10B0258180131007B02F8010F14295D
:1064D000F8D193F827208DF8202093F828208DF804
:1064E000212093F829208DF8222093F82A208DF876
:1064F000232093F82B2093F828108DF82420154A98
:1065000011BB93F8291001F0FF00E9B9107093F85E
:106510002C2062B193F83F204AB109A900229818B3
:10652000013290F82C0001F8010F142AF7D10A4823
:106530004FF40061FCF7DEFC20B9074840226946B1
:10654000FCF7DEFB10B010BD01211170DFE700BFCA
:1065500058030020A403002000F8030810B500220F
:1065600004461146054B02200EF0A4F920460449CA
:10657000BDE8104040220EF0A3BA00BF696C0308CA
:1065800000F8030838B5434C207963794D2BC0B22D
:1065900069D1C0EB001080000A2838BF0A204FF4F0
:1065A0007A7358433C4B1860A379E2794D2ADBB2E9
:1065B00061D1C3EB03139B004FF47A7202FB03F526
:1065C00094F82C30002B5ED194F83F30002B5AD138
:1065D00042F21070FFF760FA304B1868FFF786FA46
:1065E000237A2F4A2F49DBB213702F4B01221A70E6
:1065F000637A2E4ADBB2137094F827302C4ADBB250
:10660000137094F828302B4A03EB83035B00DBB252
:10661000137094F82930284A03EB83035B00DBB244
:10662000137094F82A30254A0133DBB2DB01138062
:1066300094F82B30224A03EB83035B00DBB2137028
:106640000023E21892F82C20D2B2CA540133142B42
:10665000F7D1A378012B1CD1E37A202B19D1BDE807
:106660003840FFF7CFB86379482B0ABF4FF4616316
:106670006379584390E7E279482A0ABF4FF4616290
:10668000E279534398E7FFF707FA2846FFF752FAF3
:10669000A6E738BD58030020140100209C03002009
:1066A000060100205E21002006000020081F0020B7
:1066B00005000020A7030020A60300203C000020C6
:1066C000A503002010B590B000213C2201A8009144
:1066D00027F050FF4022364968460EF0F1F99DF848
:1066E00000203AB99DF80100102803D19DF802104E
:1066F00001290FD000222F4B114602200EF0DAF8AC
:10670000FFF7AEFE4FF47A70FDF782FAFFF73AFF1B
:1067100010B010BD284B1A70587099709DF8031076
:10672000D9709DF8041019719DF8051059719DF8E4
:10673000061099719DF80710D9719DF8081019720B
:106740009DF8091059729DF80A1099729DF80B1066
:1067500001F03F01D972D87AD1B288421FD89DF892
:10676000272083F827209DF8282083F828209DF8EB
:10677000292083F829209DF82A2083F82A209DF8D3
:106780002B2083F82B200DF12B01002298180132C9
:1067900011F8014F80F82C40142AF7D1B6E701F127
:1067A00040006844194410F8340C08730132D2E7F1
:1067B00000F803087D6C030858030020F0B50C2393
:1067C0008BB0052600240125CDE90563182210238E
:1067D000CDE903322146714B029422460327CDE9CD
:1067E0000055022009940EF065F86D4B0294224684
:1067F0002146CDE9005702200EF05CF8CDE9016496
:106800000226684B00962246214630460EF052F88A
:10681000654B009522462146CDE9017430460EF0C5
:1068200049F809A9204606F01FF9099BC3F307227E
:106830000292C3F307421B0E0192009322465B4B68
:10684000214630460EF036F809A9284606F00CF924
:10685000099BDAB20392C3F307220292C3F3074201
:106860001B0E019200932246514B214630460EF0FA
:1068700021F8504B5048009422464FF4FA710EF024
:10688000E7FA4E4B4E48009422464FF4FA710EF050
:10689000DFFA4C4B4C4800942A464FF4FA710EF044
:1068A000D7FA4A4B4A4800942A464FF4FA710EF040
:1068B000CFFA484B484800942A4642F210710EF035
:1068C000C7FA2046FCF716FA08B1FCF737FC434B31
:1068D000009400224FF4FA6141480EF0B9FA414A9F
:1068E000002101200EF0B4F93F4A002102200EF0F1
:1068F000AFF93E4A002104200EF0AAF93C4A0021DB
:1069000008200EF0A5F900F01DFE3A493A4806F0BD
:1069100061F83A4805F04EFF2B480EF045FB384B26
:106920000021187805F09EFC36490094364B096822
:10693000364800220EF08CFA34480EF035FBFFF793
:10694000C1FE334A002110200EF082F9314A0021A5
:1069500020200EF07DF9304A002140200EF078F919
:106960002E4A002180200EF073F92D4B2D48196816
:106970002D4B009401220EF06BFA2A480EF014FB06
:106980002A4B2B4819682B4B009401220EF060FA19
:1069900027480EF009FB0BB0F0BD00BFBD6C03082B
:1069A000FD6C03081E6D03083F6D0308606D03084E
:1069B000816D03080F5A00089C1F002065620008C3
:1069C000841F00205D6100086C1F00200162000828
:1069D000541F0020055F00083C1F0020456100088F
:1069E000A8200020B9C50008F55C0008D1610008A6
:1069F0007D5C000800000301300100201801002028
:106A00007C01002014010020515A0008C020002001
:106A10000554000881540008E55400086555000835
:106A2000A0030020241F0020156100089C03002003
:106A30000C1F0020BD60000873B50D4D00262E60B0
:106A4000FEF70EFFC820FDF7E3F828683146FBF794
:106A50009DFC04460028F3D12868FBF7DFFC054BBA
:106A600000902246214601200DF024FF02B070BDA7
:106A7000AC1E0020A56D030830B50024A5B07C2213
:106A8000214605A8049427F075FD53238DF8103096
:106A900001254FF48873ADF81230ADF800408DF841
:106AA0001450FDF733F8FE23B0FBF3F000EB400089
:106AB00000EB40103A4B8DF815002246214603208A
:106AC0000DF0F8FE6846FEF71FFF9DF800309DF8B8
:106AD0000120134314D158238DF816300724802247
:106AE0000021304827F046FD224604A92D4827F012
:106AF000D7FD2C4A21460120FFF732FC25B030BDDE
:106B00000E23294601A8CDE901448DF81630ADF8D1
:106B10000C40FEF7CFFE01AB03CB234C1B88CDF816
:106B20001B10ADF81F30CDF81700FEF799FE206856
:106B3000FBF79AFC0A254FF47A7380B2B0FBF3F0AE
:106B4000B0FBF5F305FB130030308DF82100206811
:106B5000FBF78AFC642380B2B0FBF3F0B0FBF5F3E3
:106B600005FB130030308DF822002068FBF77CFC19
:106B700080B2B0FBF5F0B0FBF5F305FB130030304D
:106B80008DF823002068FBF76FFC80B2B0FBF5F3B3
:106B900005FB130030308DF8240015249FE700BF5B
:106BA000D86D0308D8200020AC1E00202DE9F04746
:106BB000044694B0BD480D46802200210DF08AFFA6
:106BC0002378592B40F04082052D5ED86378443BF2
:106BD000162B5AD8DFE813F07C01590059015900EF
:106BE00061015900590059005900BD005900440184
:106BF000590059005900D70159005900E7005900C0
:106C0000590059001700A678482E17D1A84A142118
:106C10000120FFF7A5FB41F28830FCF7F9FF0022C5
:106C2000A44B114603200DF045FE40F6B830FCF7AA
:106C3000EFFF14B0BDE8F047FFF79CBA532E0DD11B
:106C4000FFF71AFF41F28830FCF7E2FF974A15215F
:106C5000012014B0BDE8F047FFF782BB432E17D1E7
:106C6000002404A88DF8104005F01CFD8F4A4C2329
:106C70001370102393709DF810305470012041332D
:106C8000D07013710521FFF76BFB14B0BDE8F087DE
:106C9000442EFAD1854C884DA670592323705A236F
:106CA0006370FFF7C9FE2868FBF7B8FB0022834B2F
:106CB0000090114603200DF0FDFD7F220021601C95
:106CC00027F058FC102326700126A370E670267169
:106CD000FCF71CFFFE23B0FBF3F000EB40000423A5
:106CE00000EB40106071A3712868FBF7BDFB0A2719
:106CF0004FF47A7380B2B0FBF3F0B0FBF7F307FB0D
:106D000013003030E0712868FBF7AEFB642380B2DB
:106D1000B0FBF3F0B0FBF7F307FB13003030207249
:106D20002868FBF7A1FB80B2B0FBF7F0B0FBF7F3EC
:106D300007FB1300303060722868FBF795FB80B2C8
:106D4000B0FBF7F307FB13003030A07222460B2193
:106D50007EE7A378303BDBB2092B96D8584C594AD2
:106D600023702378DBB25372504A592313704D239A
:106D7000537023780321303301209370FFF7F0FA2A
:106D8000237800930022504B114601200DF092FD14
:106D9000FFF766FB23780BB1FCF72AFC14B0BDE8C3
:106DA000F047FCF7C9BCA578482D1BD13F4C5623B2
:106DB00023701023A370182363710523012000257D
:106DC000A37122460C230821E3716570E0702071E5
:106DD000FFF7C6FA3D4B00942A46114602200DF0FB
:106DE00069FD52E7432D7FF450AF00213C2205A8F6
:106DF0002E4C049127F0BEFB04A8FFF7AFFB9DF8D3
:106E0000103063709DF81130A3709DF81230E3705C
:106E10009DF8133023719DF8143063719DF815307F
:106E2000A3719DF81630E3719DF817302570237219
:106E30009DF81B509DF8183063729DF81930A372AD
:106E40002A469DF81A30E37207A904F10D00257354
:106E500027F026FC05F10D012246C9B2012012E7F8
:106E6000A07839280CD83038C0B2FEF76BFD0F4A35
:106E70002378137063785370A37893700321E7E647
:106E800014B0BDE8F047FFF7DDBAA0783928F7D88D
:106E90003038C0B2FEF75BFDE9E7A0783928EFD8BB
:106EA0003038C0B2FEF758FDE1E700BFD82000201F
:106EB000F16D0308066E0308AC1E0020286E03085F
:106EC000081F0020580300204B6E0308746E03084F
:106ED000A378303BDAB2092AD2D8E578303DEAB25D
:106EE000092ACDD82179A1F14802D2B20B2AC7D8FC
:106EF0007A4840FA02F2D007C2D40A224D2902FB96
:106F000003553BD13C235D43754B4FF47A70684386
:106F10001860744B1860FEF7E9FD734A237813700C
:106F200063785370A3789370E378D3700521237945
:106F300013710120FFF714FA6C4B002610221E700B
:106F40005A7001229A70DA70A178303901EB810011
:106F5000E178303901EB4001C9B2197122795A71D7
:106F6000634A1278D2B21A72624A1278D2B25A7254
:106F7000FFF776FA604B009532462EE74829C3D1D9
:106F80004FF46163BFE7A378303BDAB2092A3FF6DA
:106F900077AFE578303DEAB2092A3FF671AF217943
:106FA000A1F14802D2B20B2A3FF66AAF4B4840FA31
:106FB00002F2D2073FF564AF0A224D2902FB0355C6
:106FC0003DD13C235D434D4B4FF47A7606FB05F2F1
:106FD0001A601868FEF7AEFD434A23781370637891
:106FE0005370A3789370E378D370052123791371DC
:106FF0000120FFF7B5F93D4B002710221F705A7092
:1070000001229A70DA70A178303901EB8102E178BF
:10701000303901EB4201C9B299712279DA71344AEF
:107020001278D2B21A72334A1278D2B25A72FFF779
:1070300017FAB5FBF6F5324B00953A46CDE64829EE
:10704000C1D14FF46163BDE7502B40F0A881022D00
:107050007FF61BAE6178A1F13003012B3FF615AE30
:10706000A378312B7FF411AE052D51D1E378302B6D
:1070700040F0C4801E4D234E00232B702B7803F06C
:10708000FF0253B92379303BDBB23370337800937E
:1070900011461D4B02200DF00DFC16491B4A002322
:1070A0000B703378DBB213702B78104ADBB213729B
:1070B0000B78DBB25372FFF7D3F90B4B22781A70BF
:1070C00062785A70A2789A70E278DA7022791A712E
:1070D000FCF732FB0521044ABAE500BFDEF7FFFFEB
:1070E000140100209C030020D82000205803002019
:1070F00006010020081F00209E6E0308A003002048
:10710000D56E0308040000201F6F0308060000204E
:10711000082D67D1E378462B40F0EA802179A1F170
:107120003000C0B2092800F238816279A2F1300340
:10713000092B00F23281A679A6F13003092B00F267
:107140002C81E379A3F13005092D00F2268101EBB2
:1071500081014900AF4D203102EB8202C9B25200D9
:1071600029702032AC49D2B22F3E0A70F6B2AB4A37
:1071700003EB8303F6015B0016802033A84ADBB2E1
:107180001370A84A82F828006379303BDBB282F89A
:107190002930A3792F3BDBB282F82A30E379303BE8
:1071A000DBB282F82B302B782BB90B7803F0FF027F
:1071B0000BB99D4B1A70FFF753F99C4B22781A704C
:1071C00062785A70A2789A70E278DA7022791A712D
:1071D00062795A71A2799A71E279DA71FCF7ACFAA4
:1071E000082178E7042D2FD1E278A2F13003DBB239
:1071F000092B11D9A2F14103192B0AD9FFF722F962
:1072000000228B4B1146012014B0BDE8F0470DF071
:1072100051BBA2F13703DBB286480370834B207861
:107220005970312118709970DA70824B7D4A1B7841
:10723000DBB21372804B1B78DBB25372FFF710F98D
:10724000FCF77AFA042146E71D2D4FD9A61C00252C
:10725000DFF8D091DFF8E4A13746A84617F8012FF0
:10726000303AD2B2092A3ED809EB050303201A733B
:107270001B7BCDE902533B780022CDE90053114638
:1072800053460DF017FB01351E2DE7D1B8F1000F65
:10729000B4D1FEF77FF9654B50221A7000225A7064
:1072A00010229A700122DA7003F8042F203416F8A5
:1072B000012F03F8012FB442F9D15A4B00221A7062
:1072C00010225A7001229A70DA705A4A1278D2B299
:1072D0001A72594A1278D2B25A721E22DA72FFF723
:1072E000BFF82321F7E64FF00108CCE7072D85D939
:1072F00000254C4FDFF8448102342E4614F8012F4C
:10730000303AD2B2092A46D8791903200A730B7B86
:10731000CDE9025323780022CDE9005311464346BC
:107320000DF0C8FA0135082DE8D1002E7FF466AFC4
:10733000FEF7A2F93D4B3B4C50221A7010229A7076
:107340001A460121002502F8041F5D70D9706119E9
:107350000135097B082D01F1300102F8011FF6D13A
:107360000022114600930120354B0DF0A3FA0023B3
:107370002370102363700123A370E3702D4B1B78DF
:10738000DBB223722C4B1B78DBB26372E572FFF722
:1073900067F80D219FE60126C4E700219BE6412BFB
:1073A0007FF473AC6378432B7FF46FAC162D7FF4BE
:1073B0006CAC244D621C002312F8011FE954013308
:1073C000142BF9D1FDF7EEFF1F4B5B7D012B1DD177
:1073D00014490023EA5CC8180133D2B2142B80F898
:1073E0002C20F7D1144B00221A701B78DBB24B72A1
:1073F000FFF736F80D4A631E153413F8011F02F823
:10740000011B9C42F9D1094A162121E40A4B0222B0
:107410001A70EFE7A7030020A60300203C0000201D
:10742000A503002058030020A4030020D82000203A
:107430007E6F030806010020081F00203B6F030831
:10744000636F03085E210020AC09002070B505467B
:1074500088B00C46002951D033480DF0A5FD2678A0
:107460009EB3002D5ED068682E7870B3032E0BD0CB
:10747000132E45D0022E28D16978012925D00B067C
:1074800023D4FFF793FB20E06B78012B07D1007822
:10749000012802D0022800D008B905F0BDF8002567
:1074A0000DF11F008DF81F5005F0FCF81F4A4C230A
:1074B0001370102393709DF81F30557001204133D5
:1074C0000521D0701371FEF74BFF237C052B15D8D7
:1074D00094F90A20059294F909200492144A52F86A
:1074E0002330039394F90830CDE901630022E36867
:1074F000009311460F4B03200DF0DCF908B070BD6E
:107500006B78012BE1D102780B4B02F001021A706B
:107510002AB90A4B114603200DF0CCF9D5E7084BE8
:107520000022F7E72E46D0E7841F0020D820002055
:1075300008700308B66F0308B41F0020A36F030888
:10754000AD6F0308034B0022C3E902220122C3E905
:1075500000227047742100200048704774210020E9
:107560004FF0B04382B0DA6C0243DA64DB6C034064
:107570000193019B02B070472DE9F04186B00024D1
:107580000220154D0594FFF7EBFF0420FFF7E8FFFD
:10759000124F03944FF4807601230DEB0001CDE9E7
:1075A00001632846032304934FF4005801F04AF87E
:1075B00001A93846CDF8048001F044F8224641463E
:1075C000384601F065F928462246314601F060F957
:1075D000204606B0BDE8F0810004004800080048DD
:1075E000032810B50ED8012810D868B902460B48F8
:1075F0004FF4807101F04CF9002209484FF400511A
:1076000001F046F9002010BD0122F0E700220348F6
:107610004FF4807101F03CF90122EEE700040048CC
:107620000008004802207047002070470120704782
:10763000002814BF16200F20704700000D48854613
:1076400000F025F80C480D490D4A002302E0D458FB
:10765000C4500433C4188C42F9D30A4A0A4C00239C
:1076600001E013600432A242FBD326F0EBFFFBF7EC
:1076700047FDFEE70000012000000020C8070020B1
:10768000E8D50308C807002010410020FEE7704736
:1076900010B5032000F06EFC01F07CFA064B186078
:1076A0000F20FCF7ABFA044618B9FBF79FFE204603
:1076B00010BD0124FBE700BFA80300204FF0E0222B
:1076C000136923F00203136170474FF0E02213693E
:1076D00043F0020313617047014BD3F890057047E4
:1076E0000070FF1F014BD3F8940570470070FF1F17
:1076F000014BD3F8980570470070FF1F024A53688A
:1077000043F0010353607047002004E0024A5368CD
:1077100043F0020353607047002004E0024A5368BC
:1077200043F0040353607047002004E08068C0F316
:1077300080007047F7B5002301930446002800F04D
:10774000E980856D25B9FBF765F9E56584F8545046
:1077500023689A68D00040F1A1809A68D10000F1B6
:10776000B480A26D42F01002A265E26D42F0010207
:10777000E26501251846FFF7D9FFA26D02F010025D
:10778000024340F0C980A26D206922F4817242F068
:107790000202A2659A68D2075DD4226BA67E94F895
:1077A0002CC0003A18BF01221703D4E902120A4381
:1077B000217E42EA8132617E42EAC13242EA4632A9
:1077C000002842EA4C02B4BF20F000414FF40011FF
:1077D0003A430A4394F82010012903D1002E76D1B0
:1077E00042F48032616A21B1A66A01F4E07131434A
:1077F0000A43D968E66C21F4FE3121F4FF7111438C
:10780000D96094F83C206168012A01F0404C4CEAB0
:10781000060609D1D4E910273A433243A66C324315
:1078200042EA0C0242F001061F693E4A3A403243E6
:107830001A6121F00042B2F1804F0CD0B1F1004F3B
:1078400009D0394ED6F8082701F4701122F47012CD
:107850000A43C6F808275A69666BA16B22F0070233
:1078600032435A615A6922F0700242EA01125A61A7
:10787000002835D19A6A62F00F029A625B6903F0C0
:1078800007039E423CD10023E365A36D23F003036D
:1078900043F00103A365284603B0F0BD9A6823496D
:1078A00022F0104222F0170242F080529A60204AE1
:1078B0001268B2FBF1F2013252000192019A002AE1
:1078C0003FF44BAF019A013AF7E7002552E7A16D6B
:1078D00041F02001A165E16D41F00101E16581E721
:1078E000B0F5001FCAD19A6AE269013A92006FF0BE
:1078F0000F0102F01C0201FA02F2216E0A43BCE7FA
:10790000A36D23F0120343F01003A365E36D43F06E
:107910000103E3650125BEE7A36D43F01003A365F2
:10792000F8E700BF02FCFF1F00200140400D0300EC
:10793000A8030020F8B54569082D04460E460AD074
:107940000368DB68D80705D5A36D43F02003A36562
:107950000120F8BD0425FCF753F9074623681A688F
:107960002A4220D0A26D42F40072A265DA6812F4B5
:10797000406F14D1A27E92B91A6812070FD518462B
:10798000FFF7D4FE20BB5A6822F00C025A60A26DA9
:1079900022F4807222F0010242F00102A265227EEE
:1079A000FAB10020D5E7711CD9D0FCF729F9C01B2A
:1079B000B04201D8002ED1D123681B682B40CDD115
:1079C000A26D84F8543042F00402A2650320C0E79F
:1079D000A26D42F02002A265E26D42F00102E26572
:1079E000DDE70C221A60DCE70368186C70470000C2
:1079F000F7B50023019390F85430012B044600F0B2
:107A0000C08005680269012380F854302846FFF7DA
:107A10008DFE002840F0AF80D1E90030022822F02E
:107A200004027ED0B2F1004FC3F3110E35D1AA6A21
:107A300042EA0E02AA628A68686902EA032222F018
:107A40007C4222F0FF0220EA03210A43002B6A61F4
:107A50001DDA4D4A4D4DD2F80817AB4201F0E070E7
:107A600043D10D0213D4D2F8083723F0E073034357
:107A700043F40003C2F80837454B1A68454BB2FB84
:107A8000F3F20C2302FB03330193019B53BB002051
:107A9000002384F8543003B0F0BD226E00F01F07BD
:107AA0004FF00F0C0CFA07FC6FEA0C0622EA0C0CE4
:107AB000BEF1000F11D1C3F38462BA4042EA0C0256
:107AC00022668008E26901309042B4D8A86AC3F304
:107AD0008362BA4006403243ACE793FAA3F2B2FAAB
:107AE00082F2EAE7019B013BCEE72B4DAB420BD183
:107AF000C901CCD4D2F8083723F0E073034343F034
:107B00008073C2F80837C2E7244DAB42BFD14B02A5
:107B1000BDD4D2F8083723F0E073034343F4800365
:107B2000EFE7B2F1004F01BFAA6AC3F311018A4324
:107B3000AA62002BABDA154813498342D1F8082713
:107B400009D1D1F8083702F0A07223F0E0731A438C
:107B5000C1F808279BE71048834204D1D1F80837C1
:107B600002F44002F1E70D48834290D1D1F8083782
:107B700002F0C072E9E7A26D42F02002A265184649
:107B800086E7022087E700BF00200140001000B018
:107B9000A8030020400D0300004000B8002000B4FE
:107BA000026838B504461046FFF7C0FD08B900204A
:107BB00038BD9368990707D4936823F0004323F0F6
:107BC000170343F010039360FCF71AF80546236887
:107BD0009B685B07EBD5FCF713F8401B0228F6D92E
:107BE00023689B685A07F2D5A36D43F01003A36581
:107BF000E36D43F00103E3650120D9E773B500238A
:107C0000026801939368DD07044602D5002002B0A4
:107C100070BD9168214B194209D0A36D43F0100348
:107C2000A365E36D43F00103E3650120EFE793688B
:107C300023F0004323F0170343F001039360184B34
:107C4000D3F8083718021CD4637E012BDED0FBF773
:107C5000D7FF144E054622681368DB07D6D4936815
:107C6000D9075FBF9368334043F001039360FBF78C
:107C7000C7FF401B0228EED923681B68DA07EAD445
:107C8000CBE7094B094A1B68B3FBF2F301330193BD
:107C9000019B002BD8D0019B013BF8E71700008027
:107CA00000200140E8FFFF7FA8030020400D0300F3
:107CB00038B504460068FFF739FD054620BB94F847
:107CC0005430012B20D0012384F854302046FFF794
:107CD00095FFB0B9A36D226823F4706323F001030C
:107CE00043F48073A3651C23E065136084F854009B
:107CF000936823F0004323F0170343F004039360D9
:107D000038BD84F85450FBE70220F9E7026838B523
:107D1000936891680446C80701D4002038BD9907CC
:107D2000FBD4936803F00503012B19D1936823F06A
:107D3000004323F0170343F002039360032313600F
:107D4000FBF75EFF054623689B68DB07E5D5FBF77D
:107D500057FF401B0228F6D923689B68DA07F2D543
:107D6000A36D43F01003A365E36D43F00103E365E6
:107D70000120D3E770B5044600284BD0836D43F053
:107D800002038365FFF70CFF054668B92046FFF73D
:107D9000BDFF054608B90123A3652268936823F057
:107DA000104323F01703936023685A6822F4677224
:107DB00022F003025A6040F29F321A60D968164AD4
:107DC0000A40DA601A6922F040421A615A6922F0C8
:107DD00007025A611A6A02F0F0221A625A6A02F025
:107DE000F0225A62DA6A02F0F022DA629A6A0B4AE8
:107DF00000269E62D2F8083723F0FE73C2F80837D7
:107E00002046FAF71BFEE6652666A66584F85460F0
:107E1000284670BD0125FBE700023E83002001409B
:107E200010B590F85430012B044615D0012380F88A
:107E30005430FFF7B5FE58B92046FFF767FF38B951
:107E4000A36D23F4807323F0010343F00103A365C2
:107E5000002384F8543010BD0220FCE7F7B500235E
:107E6000019390F85430012B04467FD0012380F811
:107E70005430FFF74BFF23689A6812F00102054661
:107E800007D0A36D43F01003A365002384F854309A
:107E90002DE0A16D364F21F4817141F00201A16501
:107EA000DE68D96826F4FF4626F07C0621F40041FE
:107EB000360421F00301360CD96008209968394056
:107EC00041F0004199609968002913DA0199013164
:107ED00001910199B1F52E3FF5D3A36D23F0120363
:107EE00043F01003A365002384F85430012528468D
:107EF00003B0F0BDD3F8B410013801F07F010A449B
:107F0000DCD199681A48014041F001019960D3F829
:107F1000B41021F07F0141EAD202C3F8B4209A687C
:107F2000024042F002029A60FBF76AFE07462368AD
:107F30009A68D20708D4DA683243DA60A36D23F076
:107F4000030343F001039FE7FBF75AFEC01B02281F
:107F5000EDD923689B68D907E9D5A36D43F01003D9
:107F6000A365E36D43F00103E365BFE70225BEE7C8
:107F7000E8FFFF7F0749CA6822F4E06203021204A7
:107F800003F4E063120C134343F0BF6343F4003384
:107F9000CB60704700ED00E0164B30B5DC68C4F3F1
:107FA0000224C4F10703251D042B28BF0423062D3A
:107FB0004FF0FF358CBF033C002405FA03F321EAA0
:107FC0000303A54022EA0502A340002843EA020376
:107FD000ACBF00F16040084A4FEA0313B8BF00F09D
:107FE0000F00DBB2AABF00F56140135480F80033E4
:107FF00030BD00BF00ED00E014ED00E0002807DB1D
:10800000044A4109012300F01F00834042F8213057
:10801000704700BF00E100E000280CDB430906497F
:1080200000F01F0020330122824041F82320BFF3DB
:108030004F8FBFF36F8F704700E100E070B5D0E95C
:1080400013456560446D14B1D0E916456560D0E90B
:10805000105404F01C060124B4406C600468636092
:108060008368102B0BBFA260A160E160E26070BD6D
:108070000268416CD3B210B5083B1424B3FBF4F38F
:108080000B4CA24288BF0B4A21F0030199BF01F1BA
:10809000804202F50232521807338264064AC264F3
:1080A00003F01F03012202FA03F3036510BD00BFB2
:1080B000070402401C0802408008024038B500282E
:1080C0005CD002682E4B9A424FF014014AD82D4BD7
:1080D0001344B3FBF1F32C499B00C0E910130223B6
:1080E00080F825301368056923F4FF4323F07003FB
:1080F0001360D0E9024323432B43456911682B43A6
:1081000085692B43C5692B43056A2B430B431360D9
:10811000FFF7AEFFB4F5804F04BF00234360436810
:10812000816C03F07F020A60D0E91314013B032B3A
:108130004C601ED8154B1649816513449B000121E4
:10814000013A01FA02F200214365C2651960114B40
:108150005A6400230122C36380F8243080F825206C
:10816000184638BD0C4B1344B3FBF1F30B499B008D
:10817000B3E70023C0E91533C365EAE70120F0E760
:1081800007040240F8FFFDBF000002403F820010DC
:108190004009024000090240F8FBFDBF0004024014
:1081A00038B5002841D00268136823F0010313603A
:1081B0001F4B9A424FF0140130D81E4B1344B3FBAF
:1081C000F1F31D499B00C0E91013012403F01C03C7
:1081D00004FA03F3002515604B60FFF749FF836C39
:1081E00041681D60D0E913325A604A1E032A06D83E
:1081F000124B0B449B0094401D60114B5C640023A8
:10820000C363C0E91533C0E90B33C0E90D33C3655F
:1082100080F8253080F82430184638BD094B1344C7
:10822000B3FBF1F308499B00CDE70120F5E700BF60
:1082300007040240F8FFFDBF000002403F8200102B
:1082400000090240F8FBFDBF0004024070B590F841
:108250002450012D04463BD090F825600125AE4204
:1082600080F824504FF000062CD1022580F82550CC
:108270000568C6632E6826F001062E60FFF7DEFE55
:10828000036BBBB12B6843F00E032B60A36C1A6821
:10829000D20342BF1A6842F480721A60636D1BB148
:1082A0001A6842F480721A602B6843F001032B6055
:1082B000002070BD2B6823F004032B602B6843F073
:1082C0000A03E2E78023C36380F824602846F0E7CE
:1082D0000220EEE7034640B190F82520022A06D09E
:1082E0000422C263002280F8242001207047026823
:1082F000806C116821F00E011160016821F4807119
:108300000160116821F001011160D3E9100202F04F
:108310001C0101228A404260D3E9132151605A6D49
:1083200032B1116821F480711160D3E916215160D6
:108330000122002083F8252083F82400704708B527
:1083400090F82530022B03D00423C363012008BD1D
:1083500003681A6822F00E021A601A6822F00102FD
:108360001A60826C136823F480731360D0E91013D1
:1083700003F01C02012393404B60D0E913325A6092
:10838000436D33B11A6822F480721A60D0E9163254
:108390005A60012380F82530002380F82430836B55
:1083A00003B198470020D2E770B4426C046C0368B4
:1083B00026681D6802F01C020421914031420FD052
:1083C00015F0040F0CD01A6892065EBF1A6822F0EE
:1083D00004021A60036B6160002B33D070BC184735
:1083E00002219140314217D015F0020F14D01A68C3
:1083F000940606D41A6822F00A021A60012280F854
:108400002520114A93428CBF104B114B5960002319
:1084100080F82430C36ADFE708219140314211D04F
:1084200029070FD5196821F00E011960012303FAFD
:1084300002F26260C36380F82530002380F82430A4
:10844000436BC9E770BC70478000024000040240E3
:10845000000002400A4A536943F4802330B5536157
:10846000EFF3108472B60023CD58C5500433B3F532
:10847000807FF9D11369DB03FCD484F3108830BD0D
:1084800000400058064B5A69002ABFBF054A9A604F
:1084900002F188329A60BABF5869C00F0020704755
:1084A0000040005823016745044B5A6942F00042DE
:1084B0005A615869C043C00F704700BF0040005860
:1084C00070B50546FBF79CFB124E04463369D90391
:1084D00013D43369DA0744BF012232614CF2FA3215
:1084E000134011D10B4E306910F480200BD0FBF7F4
:1084F00087FB001BA842F6D304E0FBF781FB001BBF
:10850000A842E3D3032070BD024A1361024A01204E
:108510005360F8E700400058842100202DE9F04125
:10852000184D98462B78012B06460C46174626D048
:1085300001232B704FF47A7000236B60FFF7C0FFAC
:10854000A0B9012E16D1104A536943F001035361BB
:108550002760BFF36F8FC4F804804FF47A70FFF781
:10856000AFFF094A536923EA0603536100232B70C6
:10857000BDE8F08139462046FFF76CFFEDE70220A9
:10858000F6E700BF8421002000400058054A5369E7
:1085900023F47E7343EAC00040F4803040F00200D0
:1085A00050617047004000582DE9F041234F3B785F
:1085B000012B054688463FD001233B704FF47A706B
:1085C00000237B60FFF77CFF044688B92B68042BEF
:1085D00013D11B4A536943F4803343F004035361BE
:1085E0004FF47A70FFF76CFF0446154B1A681B684E
:1085F00000233B702046BDE8F0814FF0FF33C8F800
:1086000000306E68D5E901321344B3420AD93046CE
:10861000FFF7BCFF4FF47A70FFF752FF50B1C8F874
:1086200000600446064A536923F47E7323F0020374
:108630005361DAE70136E5E70224DBE78421002015
:10864000004000582DE9F04F524C00234FF00F0925
:108650000A6832FA03F501D1BDE8F08F012505FA69
:1086600003F818EA020200F08E804E68032706F035
:1086700003054FEA430E07FA0EFC6F1E012F6FEA47
:108680000C0C32D8876807EA0C0ACF6807FA0EF795
:1086900047EA0A078760476827EA0808C6F3001711
:1086A0009F4047EA08074760C76807EA0C088F68D9
:1086B00007FA0EF747EA0807022DC76017D14FEAFD
:1086C000D30800EB880803F0070AD8F820704FEAB7
:1086D0008A0A09FA0AFB27EA0B0B0F6907FA0AF75D
:1086E00047EA0B07C8F8207001E0032DDCD10768CA
:1086F00005FA0EF507EA0C073D4316F4403F056006
:1087000041D023F0030707F1804707F5803703F0D6
:10871000030CBD684FEA8C0C4FF0070E0EFA0CFEEE
:10872000B0F1904F25EA0E0E2FD01B4DA8422ED04F
:1087300005F58065A84214BF0725022505FA0CF54A
:1087400045EA0E05BD602568D74316F4801F0CBFAF
:108750003D4015432560656816F4001F0CBF3D4081
:1087600015436560D4F8805016F4803F0CBF3D403F
:108770001543C4F88050D4F88450B60354BF3D402C
:108780001543C4F88450013362E70025D6E701257C
:10879000D4E700BF0008005800040048374A2DE91C
:1087A000F04F00234FF0010A4FF0070B4FF00F0975
:1087B00031FA03F401D1BDE8F08F0AFA03FC1CEA98
:1087C000010654D023F0030404F1804404F58034FE
:1087D00003F00307A568BF000BFA07F8B0F1904F4C
:1087E00008EA050E45D0264DA84244D005F580651F
:1087F000A8420CBF02250725BD40754517D1D2F808
:10880000805025EA0605C2F88050D2F8845025EA47
:108810000605C2F88450156825EA060515605568F6
:1088200025EA06055560A56825EA0805A5600568DE
:1088300003265C0006FA04F423FA06F6254300EB4F
:108840008606056003F00705376AAD0009FA05F5ED
:1088500027EA05073762856825EA040585604568CB
:1088600025EA0C054560C56825EA0404C4600133A7
:108870009EE70025C0E70125BEE700BF00080058BD
:10888000000400480369194214BF0120002070470A
:108890000AB18161704781627047436901EA03024E
:1088A00021EA030141EA024181617047044AD1682B
:1088B000014208B502D0D060FDF7D6FC08BD00BF6C
:1088C00000080058024A136843F48073136070472D
:1088D000000400580D4B10B55B690C4628B99A0589
:1088E00007D500F027F820B110BD9B0501D400F09A
:1088F00019F8074A1369012C23F00403136101D10D
:1089000030BFF1E740BF20BF20BFEDE700040058B3
:1089100000ED00E0024B186800F4C060704700BF33
:1089200000040058024A136843F480431360704700
:10893000000400580C4A136823F4804313600B4B67
:108940001B6832214B430A49B3FBF1F35169890596
:1089500000D533B9536913F4007F14BF03200020FE
:108960007047013BF2E700BF00040058A803002055
:1089700040420F000B4A136823F0070343F0020341
:108980001360094B1A69012842F004021A6105D1EB
:1089900030BF1A6922F004021A61704740BF20BF3D
:1089A00020BFF6E70004005800ED00E04FF0B043B0
:1089B0001868C0F3404070474FF0B0431868C0F3E8
:1089C000400070474FF0B042536823F47F4343EABE
:1089D0000023536070474FF0B0431868C0F3406005
:1089E000704700007FB54FF0B0432C4AD3F80831F0
:1089F000C0F3031003F00F0352F82040284A52F846
:108A00002330B4FBF3F4FFF785FF264B054693E8CC
:108A10000700B5F5007F04AB03E9070010D0224B37
:108A20009C4218D303F5B70303F67F539C4229D920
:108A300003F5741303F510639C4225D802230BE061
:108A40001A4B9C4207D91A4B9C421BD903F537039A
:108A500003F5D853F0E7002304AA02EB830353F88D
:108A60000C4C144D2B6823F0070323432B60FBF7BA
:108A7000C7F806462B6803F007039C4206D1002086
:108A800004B070BD0123E7E70024EAE7FBF7B8F87C
:108A9000801B0228EED90320F2E700BF20700308F4
:108AA00080700308601B0308C0CF6A00BFEA210181
:108AB0003F933402004000584FF0B04310B59A681D
:108AC000D96812F00C0205D00C2A4AD101F0030338
:108AD000012B51D14FF0B0412B480B6813F0080324
:108AE00006D00B6813F0080337D1D1F8941007E0D3
:108AF0000C68240756BFD1F894300968C3F30323E8
:108B000050F82330002A0CBF184600204FF0B04127
:108B10008A6802F00C020C2A1ED1CA6802F0030215
:108B2000022A2ED0032A06D10B68184A13F4801F9C
:108B3000174B18BF13464FF0B042D068D168D268C7
:108B4000C0F306205843C1F302130133B0FBF3F026
:108B5000530F0133B0FBF3F010BD0B68C3F30313E5
:108B6000CEE7042A05D0082A06D11B6813F4801327
:108B700005D006480023C9E700231846C6E7044885
:108B8000C4E7024BD7E700BF207003080024F400BD
:108B90000048E80108B5FFF78FFF4FF0B043044AE3
:108BA0009B68C3F3031352F82330B0FBF3F008BD06
:108BB000807003082DE9F0410446002853D04FF09F
:108BC000B0439D68DE6803689B0605F00C0506F05F
:108BD000030668D5026A1DB10C2D46D1012E44D181
:108BE000002A40D04FF0B043A16A1A68170756BF59
:108BF000D3F894301B681B0903F0F00399421FD986
:108C00000846FFF7EFFE00282DD14FF0B042136861
:108C100043F0080313601368A16A23F0F0030B43C9
:108C20001360606AFFF7CEFEFFF7B4FFAB4B18602E
:108C3000AB4B1868FAF7E2FF002834D0BDE8F081AA
:108C40004FF0B042136843F008031360136823F039
:108C5000F0030B431360606AFFF7B4FE0846FFF7AA
:108C6000C1FE0028E0D00120E8E74FF0B043002A21
:108C700054D01A6842F001021A60FAF7C1FF0746A1
:108C8000FFF79AFE002842D04FF0B042136843F03D
:108C9000080313601368A16A23F0F0030B43136009
:108CA000606AFFF78FFE2368D80748D423689907C6
:108CB00000F18C8023681E0740F1FA80A3694FF011
:108CC000B046002B00F0E180D6F89430E16903F063
:108CD0001002914200F0C48003F00302022AC2D0C5
:108CE000D80740F1B380D6F8943023F00103C6F8DA
:108CF0009430FAF785FF0746D6F89430990740F18B
:108D0000A580FAF77DFFC31B112BF5D904E0FAF714
:108D100077FFC01B0228B3D903208FE71A6822F01F
:108D200001021A60FAF76CFF0746FFF745FE0028BC
:108D3000B9D0FAF765FFC01B0228F6D9ECE7082D79
:108D400003D00C2D05D1032E03D16368002BADD1C8
:108D500089E74FF0B043A1681A6822F480120A43F1
:108D60001A606268B2F5803F10D11A6842F480320E
:108D70001A60FAF745FF0746FFF718FE002895D15D
:108D8000FAF73EFFC01B6428F6D9C5E7B2F5041F09
:108D900004D11A6842F400121A60E6E7196821F457
:108DA00080311960196821F400111960002AE0D19E
:108DB000FAF726FF0746FFF7F9FD00283FF476AFE4
:108DC000FAF71EFFC01B6428F5D9A5E7042D236917
:108DD00003D00C2D0ED1022E0CD1002B3FF443AF4B
:108DE0004FF0B0426169536823F0FE4343EA0163E8
:108DF00053605FE74FF0B046BBB1336843F4807314
:108E00003360FAF7FDFE074633685A0505D4FAF7D2
:108E1000F7FEC31B022BF7D97EE77368626923F064
:108E2000FE4343EA0263736044E7336823F48073CC
:108E30003360FAF7E5FE074633685B057FF53AAF26
:108E4000FAF7DEFEC31B022BF6D965E74FF0B042FE
:108E5000E169D2F8943023F010030B43C2F8943048
:108E60004FF0B047D7F8943043F00103C7F894307F
:108E7000FAF7C6FE0646D7F894309A0718D4FAF7E0
:108E8000BFFE831B112BF6D946E7D6F8943023F0AA
:108E90000103C6F89430FAF7B3FE0746D6F89430CB
:108EA0009B0705D5FAF7ACFEC31B112BF6D933E7A8
:108EB0002368580754D50B4F3B68D90514D4FFF7E6
:108EC00001FDFAF79DFE06463B68DA050CD4FAF779
:108ED00097FE831B022BF7D91EE700BFA8030020D3
:108EE000AC03002000040058E3684FF0B046002BAC
:108EF00058D023F08003052B02BFD6F8903043F002
:108F00000403C6F890304FF0B046FAF779FED6F871
:108F1000903043F001030746C6F8903041F288389C
:108F2000D6F890309B0705D4FAF76AFEC31B434579
:108F3000F6D9F1E6E36823F00403812B1BD1FAF79D
:108F40005FFED6F8903043F08003C6F890300746B5
:108F50004FF0B04641F28838D6F89030180504D565
:108F6000E36A002B4AD1002068E6FAF749FEC01BED
:108F70004045F1D9D0E6FAF743FED6F8903023F019
:108F80008003C6F8903007464FF0B04641F288386B
:108F9000D6F890301905E3D5FAF732FEC01B4045EC
:108FA000F6D9B9E6FAF72CFED6F8903023F0800314
:108FB0000746C6F8903041F28838D6F890301A0546
:108FC00016D4FAF71DFED6F8903023F00103C6F848
:108FD000903007464FF0B04841F28836D8F89030CC
:108FE0009B07BDD5FAF70CFEC31BB342F6D993E637
:108FF000FAF706FEC01B4045DFD98DE60C2D4ED09A
:10900000022B4FF0B0431A6822F080721A6033D1FD
:10901000FAF7F6FD0546FFF7DEFC38BBD4E90C3164
:109020004FF0B0420B43D0682D4901400B43E16B38
:109030000B43216C0B43616C0B43A16B43EA01238F
:10904000D360136843F080731360D36843F0805398
:10905000D360FAF7D5FD0446FFF7BDFC002882D1A6
:10906000FAF7CEFD001B0A28F6D955E6FAF7C8FD37
:10907000401B0A28CFD94FE6FAF7C2FD0446FFF796
:10908000AAFC30B94FF0B042164BD1680B40D36008
:1090900069E7FAF7B5FD001B0A28F0D93CE6012B79
:1090A0003FF4E1AD4FF0B043D868236B00F003020A
:1090B0009A427FF4D8AD626B00F0700393427FF464
:1090C000D2ADA26B00F4FE43B3EB022F7FF4CBAD25
:1090D000636C00F06040C01A18BF0120AEE500BF0D
:1090E0008C80C111FCFFFEEE2DE9F0410D460446D7
:1090F00010B90120BDE8F081684E336803F0070322
:109100008B4216D323689A0727D54FF0B047A26841
:10911000BB6823F0F0031343BB60FAF771FD06460A
:10912000BB68DB0319D4FAF76BFD831B022BF7D95D
:1091300011E0336823F007030B433360FAF760FD57
:109140000746336803F00703AB42DBD0FAF758FD5C
:10915000C01B0228F5D90320CCE72368580617D591
:109160004FF0B0476269D7F8083123F00F0343EAA4
:109170001213C7F80831FAF743FD0646D7F808314D
:10918000D90305D4FAF73CFD831B022BF6D9E2E79D
:1091900023685A0713D54FF0B047E268BB6823F441
:1091A000E0631343BB60FAF72BFD0646BB689B03E5
:1091B00005D4FAF725FD831B022BF7D9CBE72368EB
:1091C000180714D54FF0B0472269BB6823F46053E9
:1091D00043EAC203BB60FAF713FD0646BB685903B6
:1091E00005D4FAF70DFD831B022BF7D9B3E72368EB
:1091F000DA070FD4294C236803F00703AB4239D8B0
:10920000FFF7C8FC264B1860264BBDE8F0411868F4
:10921000FAF7F4BC6268022A1DD1FFF7C7FB0028E9
:109220003FF467AF4FF0B04641F28838B36823F09F
:1092300003031343B360FAF7E3FC0746B3686268BD
:1092400003F00C03B3EB820FD4D0FAF7D9FCC01BA8
:109250004045F3D97FE7032A02D1FFF7BCFBDEE7E5
:1092600012B9FFF7A9FBDAE74FF0B0431B685B05C3
:10927000D8D43EE7236823F007032B432360FAF793
:10928000BFFC0646236803F00703AB42B8D0FAF7E9
:10929000B7FC801B0228F5D95DE700BF00400058ED
:1092A000A8030020AC03002008B5FFF773FC4FF0C3
:1092B000B043044A9B68C3F3022352F82330D840DA
:1092C00008BD00BF6070030808B5FFF763FC4FF0EE
:1092D000B043044A9B68C3F3C22352F82330D840FA
:1092E00008BD00BF607003084FF0B043D3F8900092
:1092F000C0F3400070474FF0B0410209D1F8883008
:1093000002F47F22000123EA020300F47F200343DA
:10931000C1F8883070474FF0B041020CD1F8883066
:10932000120423EA020343EA0040C1F888007047B0
:109330000368DA0370B5044639D5FFF7C3FAFAF7C4
:109340005FFC614E05463368DB0532D54FF0B04314
:10935000616BD3F8902002F4407291421DD0D3F893
:109360009010D3F8902042F48032C3F89020D3F8C4
:10937000902021F4407022F480328D07C3F89020B1
:10938000C3F8900009D5FAF73BFC41F28836054650
:10939000FFF7AAFF012840F090804FF0B042616BC8
:1093A000D2F8903023F440730B43C2F8903000267B
:1093B00005E0FAF725FC401B0228C4D903262568DE
:1093C000E8070AD54FF0B0416268D1F8883023EA47
:1093D000124392B21343C1F88830A9070AD54FF05F
:1093E000B041A268D1F8883023EA124392B2134305
:1093F000C1F88830AA0609D54FF0B0422169D2F8E9
:10940000883023F440630B43C2F88830AB0502D5A3
:10941000206AFFF780FF680502D5606AFFF77BFFCF
:10942000290502D5A06AFFF776FF6A0602D56069B2
:10943000FFF761FF2B0602D5A069FFF75CFFE80587
:1094400002D5E069FFF757FFE90610D54FF0B042AB
:10945000E168D2F8883023F440730B43C2F88830B7
:10946000B1F5807F02BFD36843F08073D3602A04D4
:109470000ED54FF0B042216BD2F8883023F0404334
:109480000B43C2F8883019B9D36843F08073D360B6
:109490006B0410D54FF0B042E16AD2F8883023F067
:1094A00040530B43B1F1005FC2F8883003D1D36859
:1094B00043F48033D360304670BDFAF7A1FB401B04
:1094C000B0427FF665AF79E70004005830B590F8F8
:1094D0002C30012B02464FF0020022D0174B82F8AD
:1094E0002D00CA24012582F82C505C6253245C6252
:1094F000B1F5807F146B996914D121F48851996179
:10950000596C24F0010421F0004159641463DD65B5
:109510000A4BFF2159620020012382F82D3082F886
:109520002C0030BD21F408519961D96C24F002045B
:1095300021F00041D9641463D865E9E700280040B0
:1095400070B50B4E036B756D1D40EA07044603D5DD
:109550000123F365FAF7C9FDAB0704D50223F365D0
:10956000204600F0C9F9012384F82D3070BD00BFFA
:109570000028004038B50A4CE36823F02003E3607C
:10958000FAF73EFB0546E3689B0601D5002038BD8F
:10959000FAF736FB401BB0F57A7FF4D90320F6E7E3
:1095A00000280040F8B5114DEC6814F04004064660
:1095B0001AD1EB6843F08003EB60FAF721FB2346F6
:1095C0000746EC6814F0400401D1032B01D1184682
:1095D000F8BDFAF715FBC01BB0F57A7F234684BFB0
:1095E000032386F82D30ECE70023F0E70028004045
:1095F00038B50F4CE36823F08003E360A3699B0652
:10960000054606D4FFF7B6FF10B1032085F82D00FC
:1096100038BDA36923F02003A361FFF7ABFF10B1AE
:10962000032085F82D00A36943F02003A361EFE731
:109630000028004038B5044600284BD090F82D3063
:1096400003F0FF021BB980F82C20F9F7B3FD0223C9
:10965000214D84F82D30EB68DB0636D4CA236B62CB
:1096600053236B622046FFF79DFF10B1FF236B620F
:1096700038BDAB6923F08E6323F04003AB612169F1
:109680006368AA690B431343A2691343AB61D4E92E
:10969000022343EA02432B61D4E90931EA680B4310
:1096A00022F4F8521343EB602046FFF7A1FF002895
:1096B000DCD1D4E90713AA690B4322F060421343BB
:1096C00062691343AB61FF236B62012384F82D3081
:1096D0000020CDE70120CBE7002800400023092827
:1096E00003D840EA0310C0B270470A380133C0B251
:1096F000F5E700002DE9F04790F82C30012B0546E6
:109700004FF0020069D0012385F82C304E4B85F8CC
:109710002D00DE6806F44076B6F5807F78D04C697F
:10972000087891F8019091F802A091F82470002A2D
:1097300055D19B6913F0400308BFCB70FFF7CEFFF4
:1097400080464846FFF7CAFF02465046FFF7C6FF6D
:1097500081463846FFF7C2FF0B6ACF78234343EABE
:10976000875343EA090343EA084343EA022343EAEF
:109770000063354ACA205062532050628C6A88695F
:10978000B4F5807F946945D124F488549461012410
:10979000D465B6F5807F09BFCB6913640343536476
:1097A00018BF5064284B4A681A672A6B42F00102BE
:1097B0002A639A6942F488529A61244AD2F8803026
:1097C00043F40033C2F880301F4BFF225A6200205E
:1097D000012385F82D3085F82C00BDE8F087B4F121
:1097E000803F07D0B4F5000F04D09B6913F040030D
:1097F00008BFCB700B6ACA781C4344EA0A0444EAE7
:10980000004343EA092343EA825343EA0763B0E78C
:109810000023AEE724F4085494610224D465B6F51D
:10982000807F09BFCB6993640343D36418BFD064BE
:10983000054B4A685A672A6B42F002022A639A690A
:1098400042F40852B8E700BF002800400008005862
:1098500090F82C20012A03464FF0020012D00A4A49
:1098600083F82D00CA21516253215162916941F060
:1098700020019161FF2151620020012283F82D20F7
:1098800083F82C00704700BF0028004090F82C207F
:10989000012A03464FF0020019D00D4A83F82D002B
:1098A000CA2151625321516291690A4841F08001F5
:1098B0009161D0F8801041F48021C0F88010FF2120
:1098C00051620020012283F82D2083F82C0070477C
:1098D0000028004000080058064B5A6D520610B58B
:1098E000044603D54022DA65FAF702FC012384F826
:1098F0002D3010BD002800407047890001F18041E3
:1099000001F531410A607047890001F1804101F59C
:1099100031410868704700002DE9F3471F4689462A
:1099200090460446FAF76CF90A9D3D442D1AFAF761
:1099300067F9264B1E68C6F3CB366E438246019606
:109940002268936839EA03030CBF012300234345CF
:1099500001D100202EE07B1CF3D0FAF751F9A0EBE7
:109960000A00A84229D323685A6822F0E0025A600C
:109970006268B2F5827F0AD1A268B2F5004F02D0C8
:10998000B2F5806F03D11A6822F040021A60A26A11
:10999000B2F5005F07D11A6822F400521A601A6803
:1099A00042F400521A60012384F85D30002384F8E9
:1099B0005C30032002B0BDE8F087019A019B002AC9
:1099C00003F1FF33019308BF1546B9E7A803002050
:1099D0002DE9F74F994600238DF803300446884659
:1099E0001746FAF70DF90C9D4D442D1AFAF708F9B0
:1099F0002C4BD4F800B01E6823235E43360D6E4313
:109A0000824601962268936803EA0803BB4201D1AB
:109A100000203AE0B8F5C06F07D137B99BF80C3099
:109A2000DBB28DF803309DF80330B9F1FF3FEAD087
:109A3000FAF7E6F8A0EB0A00A84229D323685A688F
:109A400022F0E0025A606268B2F5827F0AD1A26811
:109A5000B2F5004F02D0B2F5806F03D11A6822F040
:109A600040021A60A26AB2F5005F07D11A6822F4B8
:109A700000521A601A6842F400521A60012384F8F6
:109A80005D30002384F85C30032003B0BDE8F08F24
:109A9000019A019B002A03F1FF33019308BF154689
:109AA000B0E700BFA803002073B50B4600920D4637
:109AB00016464FF4C05100220446FFF789FF0246C4
:109AC00030B1236E43F020032366032002B070BD43
:109AD00000962B4680212046FFF71EFF02460028F5
:109AE000EFD100962B464FF4C0612046FFF770FF80
:109AF0000028EBD0E5E74368B3F5827FF7B504466D
:109B00000E4617460BD18368B3F5004F02D0B3F56C
:109B1000806F04D12268136823F04003136000971C
:109B20003346002280212046FFF7F6FE054628B185
:109B3000236E43F020032366032514E06368B3F526
:109B4000827F10D1A368B3F5004F02D0B3F5806FC8
:109B500009D10097334600224FF4C0612046FFF739
:109B600037FF0028E4D1284603B0F0BDF8B504461D
:109B700000287ED0436A002B50D14268B2F5827F24
:109B800000D0C36194F85D3003F0FF0223B984F87C
:109B90005C202046F9F774FB2268E068022384F811
:109BA0005D301368B0F5E06F23F0400313604FF0B1
:109BB000000337D91D46B0F5706F18BFA362A768C0
:109BC0006368A169A66A07F4044703F482733B4300
:109BD000276907F002073B43676907F001073B432A
:109BE00001F400773B43E76907F038073B43276AF6
:109BF00007F080073B4306F400573B43B6F5005F90
:109C0000136014D1236B8BBBB0F5E06F0DD9022329
:109C10002363136843F40063136008E00023C0E982
:109C20000433AFE74FF48055C7E701232363636A2A
:109C3000676B03F0100307F0080700F470603B4304
:109C4000090C034301F004010B432B43B6F5005FFD
:109C5000536004BFA38D1361D36923F40063D36100
:109C600000200123206684F85D30F8BD022BDED190
:109C7000CFE70120F9E7000070B5044690F85C00DA
:109C8000012800F0CF80012084F85C0094F85D008A
:109C900066680128C5B20AD0B6F5827F40F0C08060
:109CA000A068002840F0BC80042D40F0B980002955
:109CB00051D0002A4FD0002B4DD094F85D00A16305
:109CC00004281CBF052084F85D0000202066C4E93C
:109CD0001300A06AE387B0F5005F2168A3872264C0
:109CE000A4F84430A4F8463007D1086820F40050A6
:109CF0000860086840F400500860486820F4C040DC
:109D00004860E068B0F5E06FA06D29D94B6823F496
:109D100080534B6094F85D30434E444D042B444BCC
:109D200018BF1D46434B18BF3346C0E90B35424BA5
:109D3000436300238363B4F846300C319BB2FEF7D3
:109D400085FA0346002848D0236E43F010032366AB
:109D5000012384F85D300120002384F85C3070BD5D
:109D60004D6845F480554D60656DAD69B5F5806F02
:109D70000AD113F0010F4B681ED123F480434B60CE
:109D8000E38FC3F34E03E3878369B3F5806FC1D1DB
:109D90004B6823F480534B60B4F8463013F0010F46
:109DA0004B6811D123F400534B60B4F84630C3F331
:109DB0004E03A4F84630ADE743F480434B60E38F95
:109DC000C3F34E030133DEE743F400534B60B4F8B2
:109DD0004630C3F34E030133EBE72268606D5168F0
:109DE00041F001015160C0E90B33C0E90D33E38F4D
:109DF000A16B9BB20C32FEF729FA0028A4D123688C
:109E00001A6852065EBF1A6842F040021A605A6829
:109E100042F020025A605A6842F002025A609BE700
:109E2000022099E702209AE7719F0008419E0008EE
:109E30004D9E00087B9E0008599E000870477047A1
:109E400008B5806AFFF7FBFF08BD704708B5806A58
:109E5000FFF7FBFF08BD7047806A026808B55368CA
:109E600023F003035360036E43F0100303660123E2
:109E700080F85D30FFF7EFFF08BD7FB50646002391
:109E80000393846A8DF80B30F9F7BAFE33681B68C8
:109E90009A06054668D42268536823F0200353606D
:109EA000A36AB3F5005F13D1012200906423114629
:109EB0002046FFF731FD18B1236E43F002032366FD
:109EC000E3682668B3F5E06F2ED9F3680393039B2C
:109ED000A2682368002A43D16268B2F5827F3FD12D
:109EE0005A6822F003025A6064212A462046FFF78E
:109EF00002FE08B1202323660023A4F8463022681E
:109F0000012384F85D309368DB0606D5236E43F0A9
:109F1000020323664FF6EF739360236E23B320464C
:109F2000FFF799FF04B070BD337BDBB28DF80B30C7
:109F30009DF80B30236B022BCAD1012200956423BC
:109F400011462046FFF7E8FC18B1236E43F00203E8
:109F50002366337BDBB28DF80B309DF80B30B7E70F
:109F60005A6822F00102BEE72046FFF767FFD9E7F3
:109F70007FB5064600230393846A8DF80B30F9F70A
:109F80003FFE33681B68990605465ED42268536815
:109F900023F020035360A36AB3F5005F1BD1E3688D
:109FA000B3F5E06F3ED1236B012B3BD100906423CE
:109FB0004FF400724FF4C0612046FFF709FD18B15D
:109FC000236E43F00203236623681B7BDBB28DF80C
:109FD0000B309DF80B302A4664212046FFF764FDC4
:109FE00018B1236E43F02003236623685A6822F0D9
:109FF00003025A600022E287A4F84620012284F876
:10A000005D209A68D20606D5226E42F002022266D0
:10A010004FF6EF729A60236EBBB12046FFF71BFF2D
:10A0200004B070BD009564234FF480624FF4C061AA
:10A030002046FFF7CDFC18B1236E43F002032366E0
:10A040002368DB680393039BC5E72046F8F734FCDD
:10A05000E6E70000036830B559689A6802F04105E8
:10A06000012D85B0044606D14D0604D5C36C05B05C
:10A07000BDE830401847950704D5080602D5236D82
:10A080002046F4E712F4B07F59D08D0657D550061C
:10A090000FD594F85D0003284FF0000549D0206EDD
:10A0A00040F0040020660095D86800909868009001
:10A0B000009895060CD5206E40F001002066002027
:10A0C000029098680290186820F04000186002988A
:10A0D000D00508D5226E42F00802226600220392C3
:10A0E0009A680392039A226E4AB35A6822F0E002F9
:10A0F0005A60012284F85D208A0722D05A68A06D38
:10A1000022F003025A6040B1104B8363FEF717F947
:10A1100018B1236E43F040032366606D78B10B4B9A
:10A120008363FEF70CF950B1236E43F040032366BE
:10A1300005E00195DA6801929B680193019B05B0E7
:10A1400030BD2046FFF787FEF9E700BF51A10008A8
:10A1500008B5806A0023A0F84630C387FFF77BFE6E
:10A1600008BD0000034AD2F8903043F40043C2F81F
:10A170009030704700040058034AD2F8903023F41E
:10A180000043C2F89030704700040058074B1A682B
:10A1900022F040021A6040F441704FF4B852186047
:10A1A0005A601A6842F040021A6070470000015875
:10A1B00037B5054600284ED0837903F0FF046BB114
:10A1C000032C0BD0254B4FF400629A612868FFF7EF
:10A1D000DDFF002401232B71AC602FE000236B71A5
:10A1E0002846F9F721FC1E4AD2F8903043F48053F8
:10A1F000C2F89030002CE5D102234FF0B042AB7191
:10A20000D2F8943023F40043C2F89430154B1B6805
:10A210001C214B43DB0C64214B430193019B93B9FD
:10A220000124AC60FFF79EFF0C4B9A6842F4006279
:10A230009A604FF400629A61002CC7D00123AB7181
:10A24000204603B030BD019B013B0193D2F894300E
:10A250005B04E3D4E6E70124F2E700BF0004005802
:10A2600000080058A803002037B5174D2B68024698
:10A270001C204343DB0C6420434314480193019B9F
:10A2800093B901209060114C21732B681C214B4322
:10A29000DB0C64214B430193019B6BB9012090605F
:10A2A0000A4BDB6803B030BD019B013B019383681F
:10A2B0009C07E4D50020E6E7019B013B0193A368DE
:10A2C000DB07E9D5ECE700BFA80300200000015838
:10A2D00037B5184D2B6802461C204343DB0C642025
:10A2E000434315480193019BA3B901209060124C90
:10A2F000FF2323732B681C256B43DB0C64256B4306
:10A300000193019B73B9012090600B4BDB680B70CC
:10A3100003B030BD019B013B019383689C07E2D5EC
:10A320000020E4E7019B013B0193A368DB07E8D52C
:10A33000EBE700BFA8030020000001580E4B0F49B7
:10A340001B681822534382B01B0D642253430193B0
:10A350004B69019AC3F3800322B902238360012071
:10A3600002B07047019A013A01924A69920701D5F9
:10A37000002BEDD10020F3E7A803002000040058D3
:10A3800007B50379012B0FD10A4B1B6818225343E1
:10A390001B0C0193FFF7F0FE019B013B0193019B16
:10A3A000002BF9D1FFF7DEFE03B05DF804EBFFF7F9
:10A3B000C5BF00BFA8030020F8B51E468379012B56
:10A3C000154604460F46DAB22DD14379012B2AD027
:10A3D000022342718371FFF7D3FF0D212046FFF75F
:10A3E000CBFEFFF741FF390A2046FFF73DFFF9B2E8
:10A3F0002046FFF739FF2E44B5420ED12046FFF725
:10A40000B1FEFFF79BFFA06801230038A3714FF056
:10A41000000318BF01206371F8BD15F8011B204629
:10A42000FFF722FFE8E70220F6E7F8B51E4683793A
:10A43000012B154604460F46DAB22FD14379012B82
:10A440002CD04271FFF79CFF1D212046FFF794FEA0
:10A45000FFF70AFF390A2046FFF706FFF9B2204648
:10A46000FFF702FF00212046FFF7FEFE2E44B54213
:10A470000ED12046FFF776FEFFF760FFA0680123AC
:10A480000038A3714FF0000318BF01206371F8BDBD
:10A4900029462046FFF71CFF0135E8E70220F6E7D2
:10A4A000F8B51F468379012B154604460E46DAB2ED
:10A4B0002CD14379012B29D04271FFF761FF06F0BF
:10A4C000EF03A3F1840253425341237131462046E6
:10A4D000FFF752FEFFF7C8FE2F44AF4210D1FFF73F
:10A4E00041FE842E02D02046FFF728FFA0680123FA
:10A4F0000038A3714FF0000318BF01206371F8BD4D
:10A5000015F8011B2046FFF7AFFEE6E70220F6E74D
:10A51000F8B51E468379012B154604460F46DAB27C
:10A5200027D14379012B24D04271FFF729FF394607
:10A530002046FFF721FEFFF797FE00212046FFF798
:10A5400093FE2E44B5420ED12046FFF70BFEFFF7D7
:10A55000F5FEA06801230038A3714FF0000318BF77
:10A5600001206371F8BD29462046FFF7B1FE013591
:10A57000E8E70220F6E737B50023ADF8043001AA7A
:10A58000022312210546FFF7C3FFBDF80440022352
:10A5900064BA01AAA4B219462846FFF781FFE20770
:10A5A00002D528460AF01EF8A30702D528460AF06D
:10A5B0001FF8600702D528460AF044F8210702D5A3
:10A5C00028460AF045F8E20602D528460AF046F881
:10A5D000A30602D528460AF02FF8600602D52846C1
:10A5E0000AF00CF8210606D514F4807118BF012179
:10A5F00028460AF009F8A20502D528460AF014F800
:10A60000630402D528460AF02FF803B030BDF8B530
:10A610001E468379012B154604460F46DAB227D130
:10A620004379012B24D04271FFF7AAFE0E21204668
:10A63000FFF7A2FDFFF718FE39462046FFF714FE8C
:10A640002E44B5420ED12046FFF78CFDFFF776FE73
:10A65000A06801230038A3714FF0000318BF012048
:10A660006371F8BD15F8011B2046FFF7FDFDE8E713
:10A670000220F6E7F8B51E468379012B15460446FD
:10A680000F46DAB22BD14379012B28D04271FFF764
:10A6900077FE1E212046FFF76FFDFFF7E5FD3946E7
:10A6A0002046FFF7E1FD00212046FFF7DDFD2E44A7
:10A6B000B5420ED12046FFF755FDFFF73FFEA068DB
:10A6C00001230038A3714FF0000318BF012063710C
:10A6D000F8BD29462046FFF7FBFD0135E8E70220DB
:10A6E000F6E70000036A23F001030362036A70B512
:10A6F000446882690D6822F4803222F073022A4392
:10A700008D6823F002032B43124DA84206D0124E4F
:10A71000B04203D0A6F58066B04214D1CE6823F0D3
:10A7200008033343A84223F0040306D00B4DA8428C
:10A7300003D005F58065A84205D124F44075D1E920
:10A74000054634432C43446082614A684263036295
:10A7500070BD00BF002C0140004801400044014092
:10A76000036A23F480730362036A426870B5C469A4
:10A770000D6824F4803424F073042C438D6823F492
:10A78000007343EA05230F4DA8420ED1CD6823F490
:10A79000006343EA052323F48063D1E9055622F4DC
:10A7A0004052354342EA051206E0074DA842F4D074
:10A7B00005F58065A842F0D042604A68C461C26372
:10A7C000036270BD002C014000440140036A23F481
:10A7D00080530362026A30B54468C3690D6823F090
:10A7E000807323F4E64343EA05238D6822F4005284
:10A7F00042EA05320A4DA84207D005F5C055A842E5
:10A8000003D005F58065A84204D14D6924F4804445
:10A8100044EA85144460C3614B680364026230BD3E
:10A82000002C0140036A23F480330362026A30B5CE
:10A830004468436D0D6823F4803323F070032B4389
:10A840008D6822F4003242EA05420B4DA84207D03F
:10A8500005F5C055A84203D005F58065A84204D18E
:10A860004D6924F4803444EA0524446043654B6810
:10A870008365026230BD00BF002C0140036A23F4EF
:10A8800080130362026A30B54468436D0D6823F09B
:10A89000807323F4E04343EA05238D6822F4001219
:10A8A00042EA05520A4DA84207D005F5C055A84214
:10A8B00003D005F58065A84204D14D6924F48024B5
:10A8C00044EA8524446043654B68C365026230BD39
:10A8D000002C0140704710B5846A626A82420BD135
:10A8E00001232377D2690AB984F83E302046F9F76C
:10A8F0005FF80023237710BDA36A834208D10222A8
:10A900002277DB69002BF1D1012384F83F30EDE79A
:10A91000E36A834208D104222277DB69002BE5D168
:10A92000012384F84030E1E7236B8342DED1082223
:10A930002277DB69002BD9D1012384F84130D5E798
:10A94000704710B5846A636A834207D10123237775
:10A950002046FFF7F5FF0023237710BDA36A83424B
:10A9600001D10223F3E7E36A834201D10423EEE736
:10A97000236B8342ECD10823E9E7704710B5846A62
:10A98000636A834209D10123237784F83E3020464D
:10A99000FFF7F3FF0023237710BDA36A834205D19D
:10A9A00002232377012384F83F30F0E7E36A8342F0
:10A9B0004FF0010304D10422227784F84030E6E707
:10A9C000226B824203BF0822227784F8413084F848
:10A9D0003D30DCE71A4A0368904210B502D0B0F16E
:10A9E000804F09D14C6823F07003904243EA04037E
:10A9F00009D0B0F1804F06D0124A904203D002F540
:10AA00008062904203D1CA6823F4407313434A69B9
:10AA100023F08003134303608B68C3620B68836277
:10AA2000074B984207D003F5C053984203D003F573
:10AA30008063984201D10B6903630123436110BD18
:10AA4000002C01400044014010B5044650B390F87A
:10AA50003D3003F0FF021BB980F83C20F9F7A8F95C
:10AA60000223206884F83D30211DFFF7B3FF012346
:10AA700084F84830002084F83E3084F83F3084F871
:10AA8000403084F8413084F8423084F8433084F810
:10AA9000443084F8453084F8463084F8473084F8F0
:10AAA0003D3010BD0120FCE710B5044650B390F8CE
:10AAB0003D3003F0FF021BB980F83C20FFF70AFF8E
:10AAC0000223206884F83D30211DFFF783FF012316
:10AAD00084F84830002084F83E3084F83F3084F811
:10AAE000403084F8413084F8423084F8433084F8B0
:10AAF000443084F8453084F8463084F8473084F890
:10AB00003D3010BD0120FCE7036A23F0100303620F
:10AB1000036A426870B584690D6824F0807424F477
:10AB2000E64444EA05248D6823F0200343EA051334
:10AB30000F4DA8420ED1CD6823F0800343EA0513E0
:10AB400023F04003D1E9055622F44062354342EA3E
:10AB5000850206E0074DA842F4D005F58065A842BD
:10AB6000F0D042604A6884618263036270BD00BFB6
:10AB7000002C01400044014038B590F83C30012BD6
:10AB8000044673D001200C2A84F83C004ED008D82B
:10AB9000042A2BD0082A39D0BAB1002384F83C30DB
:10ABA00038BD102A52D0142AF7D12068FFF766FE6C
:10ABB000436D0A6943F400634365436D23F4806386
:10ABC0004365436D43EA02234EE02068FFF78AFDA8
:10ABD00083690A6943F008038361836923F00403EE
:10ABE00083618369134383610020D6E72068FFF700
:10ABF0008BFF83690A6943F400638361836923F4EB
:10AC000080638361836943EA0223ECE72068FFF7EE
:10AC1000A7FDC3690A6943F00803C361C36923F050
:10AC20000403C361C3691343C361DDE72068FFF711
:10AC3000CDFDC3690A6943F40063C361C36923F4AA
:10AC40008063C361C36943EA0223EDE72068FFF72D
:10AC5000E9FD436D0A6943F008034365436D23F042
:10AC600004034365436D13434365BDE7022097E743
:10AC700010B584680A4324F47F4442EA0322224345
:10AC8000826010BD38B590F83C30012B04464FF07F
:10AC9000020000F0958084F83D000122206884F8CD
:10ACA0003C208568474B2B4083600B68602B54D059
:10ACB00037D8402B6BD019D8202B0DD00AD833F0C1
:10ACC000100109D0012384F83D30002384F83C3082
:10ACD000104638BD302BF5D1826822F4401222F0A4
:10ACE00070021A4342F0070282602BE0502BE9D138
:10ACF0004A68CD68016A036A23F00103036283692D
:10AD000021F00A0123F0F00343EA05130A438361AB
:10AD10000262836823F4401323F0700343F0570367
:10AD20000FE0B3F5805F0DD0B3F5005F0CD0702B52
:10AD3000C8D1CB68D1E90121FFF79AFF836843F0BE
:10AD4000770383600022BDE7CB68D1E90121FFF7DB
:10AD50008FFF836843F48043F3E7036A4D68C96853
:10AD600023F0100303628269036A22F4704223F025
:10AD7000A00343EA051342EA013282610362836859
:10AD800023F4401323F0700343F06703D9E74A68C4
:10AD9000CD68016A036A23F001030362836921F02D
:10ADA0000A0123F0F00343EA05130A4383610262B8
:10ADB000836823F4401323F0700343F04703C0E794
:10ADC000024685E78800CEFF036A01F01F0110B537
:10ADD00001248C4023EA04030362036A8A401A4375
:10ADE000026210BD38B50D46082D044611461BD031
:10ADF00005D85DB1042D14D094F8430008E00C2D63
:10AE000015D0102DF8D190F8420001E090F83E00E6
:10AE1000A0F1020CDCF1000040EB0C0050B102206C
:10AE200076E090F83F00F3E790F84000F0E790F804
:10AE30004100EDE7082D1AD007D86DB1042D13D0CD
:10AE400094F84320012A19D00CE00C2D27D0102DA6
:10AE5000F6D194F842000CE094F83E20501E424295
:10AE600042415AB9012053E094F83F20F6E794F8A4
:10AE70004000421E504250410028F3D00029F1D03A
:10AE8000002BEFD0082D4FF0020256D00AD885B122
:10AE9000042D3ED0042D84F84320E3D13BE094F808
:10AEA0004100E6E70C2D5CD0102DF3D184F8422050
:10AEB000D8E7606A84F83E203A4AC2623A4A02639E
:10AEC0003A4A426322683432FDF7C0F90028C9D1FA
:10AED0002268D36843F400732068D36029460122B6
:10AEE000FFF772FF324A904250D0324B98424DD019
:10AEF00003F58063984249D0B0F1804F4DD182680C
:10AF00002D4B1340062B02D0B3F5803F45D10020D6
:10AF100038BD84F83F20A06A224AC262224A0263F6
:10AF2000224A426322683832FDF790F9002899D10D
:10AF30002268D36843F48063CEE7E06A84F8402057
:10AF4000184AC262184A0263184A426322683C32B5
:10AF5000FDF77CF9002885D12268D36843F40063AB
:10AF6000BAE7206B84F841200E4AC2620E4A02639F
:10AF70000E4A426322684032FDF768F900287FF4E8
:10AF800071AF2268D36843F48053A5E7436C9042C5
:10AF900043F400434364B2D0AEE7036843F00103D7
:10AFA0000360B4E7D7A8000843A900087DA90008FA
:10AFB000002C01400044014007000100FFF712BFD0
:10AFC000082938B504460D464FD004D861B104298C
:10AFD00044D0012038BD0C29FBD10268006BD36836
:10AFE00023F48053D36005E00268406AD36823F4F9
:10AFF0000073D360FDF7A3F9206800222946FFF70C
:10B00000E3FE2A4B984207D003F5C053984203D081
:10B0100003F5806398420DD1026A41F211131A427E
:10B0200008D1026A40F244431A4202BF436C23F43F
:10B0300000434364026A41F211131A4208D1026AC2
:10B0400040F244431A4202BF036823F00103036045
:10B0500001238DB984F83E300020BBE70268806A86
:10B06000D36823F48063D360C4E70268C06AD368FE
:10B0700023F40063D360BDE70C2D13D007D8042D53
:10B080000AD0082D0BD0012384F84330E4E7102DBB
:10B09000F9D184F84230DFE784F83F30DCE784F808
:10B0A0004030D9E784F84130D6E700BF002C01409A
:10B0B000FFF786BF70B590F83C30012B02464FF089
:10B0C000020020D082F83D000F4D1068436884686C
:10B0D000A84202BF4E6823F4700333430E6823F086
:10B0E00070033343A842436002D0B0F1804F04D1D3
:10B0F000896824F080030B4383600123002082F8D9
:10B100003D3082F83C0070BD002C0140026852E8DE
:10B11000003F23F0C00342E8003102680029F5D166
:10B1200002F1080353E8003F23F4000302F1080C86
:10B130004CE800310029F3D12023C0F88830704753
:10B1400010B5026852E8003F23F4907342E80031E2
:10B1500002680029F5D10F4C02F1080353E8003FC3
:10B16000234002F1080C4CE800310029F4D1C36EF1
:10B17000012B07D152E8003F23F0100342E80031D1
:10B180000029F7D12023C0F88C300023C366436721
:10B1900010BD00BFFEFFFFEFF8B504461346D4F81C
:10B1A0008850202D32D1F1B1EAB1E06FA4F85620D9
:10B1B000A4F8542000262122C4F890602165C4F828
:10B1C0008820226888B1124FC762124F0763124F5E
:10B1D0002832C0E90D76FDF739F830B11023C4F8F4
:10B1E0009030C4F888500120F8BD236840221A62CC
:10B1F000226802F1080353E8003F43F0800302F1A4
:10B20000080141E800300028F3D1EDE70220EBE728
:10B210001DB2000865B2000871B2000808B5034607
:10B22000806A1B681B6813F0200317D1A0F8563002
:10B23000026802F1080353E8003F23F0800308325C
:10B2400042E8003102680029F2D152E8003F43F0A1
:10B25000400342E800310029F7D108BDF9F77CF836
:10B26000FBE7704708B5806AFFF7FBFF08BD704732
:10B27000806A38B50468D0F88830D0F88C50A2685D
:10B28000120606D5212B04D10023A0F85630FFF773
:10B290003DFFA3685B0606D5222D04D10023A0F84C
:10B2A0005E30FFF74DFFD0F8903043F01003C0F848
:10B2B0009030FFF7DCFF38BD08B5806A0023A0F8A6
:10B2C0005E30A0F85630FFF7D2FF08BD704700008F
:10B2D0000368D9691A682DE9F04140F60F0631423A
:10B2E0009D68044610D18E0640F1978002F020063A
:10B2F00005F080573E4300F09080436F002B00F034
:10B300008580BDE8F0411847AB4EAC482E40104058
:10B31000304300F08280CF0709D5D00507D5012042
:10B320001862D4F8900040F00100C4F890008F0734
:10B3300009D5E80707D502201862D4F8900040F03C
:10B340000400C4F890004F0709D5E80707D504208A
:10B350001862D4F8900040F00200C4F890000F0783
:10B360000BD502F02000304307D008201862D4F833
:10B37000900040F00800C4F890000E050AD5500176
:10B3800008D54FF400601862D4F8903043F02003E1
:10B39000C4F89030D4F89030002B37D08B0609D504
:10B3A00002F0200205F080552A4303D0636F0BB1F1
:10B3B000204698472668D4F89020B36802F0280207
:10B3C00003F0400353EA0205204621D0FFF7B8FE00
:10B3D000B3685F0617D5226802F1080353E8003FFF
:10B3E00023F04003083242E800310029F3D1D4F8B9
:10B3F000800040B1724B8363FCF7A1FF30B1D4F8F9
:10B400008000836B7DE72046FFF731FFBDE8F081C8
:10B41000FFF72DFFC4F89050F8E7E06E012840F0E8
:10B420008980CE0640F18680D00640F183801022CC
:10B430001A629A6851064BD5D4F8802011684A6880
:10B4400092B2002AE2D0B4F85C009042DED9A4F8AF
:10B450005E200A6892062FD453E8002F22F48072EF
:10B4600043E800210029F7D103F1080252E8002F38
:10B4700022F0010203F1080040E800210029F3D185
:10B4800003F1080252E8002F22F0400203F1080005
:10B4900040E800210029F3D12022C4F88C20E16685
:10B4A00053E8002F22F0100243E800210029F7D1D1
:10B4B000D4F88000FCF70EFF02232367B4F85E3057
:10B4C000B4F85C10C91A89B22046FFF7FFFE9DE769
:10B4D000B4F85E20B4F85E00B4F85C1080B292B2AA
:10B4E000002893D0891A89B200298FD053E8002F01
:10B4F00022F4907243E800200028F7D1314D03F187
:10B50000080252E8002F2A4003F1080646E800200E
:10B510000028F4D12022C4F88C206067E06653E84C
:10B52000002F22F0100243E800200028F7D1022368
:10B530002367C9E7CF0209D56E0207D54FF4801201
:10B5400020461A62BDE8F04100F0A0BD08060BD508
:10B5500002F0800005F40005284305D0A36F002BFE
:10B560003FF454AF2046CCE64F0611D556060FD512
:10B5700053E8002F22F0400243E800210029F7D1D0
:10B580002023C4F88830A1672046F8F7E5FE3DE7A0
:10B590000D0206D5500004D52046BDE8F04100F06C
:10B5A00077BDCB017FF532AF002ABFF62FAF204623
:10B5B000BDE8F04100F06BBD010000102001000467
:10B5C000B9B20008FEFFFFEFD0F88C20B0F8601091
:10B5D000222A08B5036855D15B6A826D0B4013704F
:10B5E000836D01338365B0F85E30013B9BB2A0F8F8
:10B5F0005E30B0F85E309BB2002B42D1026852E858
:10B60000003F23F4907342E8003103680029F5D12C
:10B6100003F1080252E8002F22F0010203F1080CA6
:10B620004CE800210029F3D12022C0F88C20184AD0
:10B6300041679342016705D1C26E012A0ED0F8F727
:10B6400099FE1EE05A681102F6D553E8002F22F049
:10B65000806243E800210029F7D1EDE70022C266AD
:10B6600053E8002F22F0100243E800210029F7D10F
:10B67000DA69B0F85C10D20644BF10221A62FFF7F4
:10B6800025FE08BD9A6942F008029A61F9E700BFF9
:10B6900000800040D0F88C20B0F86010222A08B555
:10B6A000036852D15A6A1140826D22F8021B8265EA
:10B6B000B0F85E20013A92B2A0F85E20B0F85E20A9
:10B6C00092B2002A40D153E8002F22F4907243E84E
:10B6D00000210029F7D103F1080252E8002F22F0DF
:10B6E000010203F1080C4CE800210029F3D12022CB
:10B6F000C0F88C20174A41679342016705D1C26E9A
:10B70000012A0ED0F8F736FE1EE05A681102F6D56F
:10B7100053E8002F22F0806243E800210029F7D18E
:10B72000EDE70022C26653E8002F22F0100243E842
:10B7300000210029F7D1DA69B0F85C10D20644BFC5
:10B7400010221A62FFF7C2FD08BD9A6942F0080292
:10B750009A61F9E7008000402DE9F84F0368B0F8DE
:10B760006060D3F81CB01F689D68D0F88C20222A36
:10B77000044640F0B980B0F8683043B1DFF8749106
:10B78000DFF874A14FF000081BF0200F20D1B4F8AF
:10B790005E309BB2D3B1B4F868209A4216D92268C1
:10B7A00002F1080353E8003F23F08053083242E8D7
:10B7B000003122680029F2D1504B636752E8003F04
:10B7C00043F0200342E800310029F7D1BDE8F88FAB
:10B7D0002368A26D5B6A33401370A36D0133A365C8
:10B7E000B4F85E30013B9BB2A4F85E302368D3F816
:10B7F0001CB01BF0070F2ED01BF0010F09D0F9056C
:10B8000007D501221A62D4F8902042F00102C4F850
:10B8100090201BF0020F09D0EA0707D502221A6216
:10B82000D4F8902042F00402C4F890201BF0040FDA
:10B8300009D0E80707D504221A62D4F8903043F003
:10B840000203C4F89030D4F8903023B12046FFF7BB
:10B850000EFDC4F89080B4F85E309BB2002B93D1FB
:10B86000226852E8003F23F4807342E800312368E5
:10B870000029F5D103F1080252E8002F02EA09027B
:10B8800003F1080040E800210029F3D120225345AC
:10B89000C4F88C20616721670AD05A68110207D565
:10B8A00053E8002F22F0806243E800210029F7D1FD
:10B8B000E26E012A14D10022E26653E8002F22F042
:10B8C000100243E800210029F7D1DA69B4F85C10CE
:10B8D000D20644BF10221A622046FFF7F7FC53E756
:10B8E0002046F8F747FD4FE79A6942F008029A614F
:10B8F0006CE700BFFEFFFFEF00800040C9B5000805
:10B900002DE9F84F0368B0F86060D3F81CB01F68E9
:10B910009D68D0F88C20222A044640F0B780B0F809
:10B92000683043B1DFF87091DFF870A14FF0000884
:10B930001BF0200F20D1B4F85E309BB2D3B1B4F825
:10B9400068209A4216D9226802F1080353E8003FA2
:10B9500023F08053083242E8003122680029F2D1F6
:10B960004F4B636752E8003F43F0200342E8003149
:10B970000029F7D1BDE8F88F2368A26D596A3140DC
:10B9800022F8021BA265B4F85E20013A92B2A4F834
:10B990005E20D3F81CB01BF0070F2ED01BF0010F58
:10B9A00009D0F90507D501221A62D4F8902042F097
:10B9B0000102C4F890201BF0020F09D0EA0707D556
:10B9C00002221A62D4F8902042F00402C4F89020B7
:10B9D0001BF0040F09D0E80707D504221A62D4F837
:10B9E000903043F00203C4F89030D4F8903023B183
:10B9F0002046FFF73CFCC4F89080B4F85E309BB260
:10BA0000002B95D1226852E8003F23F4807342E86E
:10BA1000003123680029F5D103F1080252E8002F14
:10BA200002EA090203F1080040E800210029F3D1ED
:10BA300020225345C4F88C20616721670AD05A68D8
:10BA4000110207D553E8002F22F0806243E800215D
:10BA50000029F7D1E26E012A14D10022E26653E8F0
:10BA6000002F22F0100243E800210029F7D1DA6903
:10BA7000B4F85C10D20644BF10221A622046FFF7C9
:10BA800025FC55E72046F8F775FC51E79A6942F026
:10BA900008029A616EE700BFFEFFFFEF00800040E2
:10BAA00095B6000838B5044603682169A2681D6888
:10BAB000C0690A4361690A437749024329400A433E
:10BAC0001A605A68E16822F440520A435A60734A85
:10BAD000A16993421CBF226A11439A6822F06E4208
:10BAE00022F430620A439A60DA6A616A22F00F0235
:10BAF0000A43DA626A4A934219D14FF0B043694A65
:10BB0000D3F8883003F0030343F44033934200F04A
:10BB1000B480B3F1031F24D0013A934240F0B580C2
:10BB2000B0F5004F40F08F80FCF7C6FF6EE05E4A34
:10BB300093421CD14FF0B0435C49D3F8883003F0F6
:10BB40000C0343F440228A4200F0978006D8002B71
:10BB50007CD0574B9A42E3D0012026E0B2F10C1F73
:10BB6000FAD1B0F5004F53D04FF4004075E04B4A86
:10BB70009342F1D14FF0B043D3F8883003F44063DF
:10BB8000B3F5006F18D006D85BB1B3F5806FE3D181
:10BB9000FCF792FF07E0B3F5406FDDD14FF40040B2
:10BBA0000BE0FDF781FB40B900204FF00113A366C5
:10BBB0000023C4E91D3338BD3E4865683E4B626AC8
:10BBC00005EB450133F81220B0FBF2F39942C3D8DC
:10BBD000B3EB053FC0D800231946F6F765FC090210
:10BBE00041EA10616B080002C0182A464FF00003BA
:10BBF00041F10001F6F758FC304BA0F540729A4233
:10BC0000AAD82368D860CFE7FDF74EFB0028CBD039
:10BC10006168294B626A33F81220B0FBF2F24B08DC
:10BC200003EB42034FF6EF72B3FBF1F3A3F1100104
:10BC3000914291D823F00F02216892B2C3F34203DC
:10BC40001343CB60B0E7FCF737FF04E0B0F5004FDB
:10BC5000DAD0FDF729FB0028A6D06368616A164A8E
:10BC600032F81120B0FBF2F000EB5300B0FBF3F020
:10BC70004FF6EF73A0F11002C1E7B0F5004F0D4889
:10BC8000EBD1C5E7FDF720FBC0E7B0F5004FF9D0D9
:10BC9000FDF71AFBDFE700BFF369FFCF008000402C
:10BCA00000380140020003000044004008000C007E
:10BCB00004000C000024F400C0700308FFFC0F0017
:10BCC000836ADA0710B506D50168C46A4A6822F4A7
:10BCD000003222434A609C0706D50168046B4A681B
:10BCE00022F4803222434A60590706D50168446B2A
:10BCF0004A6822F4802222434A601A0706D5016866
:10BD0000846B4A6822F4004222434A60DC0606D56E
:10BD10000168C46B8A6822F4805222438A609906C3
:10BD200006D50168046C8A6822F4005222438A60B6
:10BD30005A060FD50168446C4A6822F480122243E7
:10BD4000B4F5801F4A6005D14A68846C22F4C002B1
:10BD500022434A601B0606D50268C16C536823F46F
:10BD600000230B43536010BD2DE9F843DDF820900C
:10BD700005460F46164698462A68D36937EA0303F4
:10BD80000CBF01230023B34201D0002029E0B9F108
:10BD9000FF3FF2D0F7F734FFA0EB080048452C68CE
:10BDA00002D8B9F1000F1ED154E8003F23F4D0733C
:10BDB00044E80032002AF7D104F1080353E8003FB9
:10BDC00023F0010304F1080141E80032002AF3D115
:10BDD0002023C5F88830C5F88C30002385F88430DE
:10BDE0000320BDE8F88323685A07C5D5E3691B051E
:10BDF000C2D54FF40063236254E8003F23F4D073AC
:10BE000044E80032002AF7D104F1080353E8003F68
:10BE100023F0010304F1080141E80032002AF3D1C4
:10BE20002023C5F88830C5F88C30C5F89030D4E7A9
:10BE300073B504460026C0F89060F7F7E1FE23686A
:10BE40001B681A07054619D423681B685B070AD5C7
:10BE50006FF07E43009300222B464FF48001204672
:10BE6000FFF782FFB0B900202023C4F8883084F89F
:10BE70008400C4F88C30E06620670CE06FF07E43ED
:10BE80000093324603464FF400112046FFF76CFF43
:10BE90000028D9D0032002B070BD10B5044650B3BD
:10BEA000D0F888301BB980F88430F8F763F922683D
:10BEB0002423C4F88830136823F00103136020465C
:10BEC000FFF7F0FD012816D0A36A13B12046FFF753
:10BED000F7FE23685A6822F490425A609A6822F06A
:10BEE0002A029A601A6842F0010220461A60BDE8F0
:10BEF0001040FFF79DBF012010BD000030B58165E7
:10BF00008168A0F85C200023B1F5805FA0F85E2076
:10BF1000436735D10369002B40F2FF1318BFFF239D
:10BF2000A0F860300023C0F890302223C0F88C3095
:10BF3000016801F1080353E8003F43F001030831B1
:10BF400041E800340368002CF2D1456E8468016931
:10BF5000B5F1005F32D1B0F8685095422ED8B4F5F3
:10BF6000805F244A03D1244C002908BF224642673F
:10BF7000B1B153E8002F42F4807243E80021F7E7A3
:10BF800029B90369002B14BF7F23FF23C8E7B1F150
:10BF9000805FC5D10369002B14BF3F237F23BFE718
:10BFA00003F1080252E8002F42F0805203F108002A
:10BFB00040E800210029F3D1002030BDB4F5805FB6
:10BFC0000E4A03D10E4C002908BF2246426741B1F8
:10BFD00053E8002F42F4907243E800210029F7D182
:10BFE000EAE753E8002F42F0200243E8002100294D
:10BFF000F7D1E1E759B7000801B90008C9B5000851
:10C0000095B60008D0F88C30202B30B415D1B9B1DA
:10C01000B2B100230468C3660A4B9C420AD063682D
:10C020001B0207D554E8003F43F0806344E8003525
:10C03000002DF7D130BCFFF761BF022030BC704744
:10C040000120FBE700800040436E30B52BB901238F
:10C05000A0F86A30A0F8683030BD0368094D9A68CE
:10C060009968094C490FC2F342626B5C615CDB006A
:10C07000B3FBF1F3A0F86A30AB5CA25CDB00B3FB6E
:10C08000F2F3E7E7E0700308D870030870477047E1
:10C0900070471FB504AB03E9060090F88430012B0C
:10C0A00004463AD0012380F884302423C0F8883035
:10C0B00003681A6822F001021A609A6822F440129A
:10C0C0000A439A6071B95A68BDF80C009DF80E10C9
:10C0D00022F0100202435A605A6822F07F4242EA7C
:10C0E00001625A601A6842F001021A60F7F788FD8F
:10C0F0006FF07E42034600924FF4800100222046FA
:10C10000FFF732FE38B92023C4F88830002384F8C2
:10C11000843004B010BD0320F8E70220F9E790F85E
:10C120008430012B0FD0012380F88430016851E85E
:10C13000002F42F0020241E80023002BF6D180F8E4
:10C140008430184670470220704710B590F884304C
:10C15000012B044617D02423C0F8883003681A68DE
:10C16000196821F00101196042F000524FF00051AE
:10C1700041661A60FFF768FF2023C0F8883000206E
:10C1800084F8840010BD0220FCE770B590F884307C
:10C19000012B044617D005682423C0F888302E6888
:10C1A0002B6823F001032B60AB6823F06043194335
:10C1B000A960FFF749FF20232E60C0F888300020D7
:10C1C00084F8840070BD0220FCE770B590F88430DC
:10C1D000012B044617D005682423C0F888302E6848
:10C1E0002B6823F001032B60AB6823F060631943D5
:10C1F000A960FFF729FF20232E60C0F888300020B7
:10C2000084F8840070BD0220FCE7000038B5084DBA
:10C21000052455F8043B2BB9013C14F0FF04F8D178
:10C22000204638BDDB6898470028F5D0F9E700BF05
:10C23000D8220020034BD870034B1B681B6C03B142
:10C2400018477047C0220020BC220020034B1874FE
:10C25000034B1B685B6C03B118477047C02200207A
:10C26000BC220020F0B5314D314B95F90420314E00
:10C2700091B00C46012795F905108DF8047002283D
:10C280008DF809208DF80A1010D18DF80800D871AA
:10C290001C7202F063FD337803B114B101A803F0FE
:10C2A000C1F9254B059A1A6011B0F0BD59714FF4D0
:10C2B00080711A71D9801C7233788DF8087053BB65
:10C2C0001F2306A88DF81C208DF8183002F024FFDB
:10C2D00020238DF8183006A82B798DF81C3002F039
:10C2E0001BFF22238DF8183006A86B798DF81C30BF
:10C2F00002F012FF21238DF8183006A86B798DF813
:10C300001C3002F009FF29238DF8183006A80B4BCA
:10C31000079302F001FF02F021FD012306A88DF82A
:10C3200018308DF81C3002F0F7FEB4E7C022002070
:10C33000E00300209C210020902200200004000146
:10C340007FB5092301A88DF8043003F06BF900389C
:10C35000044B059A1A6018BF0120404207B05DF8EF
:10C3600004FB00BF9022002070B504460B46144920
:10C3700062784A700020A2780A7208701A884A729D
:10C380009A788A72DB780B746368CB600D4B1B68FC
:10C39000DA6A2AB1237803F0FB030A2B00D0904716
:10C3A000094E002556F8043B1BB15B6A0BB12046D1
:10C3B00098470135EBB2052B6DB2F3D170BD00BFCC
:10C3C000B0030020BC220020D822002070B5044613
:10C3D00011480123037063784370A3788372E36884
:10C3E000C360E378037623694376237943720B4B6A
:10C3F0001B689B6A03B19847094E002556F8043B19
:10C400001BB19B690BB1204698470135EBB2052B58
:10C410006DB2F3D170BD00BFC4030020BC22002068
:10C42000D8220020014B1868704700BF90220020DE
:10C4300000B58BB0012368468DF8003002F046FD50
:10C4400038B99DF80400003818BF01200BB05DF822
:10C4500004FB0020FAE7000008B501F037FE40B900
:10C46000FFF7E6FF012806D0054B197AD879FFF7C8
:10C47000F9FE012008BDBDE80840FFF7C7BE00BFB8
:10C48000E00300202DE9F04186B005460E46174630
:10C4900001F01CFE002873D101F030FE044640B9C3
:10C4A000FFF7C6FF01280AD03D4B197AD879FFF76C
:10C4B000D9FE6FF00204204606B0BDE8F081DFF837
:10C4C000E48088F80860003E18BF01268DF80460FB
:10C4D000354E687833798DF81230694602F094FC55
:10C4E00000283FD08DF804400394ADF810406FF061
:10C4F000060495E803002D4B83E80300337988F8A0
:10C500000A30394601A803F091F9294B059A1A60BF
:10C5100011283FD801A353F820F000BF87C50008B9
:10C5200081C5000895C5000895C5000895C5000897
:10C5300095C5000895C50008B3C4000895C5000856
:10C5400095C5000895C500087BC5000895C500087D
:10C5500095C5000881C5000881C5000881C500088F
:10C560009BC500082B788DF808306B78ADF810303B
:10C570006B6803934FF0FF34BBE76FF005049AE755
:10C580006FF0010497E70B4B00221A70E31D18BFF0
:10C59000144690E74FF0FF348DE76FF004048AE70C
:10C5A000E0030020C4030020C0220020D4030020A8
:10C5B000902200208F22002037B501F0A9FD134DF5
:10C5C000052455F8043B4BB11A693AB19B682BB16D
:10C5D000984718B155F8043C1B699847013C14F082
:10C5E000FF04EED1FFF712FE68B9094D2B7853B165
:10C5F000084BADF80040D978019422466846FFF711
:10C6000041FF00B92C7003B030BD00BFD82200201C
:10C610008F220020C022002030B58BB0044601F0EC
:10C6200055FD0546002835D1FFF702FF012834D11A
:10C6300068468DF8005002F049FC40BB9DF804307C
:10C64000A34204D0012C22D0022C12D014B100201D
:10C650000BB030BD002BFAD068468DF8044002F0D4
:10C660005BFDA0B90E4B1B681B6B002BEFD09847EE
:10C67000EDE763B968468DF8044002F04DFD30B92E
:10C68000074B1B681B6B002BE1D02046EFE74FF0F8
:10C69000FF30DDE76FF00100DAE76FF00200D7E767
:10C6A000BC22002010B504468AB018B94FF0FF3004
:10C6B0000AB010BD002368468DF8003002F006FC79
:10C6C0000028F3D19DF804302370F1E77FB50022F4
:10C6D0000B4620498DF8072001220A7042784A70E3
:10C6E0000446002A33D102790A721A884A729A786B
:10C6F0008A72DB780B740369CB60C378164D8DF8B2
:10C700000830037B8DF80930836803932B68DB6A5C
:10C710000BB102A898472B689B6B13B1227E02B124
:10C7200098470E4E052556F8043B1BB1DB690BB14B
:10C7300020469847013D15F0FF05F4D10DF10700A3
:10C74000FFF7B0FF637913B1054B01221A7004B0F3
:10C7500070BD00BFB0030020BC220020D822002002
:10C760008F22002010B504468AB018B94FF0FF3070
:10C770000AB010BD202368468DF8003002F0A6FBF9
:10C780000028F3D1024A9DF9043023701371EFE7BA
:10C79000C022002000B58BB02323019068468DF89D
:10C7A000003002F0B9FC003818BF012040420BB045
:10C7B0005DF804FB70B5654C01468EB0182220462A
:10C7C00006F08CF8624B00221A70FAF7C5FE237847
:10C7D0004068012202FA03F1014004D15D4B084692
:10C7E00008F068F8FEE75C495C481A4602F0F8F881
:10C7F00018B14FF0FF300EB070BD272304A88DF89C
:10C80000103002F089FC564E564D002870D101239D
:10C8100033702B68DB690BB100209847272304A8ED
:10C820008DF8103002F052FB059B93F848202270DF
:10C8300093F8182193F81A316270A370464BD3E92C
:10C84000020105F03BFF05460028D2D1464E0623E3
:10C8500004A88DF8103002F039FB059B736104A821
:10C8600002F05AFC022304A88DF81030059602F05D
:10C870002DFB0836032304A88DF81030059602F02E
:10C8800025FB0F2605F0E0FF012304A88DF81430E6
:10C890008DF8106002F040FC10230DEB03008DF8C2
:10C8A00010308DF8145002F037FC04238DF810304E
:10C8B00004A8A3788DF8143002F02EFC3A238DF8EA
:10C8C000103004A86369059302F026FC02A92078C1
:10C8D0008DF8086004F09CF8003818BF0120E07162
:10C8E0001420FFF757FFE07903F062F9284682E74A
:10C8F00028238DF810302B681B6943B104A802F07F
:10C90000E5FA2B6805981B6940F2C4519847272324
:10C9100004A88DF8103002F0FFFB50B9012304A8E1
:10C920008DF8103002F0D2FA9DF81430002B7FF40D
:10C930006EAF3378002B7FF46CAF052204A88DF81E
:10C940001020059302F0E8FB78E700BFC02200202A
:10C950008F220020E870030894220020AC220020DF
:10C960009C210020BC220020FC22002037B500239F
:10C970000D4601930446D0B900F0A8FB0190019B3D
:10C98000D3B10F4A42F824300E4A9A620E4A126816
:10C99000916B1963916C596392690C49D9625A6120
:10C9A00028465B680A49F2229847002006E001A960
:10C9B00000F092FB0028E2D04FF0FF3003B030BD12
:10C9C000D822002065C20008BC22002041C3000814
:10C9D0009D210020194B07B51860194B194A1A60A0
:10C9E000194A5A60194A9A60194ADA60194B026862
:10C9F0001A6042685A6082689A60C268DA60164AB1
:10CA00001A6182695A61154BC26B5A60144A0191CE
:10CA100019609A601946134ADA600020FFF7A6FFF2
:10CA200048B901A800F056FB003818BF0120404269
:10CA300003B05DF804FB4FF0FF30F9E7BC220020A3
:10CA4000AC220020CDC30008CDC60008E1CA000812
:10CA500069C3000894220020C1090108EC220020CB
:10CA600035C200084DC2000849B118B1012804D0F0
:10CA700000207047034B0B60FAE7034BFBE74FF0D6
:10CA8000FF307047000400010100010208B503F007
:10CA9000ABF8002814BF6FF00100002008BD08B5F6
:10CAA00002F084F9002814BF6FF00100002008BDD7
:10CAB00010B504468AB018B94FF0FF300AB010BD67
:10CAC000212368468DF8003002F000FA0028F3D1E7
:10CAD000024A9DF9043023705371EFE7C022002011
:10CAE0002DE9F0412F4D304F00232B7043786B70B0
:10CAF0003B689B6A8AB004460BB128469847DFF82A
:10CB0000AC80002658F8043B1BB11B6A0BB12046D1
:10CB100098470136F3B2052B76B2F3D12378052B73
:10CB20002FD00B2B35D0012B25D1214C0623684665
:10CB30008DF8003002F0CAF90199E07905F004FEA1
:10CB400010B91C4B019A5A611B48FFF70BFE1B489A
:10CB5000FFF7AEFF6B788BB9A371194B5878FFF7CD
:10CB60005BFD3B685B6A0BB1114898476B7813B962
:10CB7000E07905F07BFE0AB0BDE8F081FF23A371E8
:10CB8000EFE7104B01225A74227A9A74627ADA74AF
:10CB9000F1E76378002BEED00AB0BDE8F041FFF773
:10CBA000CFBB00BFC4030020BC220020D82200203D
:10CBB000E0030020FC220020E4030020E503002025
:10CBC000C0220020B003002030B58BB0FFF767FF14
:10CBD0000446F0B903F0FCFE831C1DD0F8B9134DD8
:10CBE0002B685B69DBB1272368468DF8003002F0C3
:10CBF0006DF92B6801985B694FF4B961984703F0B0
:10CC0000F9FE78B92CB9094B1B68DB690BB101201F
:10CC1000984720460BB030BD6FF00704EFE74FF0A8
:10CC2000FF34ECE74FF0FF34F3E700BFBC220020F5
:10CC3000014B1878704700BF30230020014B587813
:10CC4000704700BF3023002070470000044B9A7AE1
:10CC50000AB101225A70034B5B6903B11847704750
:10CC600030230020EC03002073B5224C6378002BA6
:10CC700033D008F007F966680546FFF7D3FB064492
:10CC8000AE4214D2A37A93B1E0228DF800208DF841
:10CC90000130217AE368019301226846FFF7F2FB35
:10CCA00008B1073010D100236370A372656094F857
:10CCB0003430EBB1002384F834300F4B5B6BBBB1E5
:10CCC00002B0BDE87040184740F2DC510B4808F054
:10CCD000A5F90A4808F068F9E8E794F83520002A31
:10CCE000E5D094F8360084F83530FFF795FCDEE7A0
:10CCF00002B070BD30230020EC030020142300207C
:10CD000037B5104D104CC8B1C1B162720123002279
:10CD10002860E16023700D480D4B00924FF0FF3109
:10CD200008F096F800250B4825822022294605F0B8
:10CD3000E9FD6570A574A58603B030BD00232B60A6
:10CD40002370EFE72C230020302300201423002041
:10CD50004DCC0008442300202DE9F0478E4C237869
:10CD60008CB0002B56D0C2780AB9837B13B1238ACA
:10CD700001332382437B002B4CD0E02A4AD100238D
:10CD8000A372876897F80080B8F1220F27D8B8F10E
:10CD9000220F30D8DFE818F04100FB0052005A00A3
:10CDA00061006E0075008E009D00B400C7002F006A
:10CDB0002F002F002F002F002F002F002F002F00FB
:10CDC0002F002F002F002F002F002F002F002F00EB
:10CDD0002F002F002F002F00C900D000D400B8F181
:10CDE0007E0F00F0CC80B8F17F0F00F0DF80B8F14B
:10CDF0007D0F00F0AB80A57A002D00F05B81674CC1
:10CE0000637A3BB94FF47A71204608F007F920465F
:10CE100008F0CAF80CB0BDE8F087E36801220021F1
:10CE2000A2721970A37AE1689818A0720620C854FB
:10CE3000A37AE1689818A072CA54DCE7584B9B6A41
:10CE4000002BD8D0012102209847D4E77B7884F8C2
:10CE50003630012384F83530CDE704238DF80430D3
:10CE60007B78003B18BF012301A88DF8083002F041
:10CE700053F9C0E77878003818BF012002F098FE17
:10CE8000B9E7484E0FCE01AD0FC50FCE0FC596E8DE
:10CE9000070085E807007B780A2BACD8424A126865
:10CEA0005268002AA7D00CA901EB830353F82C0C7D
:10CEB0009047A0E77878431E012B9CD83A4B013865
:10CEC0001B6818BF012020729B68002B93D09847E5
:10CED00091E7E26801230821A3721170627A057B51
:10CEE000A17AAA4228BF2A46934284D285685A1C56
:10CEF000EB5CE56801334E1CA6726B54D3B2EDE7D0
:10CF0000E3680122A27209221A70A37AE268218AD8
:10CF1000581CA072D154A27A238AE1681B0A501CC3
:10CF2000A0728B5467E7238265E705238DF80430F0
:10CF300001A802F077FB5EE7194BDB6A98475AE7D6
:10CF4000194B78781B686075DB68BEE7037B072B9D
:10CF50007FF451AF06238DF80430B7F80130ADF8F7
:10CF600008307B793A791B0443EA0223FA781343A9
:10CF7000642253430393BB798DF81030D8E73B22EA
:10CF800001A88DF804208DF8083002F0C5F80123BF
:10CF900084F834302FE700BF302300201423002012
:10CFA000EC0300206C1B03082C2300202A2301A87B
:10CFB0008DF8043001F08AFF94F80A90E6689DF835
:10CFC00008009DF809509DF80A709DF80BC09DF867
:10CFD0000D309DF80E209DF80F109DF80CE009F122
:10CFE000010A84F80AA006F80980354E94F80A90E0
:10CFF0003668D4F80C8009F1010A84F80AA096F882
:10D0000003A008F809A094F80A90D4F80C8009F15C
:10D01000010A84F80AA096F802A008F809A094F87A
:10D020000A90D4F80C8009F1010A84F80AA096F855
:10D0300001A008F809A094F80A9009F1010A84F8FF
:10D040000AA096F80080E66806F8098094F80A803D
:10D05000E66808F1010984F80A9006F808C094F817
:10D060000AC0E6680CF1010884F80A8006F80C7022
:10D07000A77AE66807F1010C84F80AC0F555A57A8D
:10D08000E6686F1CA7727055A07AE568461CA67208
:10D090002954A17AE0684D1CA5724254A27AE16835
:10D0A000501CA0728B54A37AE268591CA17202F83A
:10D0B00003E0A0E6034807F029FF6570AAE600BF79
:10D0C0002C230020142300207047000000487047E4
:10D0D000EC030020002070474FF0FF307047000045
:10D0E000044B054A93F81831022B18BF062382F827
:10D0F00090347047D4290020982F0020034BD3F898
:10D10000483313B15B6903B118477047982F00206B
:10D11000034A137843F004031370FFF7EFBF00BF17
:10D120007C2300201FB50A4B8DF8090093F87C2062
:10D130008DF80A2093F88C2093F848000D3202A94C
:10D140008DF8082003F064FCC0B205B05DF804FB64
:10D15000D429002008B5074807F0D8FE064B93F8FD
:10D160001A2412B1012283F81924BDE80840FFF700
:10D17000C5BF00BF98330020982F002010B50C4C7D
:10D18000D4F8403343F08003C4F8403394F81A34A1
:10D1900013B10020FFF7DEFF94F8913423F012035F
:10D1A00043F0120384F89134BDE81040FFF798BFB4
:10D1B000982F00202DE9F041DFF8AC8098F8183165
:10D1C000022B06460D4602D0284BDB6A984702F038
:10D1D000A6FD044628B1022002F097FD002002F0CF
:10D1E00099FD98F81831012B17D102F09AFD0746E6
:10D1F00030B1002002F08AFD002002F08CFD3C4698
:10D2000002F091FD48B1002002F081FD002002F003
:10D2100083FDBDE8F041FFF763BF002CF9D1144C4A
:10D2200094F8902494F81A34BAB90BB184F8416494
:10D23000304602F017FFD8F82C0007F02DFED4F886
:10D24000B4339842E5D30B4807F060FE94F891346C
:10D2500043F0100384F89134DBE70BB184F84154B8
:10D26000284602F0FFFEF1E7D42900206078030889
:10D27000982F002030330020074A10B5137843F070
:10D2800002031370FFF73AFFBDE81040034B012281
:10D290000021022007F00EBB7C230020317103081F
:10D2A000074A10B5137843F008031370FFF726FF01
:10D2B000BDE81040034B01220021022007F0FABA1A
:10D2C0007C230020417103082DE9F0410F461646EA
:10D2D0001D46804607F0D6FD0B4A0C4C137827817B
:10D2E00023F0110343F01103C4E9000813706681B1
:10D2F0002573FFF703FFBDE8F041054B0122002134
:10D30000022007F0D7BA00BF7C230020682300204A
:10D310005171030813B507F0B5FD0D4B6C4618604D
:10D32000204607F003FD94E803000A4A0A4B83E80D
:10D330000300137843F020031370FFF7DFFE074B61
:10D3400001220021022002B0BDE8104007F0B2BA6D
:10D35000782300207C230020D03200205E71030857
:10D360002DE9F04192B0064602F0D9FC002840F0C9
:10D370005881AD4D95F81831012B09D02B6BAB4C72
:10D3800093B194F80431BBB1042B6FD0032003E0B8
:10D3900002F0C7FC18B10F2012B0BDE8F08102F016
:10D3A000C2FC0028EAD0F6E7B5F82031D4F81C24F6
:10D3B000013B53432B63E4E79D4803F060FA0028E8
:10D3C00040F0128194F80C3123802B6B0C930DF1FB
:10D3D000180895F839308DF83830404695F81C31EA
:10D3E0008DF83A3007F0C8FCD5F82831009302AF29
:10D3F00098E80600D5F82431384607F054FC97E841
:10D4000003000FAB83E80300EB6A0D9300238DF854
:10D4100044302388ADF8463095F8303101228DF83C
:10D4200039201BB98DF844208DF83930814B009399
:10D43000814B95F84800A3F179020CA903F05DFB3C
:10D44000C0B10B28A8D1D4F8941499B1002EA3D060
:10D45000D4F84033794843F02003C4F8403307F050
:10D46000DDFD764807F0A0FD002095E7704803F049
:10D470003AFAA4E795F8487095F9693095F939209A
:10D4800095F87D106E4E384603F044FB009641B28D
:10D49000EB6C95F850203846183603F0DFFA00960A
:10D4A000EB6C95F8502095F9701095F8480003F052
:10D4B000D5FAD4F8C413AB6DD4F8DC230B44C4F80C
:10D4C000B033EB6D1344C4F8B43394F80431042B37
:10D4D00007D02B6E0B44C4F8B0336B6E1344C4F802
:10D4E000B4330023089395F83031002B40D100234A
:10D4F0008DF8133095F839308DF8213095F83830A3
:10D500008DF82230D5F880300993D5F884300A930D
:10D510002388ADF82C3095F8303194F81B648DF8E1
:10D520002E3095F84800474B8DF820600DF113021E
:10D5300008A903F0A7FA012384F8413495F839309B
:10D5400084F842349DF8133084F84334D4F81C3402
:10D55000C4F85064C4F84834C4F8583402F0E5FB09
:10D56000C8B1D4F81C0402F0F2FBA0B1102013E7FC
:10D5700008A802F0A7FC60B995F9390094F8376261
:10D580009DF82070FFF7CEFD3E44B042AFD2082098
:10D5900002E7132000E795F81831012B01D102F0C2
:10D5A000D8FB02F0C5FB0023059394F8043195F9EC
:10D5B000395094F81B649BB1042B7FF4E7AE05A8A7
:10D5C00002F0B4FE58BB94F8183413B1059B013B2C
:10D5D0000593174B05983246E9B202F00DFF02E0C1
:10D5E000134802F0DDFE08B11120D5E6D4F840332F
:10D5F00094F80C11218043F00203C4F8403394F8EE
:10D60000183411480133DBB284F8183484F84534F7
:10D610000E4B00259B6AC4F89854984724E71220C3
:10D62000BAE60E20B8E600BFD4290020982F0020CB
:10D63000A0300020042A00202C34002000330020D9
:10D6400050330020B43300209A2F00206078030864
:10D6500073B5134D134E0096EB6C95F8502095F969
:10D66000781095F8480003F0F9F995F830313375E2
:10D6700095F8480040F2012306F13C0231467382DE
:10D6800003F0F8F950B196F83C3086F88230064B3A
:10D6900000205B6B9847F37C86F8A83002B070BD21
:10D6A000D42900208033002060780308F8B5324C7C
:10D6B00094F81831012B05460ED0022B4ED0002BCA
:10D6C00057D138B9D4E91B0104F1740383E803008E
:10D6D0000020F8BD012806D102F02CFB0028F8D16B
:10D6E00084F81851F5E7022843D1244E84F8180134
:10D6F00006F5747CBCE80F0006F57A770FC79CE846
:10D70000030094F8E92094F8003187E8030086F8D4
:10D71000FB53D2B1022B18D1D4F804316367C6F899
:10D72000EC3394F87D3094F8082186F8F83394F8B7
:10D730008C3084F8782086F8F93396F81B2486F824
:10D74000E82340F20133A6F8FA33002386F81A34AE
:10D750000B4BDB6A9847FFF77BFFB9E748B9074BEC
:10D7600084F81801062283F89024054BDB6A984759
:10D77000AEE70320ADE700BFD4290020982F00209A
:10D7800060780308F0B5504C504EB4F8DC20228786
:10D79000D4E92D0194F8B12084F8692004F16C02D9
:10D7A00082E80300D4E92F0104F1740282E8030047
:10D7B000B4F8C420A4F87C2091B0D4F8CC20D4F8DC
:10D7C000C810C4F884200025D4F8D020C4F88820DC
:10D7D0000123A4F82031C4F8801084F83051A562E8
:10D7E00084F81B5184F83A5084F81D5184F81E5176
:10D7F000C4F83451C6F89854A6F8185486F81A5448
:10D80000A4F838518DF8183004F50973039304F522
:10D810000A7394F84800049303A92D4B84F84551EA
:10D82000C4E94F55A4F84651059303F0FFF8E36EA1
:10D83000C6F8D43394F87D3086F8E03394F88C3011
:10D8400086F8E1334FF48073A6F8E23386F8D053BC
:10D8500094F8303186F8E43306F574770FCF06F587
:10D860007A740FC497E8030040F2012384E80300B0
:10D87000A6F8FA33D6F8483386F81B54CDE901559B
:10D880001BB15A685B6901920293124B0793A3F193
:10D8900048020892A3F1140209920F4A0B9229330D
:10D8A0000A93A2F19C030C93A2F198030D93131D0C
:10D8B0000E9301A902F14C0307A802F599620F9398
:10D8C00002F022FA11B0F0BDD4290020982F0020D8
:10D8D0008023002000340020B82A0020F8B50D4F26
:10D8E0000D4E0C4607F012FB3B6B98470B4A96F81F
:10D8F0004800214603F0BEF850B1094D706D95F80F
:10D90000243485F86A347B6B9847E37C85F890343F
:10D91000F8BD00BF60780308D4290020BC33002084
:10D92000982F00200F4890F81B3480F8B8330E4B26
:10D9300093F8692080F8BB2393F87D2080F8C823F2
:10D9400093F88C2080F8C92393F8303180F8CC33D9
:10D950000022A0F8CA2300F56E7100F56070FFF791
:10D96000BDBF00BF982F0020D4290020114890F897
:10D970009034EBB190F81B3480F8D0330E4BDA6E54
:10D98000C0F8D42393F87D2080F8E02393F88C200E
:10D9900080F8E12393F8303180F8E4334FF480725B
:10D9A000A0F8E22300F5747100F56670FFF796BFEA
:10D9B000704700BF982F0020D429002070B5344C48
:10D9C0002421204604F0A0FF636A984218BF6062D9
:10D9D0004FF01C012F4814BF0125002504F094FFCF
:10D9E000636C984218BF60644FF480712A4818BF76
:10D9F00045F0020504F088FFD4F84831984218BF7A
:10DA0000C4F848014FF0D401244818BF45F004057C
:10DA100004F07AFFD4F82032984218BFC4F82002EC
:10DA20004FF000011E4818BF45F0080504F06CFFD8
:10DA3000D4F82432984218BFC4F824024FF460711D
:10DA4000184818BF45F0100504F05EFFD4F8A8355B
:10DA5000984218BFC4F8A8054FF01401124818BF27
:10DA600045F0200504F050FFD4F8C03598420F4B24
:10DA700018BFC4F8C005D3F8483318BF45F04005B7
:10DA80002BB11B691BB12846BDE87040184770BD1B
:10DA9000D4290020FC2900201C2A0020202B002053
:10DAA000F82B0020FC2B0020802F0020982F002036
:10DAB0002DE9F04F8FB04FF00009012B06460F46BD
:10DAC00090468DF80D90ADF8109002D84C46BC42AF
:10DAD00002D30FB0BDE8F08F305D02F033FA20447E
:10DAE000B842F6DC335D651C023BEDB2112BF0D879
:10DAF00001A252F823F000BF41DB00086BDB0008F5
:10DB000069DC000891DC00080FDD000835DD000845
:10DB10009BDD0008C3DD000849DE0008D3DA0008F9
:10DB2000D3DA00089DDE0008D3DA0008D3DA000853
:10DB300045DF00086DDF0008A5DF0008D9DF000819
:10DB4000052002F0A7FA70B10521002002F068FA62
:10DB5000725DBA4BE51C0234E4B283F85C24325D9A
:10DB600083F85D24EDB22C46B1E700238DF80E302A
:10DB70008DF80F308DF814308DF81830B9F1000F92
:10DB80006DD1AF4C4FF0050994F87C208DF8312011
:10DB90006B1E94F839208DF83320334494F83820E4
:10DBA0000B938DF8342094F81A3194F868208DF88E
:10DBB0003520D4F82C218DF832300A9273B37B1CB7
:10DBC0005B1BDBB28DF8303006AB019305AB0093E5
:10DBD00094F848000DF10F030DF10E020AA902F0AE
:10DBE0005DFF8DF80D0000F00700072813D194F9B0
:10DBF00039209DF90E3084F839309A429DF80F3063
:10DC000084F83830B8BF01229DF81430B8BF84F8CA
:10DC10001D2184F868304FF0000A09E00523D1E7A0
:10DC200001220DF10D01032002F0A4F80AF1010A0E
:10DC30005FFA8AF29DF81830B3FBF9F19142EFD800
:10DC40002B44DDB26B1EDBB29F420BD9F25C032A80
:10DC50009AD0AF4288BF1D464FF0010983E70534D3
:10DC6000E5B2F9E71D46F7E7735D754903F00F0369
:10DC7000012281F81B31023402FA03F3A1F82031AA
:10DC8000E4B2002204A9042002F074F825466AE7F1
:10DC900007238DF80D30735DC3F3021203F00F03F9
:10DCA0008DF82830E31CDBB28DF82920F25C231DAF
:10DCB000DBB2651DF35C0234E4B21B0443EA0223C9
:10DCC000325D5F4C13436422534394F848000B9336
:10DCD0000AA902F0F2FE00F00703072BEDB28DF85F
:10DCE0000D000CD19DF8283084F8703084F878301D
:10DCF0000B9BE36663679DF8293084F869308DF8E3
:10DD00001000012204A9052002F034F82BE74B4B48
:10DD1000D3F8483363B11B6853B1984708F03F0309
:10DD20008DF810008DF81130022204A90620EBE7CF
:10DD3000FF20F3E703238DF80D30735D8DF81C3061
:10DD40000AAB0693E31CDBB2A51DF25C231DDBB21C
:10DD500006A9F35C1B0443EA0223A21CD2B20534D9
:10DD6000B25C134364225343E4B20A9300230B933F
:10DD7000335D8DF83030324B93F8480002F0A3FE4B
:10DD8000C3B20028EDB28DF80D30FFF6ECAE8DF881
:10DD90001030012204A90720B6E7735D03F00F03DA
:10DDA000012B4FF47A7238BF01235343244A0234C3
:10DDB000936503F57A73D365E4B2002204A90820C1
:10DDC00062E7735D1E4DC3F340128DF8152095F880
:10DDD0004800C3F3001205A903F00F038DF81420C7
:10DDE0008DF8163002F075FE02340130E4B23FF4D3
:10DDF0004DAFBDF81430134AA5F87C309DF81630AD
:10DE00009DF814A0D05CF4F7D5F80223C5F8800083
:10DE10000AA995F848008DF828308DF82AA002F05C
:10DE2000F7FD95F93930069040B29842B8BF1846D0
:10DE300085F83900002204A9092025E7982F002041
:10DE4000D42900206B71030803238DF80D30735D16
:10DE50008DF82830E31CDBB2651DF25C231DDBB2BC
:10DE60000234F35CE4B21B0443EA0223325D134341
:10DE7000642253430B93644B0AA993F8480002F0C1
:10DE80002EFEC3B20028EDB28DF80D30FFF66BAE5A
:10DE90008DF81030012204A90A2035E7092002F08C
:10DEA000F9F8DFF868B1002849D00921002002F014
:10DEB000B7F80023ADF81E30A31CDBB2F25CE31C04
:10DEC000DBB216F803A0735D4FEA0A4A4AEA022A57
:10DED0004AEA030A231DDBB2A51D0534F35CE4B254
:10DEE0004AEA036A335D4FF47A7253430AAC1B1259
:10DEF0002046ADF81C3006F019FF454B53440693FD
:10DF0000DBF83C3300930DF1180A9AE80600DBF8C1
:10DF1000383308A806F0C7FE099B009394E8060072
:10DF2000089B504606F0A4FE9AE8030006F0D6FED1
:10DF300001F00AFF0123EDB28BF8383413E68BF8B9
:10DF4000380410E60C2002F0A5F800283FF40BAED0
:10DF50000C21002002F064F82C4B93F89034043B21
:10DF6000012B7FF600AE01F0EBFEFCE5A31CDBB25B
:10DF7000725DF15CE31CDBB2651DF35C0434E4B25A
:10DF80001B04305D43EA012313436421594300F02D
:10DF90000F0001F0D6FEEDB28DF81000012204A9A9
:10DFA0001120B1E60D2002F075F800283FF4DBAD3A
:10DFB0000D21002002F034F8A31CDBB2154AF05CFE
:10DFC000735D1268251D0334E4B243EA0020315D1D
:10DFD000EDB201F0B8FEC6E5725DA31C251D033449
:10DFE000DBB2E4B2F15C335D1B0443EA012313436B
:10DFF0006420584301F0A9FEEDB28DF81000012213
:10E0000004A9132080E600BFD4290020982F002007
:10E01000803DD512682300200E4B93F8912492077F
:10E0200003D593F88F24012A08D90B4991F81A21B6
:10E0300022B18A6A501C18BF01328A620022A3F8FA
:10E04000182483F81A24D3F8402322F00202C3F8DC
:10E0500040237047982F0020D429002070B5184C19
:10E060001848194D06F052FFD4F84033D4F89804FC
:10E07000D5F8906023F02003C4F8403338B106F09F
:10E080000BFF864203D2002385F83A3070BD012091
:10E09000FFF766F90028F9D00B28F7D095F839304A
:10E0A00084F84234092094F8183484F8453484F80C
:10E0B000410401F0D7FFBDE87040FFF7ADBF00BFDE
:10E0C000982F002000330020D4290020094BD3F8DA
:10E0D0004023012A0AD008490978C90708D43AB967
:10E0E00093F89204013818BF012070470020704750
:10E0F00001207047982F00207C230020034BD3F889
:10E100004003431E58425841704700BF982F0020DB
:10E110002DE9F04FA9B0EFF3108272B6DFF8F0B23C
:10E120000021DBF80030CBF8001082F31088B94CE6
:10E13000002B00F0E180DAB29B06039264D5B64D65
:10E1400095F81831022B02D0B44BDB6A9847EFF3F5
:10E15000108872B6B24F06F095FE3E68D4F8B01340
:10E16000361A3144AF4806F059FFAE4806F01CFF9E
:10E17000D4F8B413AC48314406F050FFAA4806F076
:10E1800013FF88F3108894F81A34002B00F06B8189
:10E19000152312A995F848008DF8483002F038FC94
:10E1A000D4F8B4130F900144A04806F037FF9F48FD
:10E1B00006F0FAFE3B6894F81B24EB620DAF38467C
:10E1C0008DF870201D9306F0D7FDD5F82831009307
:10E1D00006AE97E80600D5F82431304606F063FD18
:10E1E00096E803001FAB83E80300D4F81C341E93A9
:10E1F00095F8303195F84800003B18BF01231CA961
:10E200008DF8713002F00DFC039BDF0648D5824D7E
:10E21000DFF81CA2D5F8E42004929BF80020BAF99C
:10E220000A809AF90C90A4F88C84002363F300020E
:10E230000A9384F84434A4F8223484F82534C4F8CA
:10E240002834A4F82C3484F82E34C4F8303484F8FC
:10E250002034C4F8343484F83834C4F83C346F4B78
:10E260008BF8002094F89024DB6A84F88E9484F86C
:10E270008F24DAF80470BAF80860984794F88F345D
:10E2800013B9694806F042FE3146384601F045FDB3
:10E290008346002800F0EA80A4F87E8484F8809405
:10E2A000039B19071AD55C4B93F81831022B02D047
:10E2B0005A4BDB6A98470220FEF712FF84F84104AC
:10E2C00001F0D0FE94F81A3413B1012384F8193404
:10E2D00094F8913443F0100384F89134039B5A0767
:10E2E00003D506210520FEF765FF039B9B0703D599
:10E2F00004210320FEF75EFF01F02DFD94F8912428
:10E30000D7065FD5002384F89234D4F840331E0634
:10E3100044BF23F08203C4F8403312F0050F00F02D
:10E32000FB820B2001F0B6FE002800F0F58294F885
:10E330009134DD0700F1F082580740F10783D4F8EB
:10E34000403323F00203C4F84033D4F8402382BBA7
:10E3500094F8915415F001011EBF2B4662F300039F
:10E3600084F8913494F891345E0744BF6FF38203CC
:10E3700084F89134012384F8923421B1D4F84433E1
:10E380002C481B6898476D070BD52B4801F08EFE73
:10E3900001F0BCFE28B194F8913443F0040384F8F2
:10E3A000913401F0C6FC94F891346FF3041384F8AF
:10E3B0009134012384F8923494F8913443F020038B
:10E3C00084F8913494F8913418070AD56FF3C30395
:10E3D0001A4984F89134D4F84433A1F12400DB685D
:10E3E000984794F8913499070AD56FF3410313497C
:10E3F00084F89134D4F84433A1F16C005B689847F9
:10E4000094F89034022B1BD1FFF722F918E000BFDB
:10E410007C230020982F0020D42900206078030856
:10E420007823002018330020303300209833002058
:10E4300068230020D8330020EC330020243400204F
:10E4400094F891349A0640F1C4826FF3451384F82E
:10E450009134D4F84033002B40F0BB8229B0BDE8A2
:10E46000F04FFFF7ABBA84F84134A3E695F81831C2
:10E47000012B0CD101F055FC804668B1584601F0E3
:10E4800045FC584601F047FC042384F88F347EB9DC
:10E49000012384F821344FE101F045FC0028F6D037
:10E4A000404601F034FC404601F036FC0523ECE721
:10E4B0003B7805935B09013B062B00F21782DFE8EE
:10E4C00013F00700150295001502920015020602CE
:10E4D000102EDDD995F830311297F6B28DF84C60D8
:10E4E000002BD5D11CA804F021F912AA1CA9FF20E9
:10E4F00002F09EF89DF85830C3F3030307468DF8E9
:10E500002C3095F8480095F87D308DF82D30072295
:10E510000BA902F090FA002F5DD100285BD09DF886
:10E5200053309DF852201599C5F8E4101B0443EAB6
:10E5300002239DF8512002201343C5F8E03004F077
:10E5400003F99DF8583095F8480085F82E71C3F30B
:10E550000212C3F3030385F8703085F878309DF814
:10E56000593085F86920012B38BF01234FF47A72A6
:10E570005343AB651344EB650DF15A034FF00108AB
:10E580001093113E94F81B348DF83C300FA985F898
:10E5900068808DF8446002F056FA0223404685F800
:10E5A000303101F077FD18B14146384601F038FDB1
:10E5B00094F88F34012B00F2A78194F81A34002BC1
:10E5C00040F09A8194F8913443F0100384F8913428
:10E5D000FEF786FD64E6012001F05CFD0028E7D02F
:10E5E00001210720E2E7012384F8203495F87D30EB
:10E5F0008DF82E3094F824348DF82D3095F88C3029
:10E6000095F848000D330BA98DF82C3002F000FA74
:10E61000A6F10D031BB2099023EAE37300B2834213
:10E620003FF736AF0B2E7FF633AFBA4B25931CA8BE
:10E63000FF231C978DF874608DF8983002F0C4F8B1
:10E64000074600287FF424AF95F81831012B13D129
:10E6500001F067FB002872D0384601F057FB3846BE
:10E6600001F059FB04239DF87C101E9884F88F3428
:10E67000C1F3001101F06EFB9DF87C301E99C4F8C7
:10E68000341413F00F0203D09DF89000002862D1DB
:10E690009DF89800002861D0002A7FF4F9AE9DF81B
:10E6A0009020002A14BF4FF003084FF00208002208
:10E6B0000A92D5F8EC2095F8E900914251D1002852
:10E6C0004FD0D5F80C1195F8EAB009680A9195F881
:10E6D0001811022902D1032184F88F14B8F1030F15
:10E6E0007FF4D6AE13F0600F7FF4D2AE0492012710
:10E6F00095F82E31BBF1000F36D0BBF1010F13D1CD
:10E70000012B33D16FF0090646FA08F606F0010630
:10E71000C6F10206F6B2BDF87E100AAA304601F034
:10E7200011FE38B3072823D0012384F821340A9B33
:10E73000C4F83034C4F86C34FEF720FDB0E501F0C5
:10E74000F2FA002898D0384601F0E1FA384601F094
:10E75000E3FA052387E74FF00008A8E74FF0010828
:10E76000A5E74FF0010BC3E70426D4E70326D2E761
:10E770000823DAE71CAB009304990A9B32465846FB
:10E7800001F0A2FE20B1022814BF0B230A2380E669
:10E790000A9BC4F83034C4F86C349DF87C3084F89B
:10E7A0002104C3F3401384F82E3484F8443494F8DD
:10E7B0008F3484F82274012B9EBF0122A86285F851
:10E7C0001E21012FC4F8280484F82C0484F8410485
:10E7D00038D1022284F8202495F83A20002A4AD120
:10E7E0009DF87C20D60646D4012B94F840149DF861
:10E7F0007C2005D8012901D1900601D501F04CFB00
:10E80000B8F1020F94F88F3443D0B8F1030F0AD057
:10E810009DF87C10B8F1010F4A4601F00F0120A8C5
:10E820003BD0FFF745F99DF8903084F82334259BC1
:10E83000C4F828349DF8983084F82C34012384F8E7
:10E840002D3430E0059A02F0E002A02A1BD195F8A1
:10E850002E11012285F83A2009B927996963012B05
:10E8600084F8202407D9D5F89020C4F83C24DAF89D
:10E870000020C4F8982495F81821002AB4D1012268
:10E8800084F82524B0E7002285F83A2084F8202473
:10E89000A6E79DF8981025984A46FFF709F99DF8D4
:10E8A000903084F823349DF89020E02A08D195F820
:10E8B0001F312BB984F82324C4F82834A4F82C344D
:10E8C00094F8913443F0020384F8913470E6114DCA
:10E8D000013EB2B2791C284604F000F80323A4F8E4
:10E8E0002034C4F8285484F82C64E9E7012384F820
:10E8F0002134FEF743FC5BE694F84434002B3FF4EC
:10E9000061AE0020FEF726FC94F88F34022B3FF412
:10E910005FAE57E6D031002094F89134590715D5F1
:10E92000012001F0B7FB60B1012001F08BFB08B9B9
:10E9300084F81804D4F8403323F00203C4F84033B9
:10E9400004E0062001F0A6FB0028F3D194F89134EE
:10E95000DA077FF5FAAC94F840240AB1032A18D1FB
:10E960001D4A94F8181492F86820914205D29B072A
:10E9700023D594F88F34012B1FD8184806F0C6FA17
:10E98000D4F8403323F02003C4F84033FFF744FBAE
:10E99000DBE4012A11D194F81924002A3FF4D5AC04
:10E9A0000D4A94F8181492F868209142E5D29F0716
:10E9B00003D594F84434002BDFD194F8913400202F
:10E9C0006FF3041384F8913484F81904FFF746FBBD
:10E9D000BBE429B0BDE8F08FD4290020003300202B
:10E9E0002DE9F04F89468DB090460746002800F08B
:10E9F0008F81002900F08C810368002B00F0888152
:10EA00004368002B00F084818368002B00F0808134
:10EA1000C368002B00F07C81104601F0F5FF002850
:10EA200000F07881BD4CBE4D384601F0AFFA40F29F
:10EA3000C4520021204603F065FF40F21C52002121
:10EA4000284603F05FFFB74BC4F82C3104F5097377
:10EA5000089304F50A7300264046099308A9B24BAF
:10EA600084F848800A9384F8186184F88C608DF8E3
:10EA70002C6001F0DBFF0F2306A994F848008DF805
:10EA8000183001F0C5FF801B18BF01204FF00A0BA2
:10EA900084F81C0106A994F848008DF818B001F01C
:10EAA000B7FF4FF0060A84F8DC0006A994F8480086
:10EAB0008DF818A001F0ACFF102384F8DD0006A942
:10EAC00094F848008DF8183001F0A2FF1123C4F823
:10EAD0009C0006A994F848008DF8183001F098FFC2
:10EAE0001223C4F8A00006A994F848008DF8183045
:10EAF00001F08EFF1323C4F8A40006A994F848007F
:10EB00008DF8183001F084FF1423C4F8A80006A97A
:10EB100094F848008DF8183001F07AFF1623C4F8F5
:10EB2000AC0006A994F848008DF8183001F070FF89
:10EB3000172384F8B10006A994F848008DF818301E
:10EB400001F066FF18230DEB0301C4F8B400C4F80C
:10EB5000BC0094F848008DF8183001F059FFC0B29D
:10EB60001D2384F8B80084F8C00006A994F8480072
:10EB70008DF8183001F04CFF1E2384F8C40006A95C
:10EB800094F848008DF8183001F042FF1F2384F8F4
:10EB9000C50006A994F848008DF8183001F038FF38
:10EBA0002023C4F8C80006A994F848008DF818304E
:10EBB00001F02EFF0B23C4F8CC0006A994F84800FE
:10EBC0008DF8183001F024FF0C2306A9A4F8D0001A
:10EBD00094F848008DF8183001F01AFFD4F89C30F2
:10EBE0006365D4F8A030A365D4F8A430E365D4F805
:10EBF000A83023664FF00108D4F8AC300590A4F893
:10EC0000D200636684F8B080C4F894B084F898A009
:10EC1000C4F84CB084F850A084F8688084F81F8150
:10EC2000C5F84893FEF7AEFDC5F84473C4E90B661A
:10EC30003E4B84F8198185F89164C5F840833246CB
:10EC40004FF0FF31009605F55A7006F001F9384B88
:10EC5000009632464FF0FF3105F5607006F0F8F887
:10EC6000344B009632464FF0FF3105F5667006F0E2
:10EC7000EFF802AF304B009632464FF0FF3105F50A
:10EC8000806006F0E5F8384606F076F897E803006D
:10EC900004F5927383E80300284B294F1E60294B2B
:10ECA000C5F84C33284BC5F85433284BC5F85C33B2
:10ECB000274BC5F85033274BC5F8583305F553702B
:10ECC0003B68984704F5A67003F04CFB20B1112671
:10ECD00030460DB0BDE8F08F204601F003FB002860
:10ECE000F5D101F039F8B8B91B4801F04DFB0646E3
:10ECF0000028ECD17B69984703F0CEFDBB6D94F8FA
:10ED000019019847FB6A9847012385F89234DFE799
:10ED10000326DDE70926DBE71326D9E7D4290020FF
:10ED2000982F002000040001802300205DE00008EF
:10ED300025D900086DD9000855D100087C23002092
:10ED40006078030815D30008C9D2000811D1000863
:10ED5000A1D2000879D20008BC2A002008B5034BD4
:10ED60000020C3F84003FEF7BBF908BD982F002030
:10ED700010B5FFF7ABF90A4C60B90A4B93F818319C
:10ED8000022B02D1084BDB6A98470123C4F84033B9
:10ED9000002010BDD4F84003013818BF0120F8E767
:10EDA000982F0020D42900206078030838B5124C31
:10EDB000204606F0ABF804F1180006F0A7F804F1BD
:10EDC000300006F0A3F804F1980006F09FF800F078
:10EDD000AFFF0A4B0025DB6A984744F8285CFEF732
:10EDE000EDFD0749074840F2C45203F077FD0123C7
:10EDF00044F8283C284638BD0033002060780308DA
:10EE0000D42900201024002070B52E4B8AB005466E
:10EE100093F8DD008DF8090093F8DC008DF80A0006
:10EE200029489A6A90F81804039200268DF80B007E
:10EE300004960C46002940D00692D3F88820079209
:10EE40001A8F93F81A118DF8151052BAADF82020C8
:10EE500093F87C2093F848308DF8243003AB8DF87C
:10EE600022008DF8232000930DF10A020DF10B030F
:10EE70000DF1090105A88DF8146000F0D7FE9DF989
:10EE80000900FEF74FF9607004A801F01BF8B0B953
:10EE9000049A0F2A0DD863789A420AD81544AB42D7
:10EEA000A3EB02012CBF002001202170C0000AB09A
:10EEB00070BD002323700820F9E70320F7E7132033
:10EEC000F5E700BFD4290020982F00201FB5044685
:10EED000002800F010810378412B00F20781DFE861
:10EEE00013F0420049004D005100550059005E00EA
:10EEF00005010501050105010501050105010501E2
:10EF0000650069006D0078007F00820085008A003E
:10EF100088008C0090009300960099009C009F0050
:10EF2000AE00B200BA00B600BE00C100C500CE00FF
:10EF3000CA00CC000501D20005010501050105014B
:10EF40000501050105010501050105010501050191
:10EF5000050105010501DA00DE00E200E700EB0033
:10EF6000EF00F300FC00664B93F81831237100208A
:10EF700004B010BD624B93F83031F7E7406803F0FE
:10EF80008FFBF4E7406803F0D1FBF0E75C4B93F8AC
:10EF90001A31EBE75A4BD3F8E0306360E7E7584BA0
:10EFA000011D93F8300103F0D9FBE0E7544B93F8CF
:10EFB0001931DBE7524B93F88C30D7E71C238DF8DF
:10EFC00008304F4B02A993F8480001F021FD606022
:10EFD000CDE74C4B043493E8030084E80300C6E714
:10EFE000494B0434F7E7494B0434F4E7484B043405
:10EFF000F1E71A23E3E71923E1E7414B93F868307F
:10F00000B4E73F4B5B6DC8E73D4B9B6DC5E73C4BA1
:10F01000DB6DC2E73A4B1B6EBFE7394B5B6EBCE75B
:10F0200002238DF80830364B02A993F87C2093F820
:10F0300048008DF80A2001F0EBFC207197E7304B77
:10F0400093F8DD3092E72E4B93F839308EE72C4B56
:10F0500093F8DC308AE72A4B93F8383086E7284B60
:10F06000DB6C9AE7264B93F850307FE7244BD3F8BC
:10F07000843063607BE7224B8FE7264B8DE7204B84
:10F08000D3F8CC30F5E71E4BD3F82C31436001F0B8
:10F090004DFDA0606BE71A4BD3F890307DE7184B1D
:10F0A00093F81F3162E7164BB3F88830A3805EE710
:10F0B000134BB3F88A30F9E7114BB3F8D030F5E7CA
:10F0C0000F4BB3F8D230F1E70D4B93F848200AB15B
:10F0D000062A12D1B3F8A035E8E7094B93F8482087
:10F0E0000AB1062A09D1D3F8A43556E704B0BDE821
:10F0F000104000F021BE03203AE7182038E700BF97
:10F10000D4290020402A0020882A0020482A0020F4
:10F11000902A0020102400207FB5044610B9032057
:10F1200004B070BDA34DD5F840339A0700F16F824B
:10F130000278412A00F26882DFE812F042004700BC
:10F1400055005B005F006400690076008100870065
:10F150008D00930099009F00A500AB00B5006602EA
:10F16000BA00DC00EF0016013801290142014B0111
:10F170004F01530157015B0166025F017101990163
:10F180008701AB01B101B801BD01C20166022802CD
:10F19000660266026602660266026602660266022F
:10F1A000660266026602660266026602660266021F
:10F1B000340239023E02430248024D0252025C020E
:10F1C0000079FEF773FA30B1AAE70379022BA6D0D3
:10F1D000794A82F8303195F8913443F0200385F86C
:10F1E000913400209CE7406803F04CFA0028F2D0EC
:10F1F00095E7406803F08AFAF8E76F4B027983F8E5
:10F200001A21E8E76C4B4268C3F8E020E3E76A4E56
:10F21000416896F8300103F097FA00287FF47FAF39
:10F220006368C6F8E430D6E7416800293FF477AF59
:10F23000002001F0DDF90028CDD0112070E74168F1
:10F2400000293FF46CAF0120F3E7416800293FF447
:10F2500066AF0820EDE7416800293FF460AF092060
:10F26000E7E7416800293FF45AAF0C20E1E7416825
:10F2700000293FF454AF0D20DBE7416800293FF43B
:10F280004EAF0E20D5E7416800293FF448AF0F206C
:10F29000CFE74A4C484B007983F81901A36D984792
:10F2A000E36A984797E7444B027983F88C2092E70A
:10F2B000414E037A8DF8043096F8480096F87D3078
:10F2C0008DF80530072201A901F0B5FB00283FF4B5
:10F2D00026AF636896F848000193002201A901F067
:10F2E000AAFB00283FF41BAF6C36D4E9010186E885
:10F2F000030070E7304E037A8DF8043096F848002A
:10F3000096F87D308DF80530072201A901F093FBB6
:10F3100000283FF404AFB436E7E7274E037A8DF8B0
:10F32000043096F8480096F87D308DF805300722B5
:10F3300001A901F080FB00283FF4F1AED4E90101FE
:10F3400006F1740383E8030096F81831022B7FF46A
:10F3500042AF96F83031002B3FF43DAF174BDB6ADC
:10F360009847FEF775F936E7134E037A8DF80430A7
:10F3700096F8480096F87D308DF80530072201A9EF
:10F3800001F059FB00283FF4CAAEBC36ADE7436834
:10F39000029301238DF80C30074B02A993F8480023
:10F3A00001F056FB00287FF416AFB8E643680293DD
:10F3B0000023EFE7982F0020D4290020607803086D
:10F3C00003795A1E0E2A3FF6AAAE934A82F8683095
:10F3D00001E7914B42685A65FDE68F4B42689A659A
:10F3E000F9E68D4B4268DA65F5E68B4B42681A66A2
:10F3F000F1E6894B42685A66EDE6874C037994F84A
:10F4000048008DF80430062201A901F014FB002801
:10F410003FF485AE9DF8043084F8DD30DBE67E4CA9
:10F4200003798DF8043094F8480094F87C308DF816
:10F430000630052201A901F0FEFA00283FF46FAE64
:10F440009DF8043084F83930C5E6734C037994F89C
:10F4500048008DF804300A2201A901F0ECFA0028D6
:10F460003FF45DAE9DF8043084F8DC30B3E66A4CBE
:10F47000037994F848008DF80430092201A901F0BD
:10F48000DAFA00283FF44BAE9DF8043084F83830A7
:10F49000A1E6614B4268C3F89420DA649BE65E4BB8
:10F4A000027983F8982083F8502094E65A4B4268FA
:10F4B000C3F884208FE6584B4268C3F8CC208AE614
:10F4C000012B40F0A480554C2421204603F01CFA67
:10F4D000636A984201D0172022E61C2104F128001B
:10F4E00003F012FA636C9842F5D14FF4807104F185
:10F4F000480003F009FAD4F848319842EBD1D421FE
:10F5000004F5A67003F000FAD4F820329842E2D154
:10F51000002104F5097003F0F7F9D4F82432984279
:10F52000D9D14FF4607104F50A7003F0EDF9D4F805
:10F53000A8359842CFD1142104F2AC5003F0E4F97D
:10F54000D4F8C0359842C6D1334E2146304640F2F9
:10F55000C45203F0C3F9204640F2C452002103F024
:10F56000D1F995F81B3485F8E833736FC5F8EC339F
:10F5700096F87D3085F8F83340F20123A5F8FA3388
:10F58000274B96F819019B6D984724E68379012B48
:10F590003FF6C5AD204B42684068C3F82C2100F00F
:10F5A000BDFE48E61C4B4268C3F8902013E61A4B98
:10F5B000027983F81F210EE6174B8288A3F8882072
:10F5C00009E6154B8288A3F88A2004E6124B82884C
:10F5D000A3F8D020FFE5104B8288A3F8D220FAE5EB
:10F5E0000D4B93F848200AB1062A12D1A288A3F83D
:10F5F000A025F0E5084B93F848200AB1062A08D167
:10F600006268C3F8A425E6E500F098FBDBE501207D
:10F6100086E5182084E500BFD429002010240020AE
:10F62000607803082DE9F04387B00023ADF800307F
:10F630000646002800F0EE800361FEF747FD20B18A
:10F640000124204607B0BDE8F08300F065FD0028E6
:10F65000F6D100F05BFD014618B96F48142203F0A3
:10F6600051F96E4D95F89134012243F0040385F869
:10F67000552485F8913433788DF804300021013B0E
:10F680008DF80520ADF806100C2B00F2BB80DFE8EA
:10F6900003F007B9B9B97982B9B990B9AD9AA9009F
:10F6A000D5F8407317F02007CAD196F80480B8F156
:10F6B000020F46D1DFF868815A4CFEF763F896F9DD
:10F6C000051098F848003A4601F00FFA88F839001A
:10F6D000B37988F83830384607238DF80530FDF7C0
:10F6E000E5FFFF2304F58670A5F80C31C5F8084145
:10F6F00085F8047103F01AF804F58A7002F0D0FF5F
:10F700003846FDF72DFE0446002839D096F905103D
:10F7100098F84800012201F0E8F988F83900D5F896
:10F7200094343361002C71D000F0F0FC002888D1B3
:10F7300095F8913485F81A0460F3820385F89134C2
:10F740007FE7B8F1010F4FF00204E8D1DFF8D09065
:10F750008DF8144099F8480089F81D7102A901F04C
:10F7600065F9337989F830318DF805708DF80680A8
:10F77000FDF7C4FC95F8913443F0100385F89134FB
:10F780000024CCE700226946022000F0F3FA0028AA
:10F79000F6D01324C3E7244BB288DB6B96F90C1028
:10F7A000B0689847D5F8403343F00203C5F84033BA
:10F7B000E6E702A90D2000F053FB0028E0D000226C
:10F7C00069460D20E1E7164B93F81831D3B9347927
:10F7D00004F0070000F0ABFA8DF800400122694602
:10F7E0001020D2E7002269461220CEE78DF80720CC
:10F7F00000F08EFA044638B900F087FA204600F08F
:10F8000089FABDE702248AE7012488E701A800F00D
:10F81000D1FB16E7032414E7EC330020982F0020D7
:10F82000D42900209A2F0020607803082DE9F04F9A
:10F8300099B08046059118B9032019B0BDE8F08F42
:10F8400000230361FEF742FC0446002840F0A58037
:10F8500046460FCE0EAD0FC51422524898F800A0B0
:10F86000B8F80C7098F90EB04F4E214603F04AF8E4
:10F870004E4B012283F8412496F83021022A254676
:10F880000BD196F81821022A07D196F81E2122B929
:10F89000BAF1010F38BF4FF0010ABAF1010F2BD0B6
:10F8A000BAF1030F2AD0BAF1000F33D102229DF82A
:10F8B0003C30DDF84090029362F34715012496F83E
:10F8C0007C108DF8321002220CA996F848008DF8B1
:10F8D000302001F09DF896F81A3196F830C196F86C
:10F8E0001D1140B2002B63D0BCF1010F57D100298C
:10F8F00055D1002C61D153E00422D8E70023DDF874
:10F900003C90BDF840709DF942B0029365F01F0530
:10F910000124D4E74FF0000BD946CDF808B0CEE76C
:10F920004FF0010084F81A04D2E005F29A420BA9C4
:10F9300000F0D4FA002800F015811320049B3387CF
:10F940001A4B002283F81A2423E105F29A452A462D
:10F950000BA900F0C3FA0028EFD10B9B84F8280113
:10F96000C4F82C5184F83031FCE0B9F1000F00F0FC
:10F97000F980002A00F0F6804946E01C02F0AEFF54
:10F9800094F8373201332380ECE01220D6E70220CE
:10F99000D4E70720D4E71320D2E701204DE7FCB9D4
:10F9A0000220F6E0D8330020D4290020982F002030
:10F9B000002CF5D05845B8BF584696F87C308DF8E5
:10F9C0002000052296F848008DF8223008A901F0A1
:10F9D00032F800283FF430AF9DF8203086F83930F7
:10F9E0006F4A704BD2F89804D3F8904038B105F0C4
:10F9F00053FA6C4B84423CBF002283F83A20198FA3
:10FA00001A8F93F830010491996A099152BA00282B
:10FA1000BFD093F81B0100B9186393F81801ADF833
:10FA20005820013893F87C2093F81A411491D0F1B2
:10FA3000000BD3F888108DF85B204BEB000B93F88C
:10FA4000482093F83A0093F868308DF85A3009ABA3
:10FA50000093554B03904FF001008DF84C00159129
:10FA60008DF85C20A3F12F01A3F1300213A88DF8CB
:10FA70004D4000F0DBF8039B4FEA0B1B4BEA431BA6
:10FA800000264BEA801B4BEAC413B145444C039358
:10FA900008BF37463A46494604F59C70CDE90A66E8
:10FAA0009B46268084F81A6402F018FFE9B2A5701C
:10FAB000C5F34215FAB2042D3A4E039B84F837225F
:10FAC0003FF42EAF072D3FF450AF022D7FF45FAF10
:10FAD000364D84F80D110420029984F80401FF20AA
:10FAE00084F80C0184F8281184F81431D6F8E41055
:10FAF000C4F8085105F59B730AA8C4F8101184F8DE
:10FB00003021C4F82C3100F011FC00287FF43DAF07
:10FB10000A9BA4F844040BA8A4F81631C4F84C348A
:10FB200000F0D0F900287FF408AF0B9BD3B196F911
:10FB30003900FDF7F7FA94F83732002B3FF405AFA0
:10FB40000B9B0F2B3FF6F1AE05F58B720BA90F2027
:10FB500000F0C4F900287FF4F0AE0B9B63F3030BB5
:10FB600084F814B10598FDF7FBFB00287FF4E6AE9E
:10FB7000099B86F83A00B36200F080F900287FF410
:10FB80000AAF94F8913484F840A443F0010384F858
:10FB90009134034BD3F89434C8F810304DE600BFCD
:10FBA000982F0020D42900203C2A00209A2F0020E2
:10FBB00037B50B4D8DF8040004460F2295F8480028
:10FBC00001A900F038FF40B1064A85F81C4192F8BF
:10FBD000913443F0200382F8913403B030BD00BF6C
:10FBE000D4290020982F002010B5FFF7C1F8044653
:10FBF00088B90A4805F08AF9094805F087F90948E3
:10FC000005F084F900F094F8FDF7BCFD064BDB6AC3
:10FC10009847204610BD0124FBE700BF00330020B9
:10FC20001833002030330020607803082DE9F04FAE
:10FC30008BB047780093149B90F90C8090F90D607D
:10FC400090F80EB08A464168196004469146002F2C
:10FC500058D002238DF8103004A9C37B007C8DF8A6
:10FC6000123000F0D5FEB4F808C0618943B2606874
:10FC7000984545466144B8BF1D46604534BF0027DE
:10FC80000127884209D30A218DF81010207C0193A6
:10FC900004A900F0BDFE019B46B2B4F808C060891B
:10FCA00061680CEB400E714519D3A1EB0C01B1FB5F
:10FCB000F0FC00FB1C1191B9984503DC2378CBB90B
:10FCC0004FF0010B21238DF81030207CE37B8DF861
:10FCD000115004A98DF8123000F09AFE45B2009B35
:10FCE0008AF80050384689F8006083F800B00BB0FD
:10FCF000BDE8F08F0223207C8DF8243006A900F0A7
:10FD000095FEDDE74546EAE7704770477047704764
:10FD100000207047704770477047002070470020F0
:10FD200070470020704700207047002070477047E0
:10FD300070477047022070470220704702207047CA
:10FD400070470020704770477047002070470020C0
:10FD5000704770477047704710B5054C4FF40372F9
:10FD60002046002102F0CEFD0020C4E9000010BDB5
:10FD7000B43400202DE9F8438146904600293CD058
:10FD80001F4C2023224604F1100012F8017F6FBBA4
:10FD90008242FAD11B4E3368013403B93460736870
:10FDA00003B11C6000252560C4F8088074601FFA48
:10FDB00088F284F80490601D02F090FDB9F1110FF3
:10FDC0004FF0000398BF104D6373D6F8083298BF08
:10FDD00025FA09F503F1010398BF05F00105434435
:10FDE0002573C6F808323846BDE8F883013B13F0A6
:10FDF000FF030446C6D10227F5E70127F3E700BF5A
:10FE0000BB340020B43400202007020010B518B322
:10FE1000124A1368984204D103681360002305E076
:10FE20000B46002BFAD019688842F9D151688842F4
:10FE300008BF53600BB101681960D2F808328168BD
:10FE4000013B00245B1A04602146C2F808321022EC
:10FE500002F058FD204610BD0120FCE7B43400201C
:10FE6000054B1B6813B11A798242FAD1002B0B6043
:10FE70000CBF032000207047B434002010B5054BA0
:10FE8000186800B910BD037B04680BB9FFF7BEFF0B
:10FE90002046F6E7B434002038B5084B084C186803
:10FEA00000B938BD03790568112B05D824FA03F38E
:10FEB000DB0701D5FFF7AAFF2846F1E7B43400209D
:10FEC0002007020028B1044BD3F808320360002059
:10FED00070470120704700BFB43400202DE9F04185
:10FEE00007460E46154642B339B3154B1C6800232E
:10FEF0002CB93046FFF7E6FF0020BDE8F081A2688C
:10FF0000F91A0132914215D32279EA54581C2289F8
:10FF10005FFA80F8611D55FA80F002F0DFFCA368FB
:10FF2000246898445FFA88F3E2E720462568FFF7E3
:10FF30006DFF2C46002CF8D1DBE70120DDE700BF88
:10FF4000B43400200238C0B211289ABF014B185CAB
:10FF5000002070477B71030830B50B4B93F82020CD
:10FF60000446084672B100211C330578A54208D02A
:10FF700001319842CDB214BF04301038AA42F4D8EF
:10FF8000002030BD1046FCE7C036002010B5084CFC
:10FF900000232060142204F10C00FF2184F820309B
:10FFA000C4E9010002F0AEFC012384F8213010BD49
:10FFB000C036002010B50E4A92F82010042915D83A
:10FFC000936804781C7044785C70C478807898706A
:10FFD0000131DC7082F8201002F11C018B4214BF49
:10FFE000043302F10C039360012010BD0020FCE7F4
:10FFF000C0360020094B93F8200068B15A6803F11D
:020000040801F1
:100000001C018A4200F1FF3014BF043203F10C02DC
:1000100083F820005A600120704700BFC0360020DE
:1000200010B5074B93F820200446084632B15968B2
:10003000FFF792FF10B101234470837010BD00BF21
:10004000C036002008B5064B93F820202AB1596825
:10005000FFF782FF08B1407808BD0120FCE700BF30
:10006000C036002030B50A4A92F82010536882F852
:10007000210061B1916801241C32DD78587005B906
:100080009C70934214BF0433103B9942F5D130BDAC
:10009000C036002008B5044B5968FFF75DFF0038F3
:1000A00018BF012008BD00BFC0360020F7B50422EC
:1000B000154E044600210DEB020096F8207002F068
:1000C00021FC0025EBB29F4201D803B0F0BD73685C
:1000D000197821705A786270987838B13368204660
:1000E0009B689847FFF786FF0135EBE7DB788DF8D3
:1000F00004108DF805208DF80730FFF77BFF01A86D
:10010000FFF758FFF0E700BFC0360020014B93F81F
:1001100020007047C0360020034B93F820000428CD
:1001200094BF002001207047C03600201FB5002476
:10013000CDE90244C41F8DF800408DF801100C0A6F
:10014000ADF80420090C120C8DF803108DF8062070
:100150008DF8073002461B0A012168468DF80240DF
:100160008DF8083002F029FA002818BF0E2004B0DC
:1001700010BD2DE9F04188B090460D460F9A074614
:10018000002847D000240121CDE904448DF8101047
:100190009DF838108DF81510ADF81630190CCDE912
:1001A00000441B0ECDE902448DF81930ADF81A2039
:1001B000130C120E07948DF818108DF81C308DF862
:1001C0001D20E3B21E01002DF6B203DC002008B0B2
:1001D000BDE8F081013310218DF81F3042466B4697
:1001E0000DEB010002F07FF90346A8B9102D284657
:1001F0003E44A8BF10206946327811F801CB013384
:1002000082EA0C02984206F8012BF5DC103D2DB273
:100210000134D6E70920DAE70E20D8E701380328B1
:1002200015D8DFE800F002080C100A4B1B681B69A8
:100230000B6000207047074B1B685B69F8E7054BB4
:100240001B689B69F4E7034B1B68DB69F0E705203B
:10025000704700BFE43600202DE9F041C4B00C46E1
:100260004A9E17461D468046B8B3B1F5807F36D802
:100270004FF488720021684602F044FB4923009342
:100280004FF48073ADF804302B0C8DF80830330C2C
:10029000ADF80650ADF80A608DF80C302246002308
:1002A000414604A82D0E360E8DF80E308DF80950FB
:1002B0008DF80D608DF80F4002F010FB04F1100175
:1002C0004B9A3B4689B2684602F0F7F810B1012814
:1002D00018BF0E2044B0BDE8F0810920FAE70D20D8
:1002E000F8E7000010B590B10A4C282200212060E8
:1002F00002F008FB2368084A1A6000204FF0FF3222
:10030000C3E90302C3E90522C3E9072210BD08209F
:10031000FCE700BFE436002000010101024B1B682E
:1003200018600020704700BFE436002030B1044B55
:100330001B68DB68013303600020704709207047A9
:10034000E436002013B500230C460193CAB101A97D
:10035000FFF764FF18B9019B591C02D1146002B069
:1003600010BD99B2611A002901DD5C18F6E702D1CF
:1003700013600720F3E71B0C1B0403F580331C44B8
:10038000ECE70920EBE7000028B1044B1B681C33A5
:100390004362002070470920704700BFE436002008
:1003A0001FB5044600B3002303A8039302F05CF9D1
:1003B000104ABDF80C30126820469380E38200F0AA
:1003C0005EFA98B904F118030093216801231322FF
:1003D00002F068F860B9204600F051FA003818BF02
:1003E0000120000104B010BD0920FBE71020F9E74F
:1003F0000E20F7E7E4360020F0B5054687B01C462E
:1004000013B9092007B0F0BD2E4E3368DB68834274
:1004100055D894F82020002A0CBF082209228342D4
:1004200005D3204600F05FFA68B11020EAE7002308
:1004300001900093A36894F82810606AFFF799FE72
:100440000028EED0DEE723792168B4F808C0A76859
:10045000043B9AB20029D4D0B2F5807F2DD8ADF8F4
:100460000EC08DF817304FEA174C04F12C033F0EE5
:100470008DF8117000932F0C08234FF0490EADF842
:100480000C008DF814708DF816002F0E0DEB030084
:10049000CDF808E08DF810C0ADF812508DF8157049
:1004A00002F000F808B10E20ACE7204600F01BFA7D
:1004B0000028BAD13368DD60A4E70D20A2E706204A
:1004C000A0E700BFE43600202DE9FF410A9D8046E9
:1004D0000F4616461C46002D5AD0002303A910468D
:1004E0000393FFF79BFE18B1062004B0BDE8F0812E
:1004F000039B9C4201D80133F6D1284600F064F9F1
:10050000002847D1264B1A78424503D01A79424534
:1005100042D10120AA68BA4240D103EB8002EB6AC3
:1005200092F801802979CDE900430439927828684E
:100530003B4689B2FFF790FE0028D6D195F82030CF
:100540000194002B4FF00103009314BF4246082290
:1005500095F82810686A3B46FFF70BFE0028C4D1C7
:10056000013E032EC1D8DFE806F002070B0F0D4B4A
:100570001B681C611C62B8E70A4B1B685C61F9E7E9
:10058000084B1B689C61F5E7064B1B68DC61ACE718
:100590000920AAE70F20A8E70B20A6E70220A4E77E
:1005A00024040020E43600201FB50B294FF000037F
:1005B000CDE90033CDE902330A4607D00C2914D027
:1005C0000A2910D00A2005B05DF804FB012802D1E9
:1005D00020238DF800300021684601F0EEFF00284E
:1005E00018BF0E20EFE73023F3E70B21F4E70000FC
:1005F00038B5054601F0DCFF044610B10E24204654
:1006000038BD002DFBD1094B1B680B219878FFF7F3
:10061000CBFF0028F2D10C21FFF7C6FF0028EDD157
:100620000A21FFF7C1FF0028E9D0E7E7E436002000
:100630002DE9F04380468FB00C461746002A6BD058
:10064000002969D0002529461D2206A805951DF020
:1006500091FF8DF81350344D2B680DF114099E88CD
:10066000CDF804900DF1130302933B7900933B689E
:1006700032462146404601F0BCFF00284ED1386882
:100680003A79494602F02AF9384600F04FF8002836
:1006900046D13C7AFA79BB79240444EA02241C430B
:1006A0002B689A6894423DD99C609DF813000B21F9
:1006B000FFF77AFF034658BB0C21FFF775FF03468F
:1006C00030BB0A21FFF770FF034608BB7B7ABA7A7A
:1006D000FF7A3F0447EA02271F433A463346214642
:1006E0000920FFF723FD034690B933463A462146D9
:1006F0000820FFF71BFD034650B92A689DF8131028
:1007000091700021D1604FF0FF31C2E90411916175
:1007100018460FB0BDE8F0830923F9E70E23F7E789
:100720000F23F5E70323F3E7E436002010B5044672
:10073000002845D00168002942D011F8013B4371DF
:100740000322063002F0CAF82046032250F8091BA3
:10075000043102F0C3F82168CB79E3600A7A43EAF6
:100760000223E3604A7A43EA0243E3608A7A43EA77
:100770000263E360CB7A23740B7B63742379212BB0
:100780001AD110220D3104F1120002F0A7F81D2237
:100790002168501C8B5C6362085C43EA0023901C58
:1007A0006362085C033243EA004363628A5C43EAA3
:1007B00002636362002010BD112B03DC0D22E7E70A
:1007C0000220F8E70120F6E710B50446002854D0CF
:1007D0000168002951D00B7843714B7883608A7887
:1007E00043EA02238360CA7843EA024383600A79BA
:1007F00043EA026383604B7903738B79C381CA79BF
:1008000043EA0223027BC38102F00F020831103059
:1008100002F064F8237B002203F00F0384F8202009
:1008200084F82820227903F10800111A04290DDD2B
:1008300021680933043AD21A085C84F82000D2B245
:10084000606A84F82820194402F048F82379226865
:100850001A44002012F8043CE36212F8031C43EA35
:100860000123E36212F8021C43EA0143E36212F837
:10087000012C43EA0263E36210BD0220FCE710B5DD
:10088000044660B3036853B30279162A29D9427922
:100890001A700146082251F8060B013002F028F8C0
:1008A0002146082251F80E0B093002F021F8236886
:1008B000E28A5A74E38A22681B0A93742368A26945
:1008C000DA74A36922681B0A13752368628B5A7550
:1008D0002368E27E9A7517232371002010BD012042
:1008E000FCE70220FAE738B50446002863D0016827
:1008F000002960D0037B90F8282003F00F03002A22
:1009000057D10833207904321344984255D3637980
:100910000B702368A2685A70A36822681B0A937040
:1009200023686289DA702368E27A1A712368227B6D
:100930005A712368E2899A71E38922681B0A214669
:10094000D371227B51F8100B02F00F02083001F036
:10095000C5FF237B94F8282003F00F0303F108055B
:100960002AB1226894F82010515503F10905206836
:1009700094F82820616A284401F0B0FF94F82830E8
:100980002268E16A2B44D1545A1CE16A206892B271
:10099000090A81549A1C2168E08D92B28854DA1CAD
:1009A000216894F82F0092B20433885423710020F8
:1009B00038BD0933A6E70120FAE70220F8E7000076
:1009C000024B1A8810431880704700BFE836002099
:1009D00008B5074B1B883BB1FEF7CAF9002814BFC6
:1009E0006FF00200002008BD6FF00100FBE700BFC0
:1009F000E836002010B5034B00241C80FEF7AEF94A
:100A0000204610BDE8360020B0FA80F0400970475B
:100A100082B018B9084602B000F0CAB8002002B08F
:100A2000704710B9084600F079B9704710B9084608
:100A300000F090B970470346084611460BB900F024
:100A4000DDB90020704710B9084600F039BD704785
:100A500010B9084600F0FEB90020704710B40446F3
:100A6000084611461A46019B14B910BC00F00CBA96
:100A700010BC70470346084611460BB900F036BA61
:100A80000020704710B40446084611461A4614B9AF
:100A900010BC00F0A3BA002010BC704730B405466B
:100AA000084611461A46DDE902341DB9029430BCED
:100AB00000F022BB002030BC704710B9084600F09F
:100AC000D3BB0020704710B9084600F037BD0020A6
:100AD000704710B9084600F0E2BB0020704710B91B
:100AE000084600F0DFBB0020704703460846114669
:100AF0000BB900F0F9BB0020704710B4044608465B
:100B000011461A46019B14B910BC00F0EFBB092036
:100B100010BC704710B40446084611461A4614B972
:100B200010BC00F02DBDC8B210BC70470048704723
:100B300001000102064B10B51B6A0446984730B10C
:100B40000448054B204498428CBF0020012010BD72
:100B500060780308403576C9405DC600F0B5114B9A
:100B600085B00C4610491F56054601F017F80F4B8B
:100B7000E4B25E6A072D4FF00103CDE9024301465E
:100B80000AD105220023CDE900234FF47A727A437B
:100B90001846B04705B0F0BD08220020CDE900207E
:100BA0003A46F5E74872030828720308607803089C
:100BB0001FB5002300930378013B372B21D8DFE8D2
:100BC00003F01C242020201E202020204143454EDD
:100BD0002055585B5E6164206C1E6E73787A7D20B0
:100BE0007F8326202020202020202020202020203D
:100BF00085878C2020858C208E92C3780BB10223B0
:100C00000093009805B05DF804FB8378F6E743781D
:100C10008DF8043007238DF805308378003B18BF2A
:100C200001235B008DF8063010238DF80730314B1F
:100C30001B6801A803F55872CDE9022300F08EFF6E
:100C40000090DEE74023DBE72023D9E7827890F9A4
:100C5000013012B9284AD35CD2E7284AFBE78278F0
:100C600090F90130002AF8D1254AF4E740F6B8336C
:100C7000C6E74FF47A73C3E74FF4FA63C0E741F273
:100C80008833BDE741F27073BAE71E484FF47A71BA
:100C900001F008FE00F5FA60D2E71B4BB0E7154BF8
:100CA0001B6803F55873ABE7124B1B6803F55B73C6
:100CB000A6E71023A4E70F4B1B68A1E701239FE7DA
:100CC0004FF0834300939CE7104BFBE7104B97E7F3
:100CD00040F21113ADF8003093E7032390E790F949
:100CE00001300C4AB7E70C4990F9010000F056FFBB
:100CF000A6E700BFF03600201D7203080D7203083E
:100D00001572030818FCFFFF00EA06379A9909409C
:100D100040F70937487203082872030837B50B4BB0
:100D200002781B680C2101FB02335B7A03EB43045E
:100D3000074B1D6803690093C3684278816805EB1F
:100D4000C40000F0A7FC03B030BD00BFF0360020A7
:100D5000EC36002030B587B0027B6423ADF800305C
:100D6000012A4FF00003CDE90133CDE903338DF8BB
:100D700002308DF8143028D0022A2FD01ABB036815
:100D80000BB34368FBB11A4C80682360194B1822DF
:100D90006946186001F0A2FD174B246893E807002C
:100DA0000C3384E8070093E8070004F10C050323E3
:100DB00085E80700A4F86C33012204F55B7104F5A3
:100DC000587000F058FC07B030BD0949086843600E
:100DD000036100F55B7100F55870F2E7044B1B6886
:100DE000B3F86023B3F86C130A43A3F86023EAE76F
:100DF000F0360020EC360020981B030808B50346A7
:100E00000A2924D8DFE801F006232323230B161B2D
:100E100023212100BDE808400068FFF78BBE90F950
:100E200000009978072271B900F0E5FB003818BF7F
:100E3000012008BD052293F900000021F4E790F994
:100E400000005978EEE70221EEE70722F3E70020E1
:100E5000EFE7000008B502791AB1012A0BD0002093
:100E600008BD084B01681B68012203F5587000F0AB
:100E700002FC0120F4E7034B01681B6803F55B707B
:100E8000F5E700BFF0360020F7B50728144D1C46E3
:100E9000A8BF072058700E462946174600F07EFE70
:100EA00094F90130A070072B13D1322000F076FDA9
:100EB0000C4BDB6D0546984704F10C0208340346E1
:100EC000019200943A463146284600F06CFD03B08A
:100ED000F0BD054A55F82310D05C00F057FDE7E758
:100EE0002872030860780308487203082DE9F04F60
:100EF000344F90F901607B68D0F804908BB00446C1
:100F0000884698470546002859D1E37C73B92E4A94
:100F10002378126803EB4303990002EB8303D3F8B1
:100F20000490B9F1000F01D152F80190274B4846C7
:100F300013F906B0FB689847A37C2289D7F818A05C
:100F40000993072E28D100230121CDE90223204A4D
:100F50000693CDE90431CDE907330521CDE9002120
:100F60004FF47A7202FB0BF24CF250311846D04724
:100F7000637C13B3174B995D7B6D0D31C9B2284665
:100F80009847E07C3246494600F01AFE88F8006037
:100F900001200BB0BDE8F08F002101250823CDE929
:100FA0000013CDE90715CDE90511CDE90311029232
:100FB000A1782B465A462846D9E7074BDBE70020A5
:100FC000E7E700BF60780308F036002048720308A6
:100FD00085450100157203081D7203082DE9F04FC5
:100FE0008DB090F90130DFF8FCA0DFF8FC90CDE97E
:100FF0000A123E4A12F903B00278DAF800300C25E2
:1010000005FB02333A4A5B7A126803EB430302EBB7
:10101000C303044693F9021090F9020000F0B9FDF1
:101020003449064694F9010000F0B8FDA2686168F1
:101030008046304600F0DFFC2178DAF80020D9F84D
:101040000C306943074650589847D9F81C309C46E5
:1010500094F901300025072B4FF47A63CDE907534B
:10106000CDE905552DD10123CDE903530523CDE964
:1010700001534FF47A7303FB0BF300933946434655
:1010800046F2A81228466746B8472378DAF80020C7
:101090000C214B4394F90110D05800F0B3FDA18905
:1010A00094F90100FFF75AFD0B9B217B1860D9F8DA
:1010B0005430284698470A9B01201E700DB0BDE8A9
:1010C000F08F01200823CDE90350CDE901032A4622
:1010D000CDF800B0654643463946A847012005468D
:1010E000D3E700BFF0360020607803084872030899
:1010F000EC360020287203082DE9F04F8FB0002451
:1011000005468A46914698460494ADF81440ADF8D9
:10111000024007264FF0010B2B7AA34206D96868DC
:1011200004A9204400F0CAFB00285DD102238DF8F9
:10113000083002A86B7A8DF80A30FFF739FDAB7AD8
:101140008DF81D309DF811308DF81E309DF812304D
:101150008DF81F309DF810308DF82030EB7A8DF827
:1011600021302B7B8DF822306B7B8DF823301023C0
:101170008DF81C608DF824303A4E8DF82C000DF15E
:1011800002030A93072332688DF82D30ADF834300E
:101190002B680C9206930DF1120204AB0DF11101B4
:1011A00006A800F0A5FB072805460BD130680C22E5
:1011B000002100F5587001F0A5FB3368BDF802204E
:1011C000A3F860239DF811308AF800309DF81230A2
:1011D00089F800309DF8103088F80030189B2846B8
:1011E0001C700FB0BDE8F08F9DF81330BDF814707F
:1011F000ADF802702044C4B2F3B917B3194A002005
:101200001168072602464FF00C0C062B1BD10CFB75
:1012100000FE51F80EE0BEF1000F04D00BFA00F210
:101220003A4397B2012201301028EED1002A3FF450
:1012300073AFADF802706FE75A1E042A01D9062B6E
:10124000DCD0062668E747FA00FE1EF0010FEAD060
:101250000CFB00FE51F80EE0BEF1000F08BF0626A1
:10126000E1E700BFF036002038B505464068FFF7DB
:1012700061FC0722841D002195F90000E4B200F012
:10128000BAF908B904F0FD0495F90100072200211C
:1012900000F0B1F908B904F0FB04204638BD002085
:1012A0007047000010B503780F2B044618D840682B
:1012B000FFF740FC22780B4902EB42020968831CCD
:1012C00001EB820051F82220DBB21AB903F0FD03D2
:1012D00058B210BD032B06BF626842600223F7E7D5
:1012E0000020F6E7F0360020022070472DE9F0419B
:1012F0003A4D0446286896B00E46904600211F4697
:101300000122032300F55870CDE90411CDE906113F
:101310008DF80C108DF80D10ADF80E3000F08DF931
:1013200030B92A68B2F8603343F00303A2F860339F
:101330002A68637A8DF8203002F55871CDE90912D8
:10134000274A94F9083012680B921022ADF8302029
:101350000DF10E020D9222680E9262680F92D4E98E
:101360000301A27A8DF8402001228DF8412011AAB4
:1013700082E80300227DE18A8DF8213018468DF83D
:101380004C20FFF7EBFB08AB15930DF10D03149008
:101390000093CDF8048003AB04AA39460EA800F0F0
:1013A00099FB044678B99DF80C10013901F07AFADE
:1013B00000F158030DEB030010F8483C3370204651
:1013C00016B0BDE8F0810C2801BF2A68B2F860337E
:1013D00043F00303A2F86033F1E700BFF0360020CA
:1013E000EC360020F8B50679012E054648D90F2EB7
:1013F00048D80368187A40F303000722002140B25E
:1014000000F0F9F82B680446187A40F3031007221D
:10141000002140B200F0EFF8B8B1B4FA84F46409E6
:1014200029680B7A086843F3030243F303135BB2A2
:1014300052B29A42C8BF0124FFF77CFB80F001033F
:10144000DBB224B10533D8B2F8BD0124E8E7DBB93B
:101450000E4F29683B6806EB460003EB80000C2228
:1014600001F03CFA3A680C2303FB062320465C7229
:10147000B2F860130123B3400B43A2F86033E3E7F3
:101480000620E1E70320DFE70420DDE7F036002057
:1014900010B4017801290ED9084B18680C234B436E
:1014A000C4180022C250C4E9012200F5587010BCD3
:1014B000102200F0A9B8002010BC7047F0360020C0
:1014C0002DE9F04186B050238DF81430037A102BAB
:1014D000074630D14368DD7B6DBB0224A8466426F5
:1014E000062C14D87A68535D03932A44517843EA52
:1014F00001230393927843EA02437343CDE903380F
:1015000063B968468DF80040FFF7C2FF0DE0CDF8E3
:101510000C808DF81480CDF81080F2E703AB01A8A1
:1015200001938DF80840FFF75DFF0134E4B2102C01
:1015300005F10305D4D106B0BDE8F0811FB50268FE
:101540000379116849B901A88DF80430FFF7A0FFAD
:1015500078B1032005B05DF804FB02A802928DF873
:101560000C30FFF73FFF042805D0052805D00028E0
:10157000EFD00020EEE70220ECE70120EAE70000D0
:10158000C90020B9034B0B449856C0B27047024BB8
:10159000F9E700BFCD7103088D710308F0B59A42D9
:1015A000069D03DB9DF914309A4220DD0020F0BD3A
:1015B00003EB430331F814C005EB830300264CFA18
:1015C00006F7FF0707D51F7A07F00F0E964502DCD6
:1015D000B2EB171F0DDD0136102E03F10C03EED117
:1015E0000134E4B22301DBB29842E1D8DEE7002403
:1015F000F8E70120DBE7884204DB9042CCBF002003
:10160000012070470020704710B51409B4EB111F7A
:1016100003464FEA11100ED391420CD202B201F0F0
:101620000F0133F81240012000FA01F124EA010110
:1016300023F8121010BD0020FCE7F0B528B100EB34
:10164000410501270020914200D3F0BD002435F868
:1016500002CB234607FA04F636EA0C0608BF01332C
:1016600004F1010408BFDBB2102CF3D1184401319E
:10167000C0B2C9B2E7E710B500B149B910BD31F841
:10168000134020F813400133DCB2A242F7D8F5E74B
:101690000023F9E782B030B504880493D2B9B3F5DA
:1016A000616F15D349F6AF2542F21072AB4298BF75
:1016B0004FF47A72944238BF14466143BDE830401B
:1016C000C3688B428CBF5B1A0023C36002B07047B3
:1016D0006422EFE7012C38BF0124EEE72DE9F04F3B
:1016E0008FB01546199F03939DF8603007930C4601
:1016F000804603F0C7FB6A4A0590A7F5F633303BF6
:10170000B3FBF2F3534303F5F63B0493182313FBA7
:1017100005430BF1300B069300254FF0FF3A069B73
:101720009C4207D1002D14BF50464FF0FF300FB040
:10173000BDE8F08FBDF96830ADF8243009991997EC
:101740003846089703F02EFB2688B8F1000F5FD1CA
:10175000B7F5616F5AD349F6AF2242F21073974240
:1017600098BF4FF47A739E4238BF1E46642E59D1FB
:10177000DFF83091A060A1680CA803F035FB0D9B49
:101780000093DDE908120C9B0AA803F08CFA039A77
:101790000A9B0AB9079A2AB122694A4502D1424AEC
:1017A00093420ED9414BC4F80C909F4209D90023B3
:1017B000ADF82C300B99CDF828B0584603F0F2FA6A
:1017C000A060606808B9C4F80C90C4F81090B8F133
:1017D000000F04D003F060FBE3680344E360D4E946
:1017E00003329342059B88BFE26063601B9BE16804
:1017F0007343994204D20398E8B9B8F1000F1AD0A4
:1018000001231D442375EDB2183488E76423AAE749
:10181000039B0BB9234BE360012EDFF8889038BFA0
:101820000126CEE7B6F57A7F0ABFDFF88490DFF8AD
:101830008490A0609FE700209342207506D85B1A31
:101840009A4505F1010528BF9A46EDB2B8F1000F9F
:10185000DAD1642E184AADF82C801DD049F6B02399
:10186000B6F57A7F18BF1346974281BF049A02F5F6
:10187000A83202F5C0729B180A931A9B00930AAE15
:1018800096E80600199B304603F00DFA96E803002F
:1018900003F088FA8246B7E74FF46163E4E700BFDC
:1018A0008051010040771B007F5101002FEC0100A7
:1018B00080A81201002E930230EC01000378032B64
:1018C00014D1437803F00F021B098A704B708378A0
:1018D0008B80C27843EA02238B800379C3F3021220
:1018E00003F00F03CA700B7005207047002070478B
:1018F0002DE9F3479A464379057990F907609146B7
:10190000044690F906208846D3B190F90870002D5E
:1019100037D00F2A1BD194F909200F2E27D194F923
:101920000A00072D02D1002F08BF012788F80020E8
:1019300089F8000028468AF8007002B0BDE8F087F8
:1019400090F90B7090F9092090F90A60DFE7A3691C
:10195000019394F91530009394F914302169207B98
:10196000FFF71CFE0028D8D105F0FD05D5E794F956
:101970001D00B042D5DC94F91C30B34203DA05F007
:10198000FB053046D2E73046CBE70000024B03FAB6
:1019900000F0B0FBF1F0704740420F004FF4FA53F3
:1019A000B3FBF0F0704730B54FF47A750C1F6A4303
:1019B00000FB042252001EBF00F1FF341219B2FBDB
:1019C000F0F2914238BF1146039A116082004843F9
:1019D0001CBF013040084FF47A71121A01FB132327
:1019E000002BCABF03F2E73393FBF1F1B3FBF1F134
:1019F000049B196030BD38B5400014460D46F0F721
:101A0000D9FA01462846F0F723FA2146F0F720FAE2
:101A1000EFF79AFE1EF0BCFEF0F79EF940B238BD1B
:101A20002DE9F74F019300239C469E46048A1E0130
:101A3000F6B2B44246D906EB46054FEA4309AD007B
:101A40000024476837F809702741FF0729D58768C0
:101A500007EB050A7F5927B3077837B9476927B1DC
:101A600037F809702741FF071BD59AF8087090F9DD
:101A700001B047F303084FFA88F8D84511DC47F363
:101A800003177FB25F450CDB9AF8097007EB470834
:101A9000C76807EBC8073F7D5FB90CF1010C5FFA1F
:101AA0008CFC0134102C05F10C05CAD10133DBB2DA
:101AB000BCE70EF1010706EB040801F80E805FFA9F
:101AC00087FEEEE7019B82F800E083F800C003B0D8
:101AD000BDE8F08F2DE9FF4704464068DDE90C675B
:101AE0001D468A46914603F0D7F923681B1A3B60CE
:101AF0004FF000080123337085F80080636813B14C
:101B00002368834224D8D4F81CC0CAF80080A36993
:101B10009CF800E00393D4E9030101AB83E80300E0
:101B2000237D0093DCF80C10237A627A7046FFF76D
:101B3000D5FD334638602A46E0694946FFF770FF15
:101B40002B782BB1C7F80080002004B0BDE8F087E7
:101B50003378002B0CBF0C200B20F6E737B590F93B
:101B6000002090F90250954204460FD0013A52B23B
:101B700095420BD0A368019394F9013000936168FA
:101B8000E0782B46FFF70AFD0028EFD0104603B09F
:101B900030BD8842B8BF08467047000051F82000A9
:101BA000054B984205D0054BC31A58425841400096
:101BB00070470120704700BF90D0030020A10700AC
:101BC00005281FB50ED80C4B53F820300093CDE9F3
:101BD00001120A4B01220021022002F06BFE05B027
:101BE0005DF804FBCDE90012054B01220021022023
:101BF00002F060FEF3E700BFB872030850720308FA
:101C00006F72030807B5054BCDE9000101220021E1
